:020000040800F2
:10000000205C0020DDCE00087DC800087FC8000805
:1000100081C8000883C8000885C8000800000000E7
:1000200000000000000000000000000087C8000879
:1000300089C80008000000008BC800088DC80008AF
:1000400031CF000835CF000839CF00083DCF000878
:1000500041CF000895C8000845CF000849CF0008E7
:100060004DCF000851CF000855CF000859CF0008E8
:1000700097C80008A1C80008ABC80008B5C80008A8
:100080005DCF000861CF0008BFC8000865CF000839
:1000900069CF00086DCF000871CF000875CF000848
:1000A00079CF00087DCF000881CF000885CF0008F8
:1000B00089CF00080000000000000000C9C8000847
:1000C0008DCF000891CF000895CF000899CF000888
:1000D0009DCF0008A1CF0008A5CF0008A9CF000838
:1000E000ADCF0008B1CF0008000000000000000004
:1000F0000000000000000000000000000000000000
:1001000000000000B5CF000800000000B9CF0008D3
:100110000000000000000000D3C80008DDC800088F
:10012000BDCF0008C1CF0008C5CF0008C9CF000867
:10013000CDCF00080000000000000000000000001B
:10014000D1CF0008D5CF0008D9CF000800000000AB
:10015000DDCF0008E1CF0008E5CF0008E9CF0008B7
:10016000EDCF0008F1CF0008F5CF00080000000037
:10017000F9CF0008FDCF00080000000000000000DB
:1001800001D0000805D0000809D0000881B000F5B2
:10019000E0700268914203D343681A44914202D34B
:1001A00080680028F5D101B07047DFF8681708684B
:1001B00090B94FF4805048604FF480324FF0FF30D8
:1001C0008A60C86008610420DFF84C27DFF84C37EC
:1001D0004861C2F8BC010B600120704701F10803BF
:1001E00013F0070F0EBF0023C3F1080303F007034A
:1001F0001944D21A8161C26042F001034B60091DAB
:1002000028238B50DFF80C170A69C26170472DE96B
:10021000FC4B074601F1080010F0070F0FBF89469D
:10022000C0F1080000F0070001EB000902F108012D
:1002300011F0070F06D002F10800C0F1080000F02D
:10024000070002441546A5EB090009EB0306A0EBE5
:10025000030B43F00303C9F80430AE4228BF01F09A
:10026000FFF92879C10758BF01F0FAF9BBF1100F67
:1002700038BF01F0F5F9B869854207D1F8685844EC
:10028000F860BE6140F00100706050E1786985421D
:100290000AD1B8688344C7F808B07E614BF001000A
:1002A000706046F80BB042E1686800F00301012974
:1002B00040F0AB80C008C0000190C0081F2839D8AA
:1002C000AC68D5F80C800090454508BF01F0C8F92E
:1002D000A54208BF01F0C4F968680099C008C000D1
:1002E000B0EBC10F18BF01F0BBF9009907F128006E
:1002F00000EBC100844206D03A699442C0F080808D
:10030000E168A9427CD1A04506D100983968012254
:1003100082409143396075E0804506D03869804558
:100320006ED3D8F80800A8426AD1C4F80C80C8F887
:10033000084067E0EC68D5F81880AC420CD0A8689B
:100340003969884222D3C168A94204BFA168A94281
:100350001CD1C460A0601BE005F11402146834B91C
:1003600005F1100214689CB101E01A46146804F10A
:1003700014031968002902BF04F11003186800284B
:10038000F3D139698A4228BF106001D201F068F9BF
:10039000B8F1000F36D0E96907F5987000EB8100DD
:1003A0000268954208D10460A4B9E869796801221D
:1003B00082409143796025E03869804508D3D8F8B8
:1003C0001000A84214BFC8F81440C8F8104001E05B
:1003D00001F046F9B4B139698C4211D3C4F81880E0
:1003E000286928B1884226BF2061846101F038F96C
:1003F000686938B13969884202D36061846101E07B
:1004000001F02EF901982D188344686840084000D7
:1004100068604BF0010171604FEADB0446F80BB0F5
:100420001F2C23D807F1280000EBC4084546BBF178
:10043000100F38BF01F014F9386820FA04F1C90729
:1004400005D4012101FA04F404433C6007E0D8F824
:100450000800396988422CBF054601F001F9C8F847
:100460000860EE60B560C6F80C8060E05FEA1B20B3
:1004700008BF002123D0B0F5803F28BF1F211ED226
:10048000A0F58072120C02F008029040A0F5805195
:10049000090C01F004018840A0F580431B0CC2F157
:1004A0000E0203F00203521AD21A984002EBD03225
:1004B000D01D2BFA00F101F0010101EB420107F51B
:1004C000987202EB8100F1610022726132617A68F8
:1004D00022FA01F3DB0707D4012303FA01F11143E8
:1004E00079600660B0611DE002681F291DBF4908E0
:1004F000C1F119010BFA01F1594600E002465068BA
:10050000C008C000584516D002F11003CC0F03EB11
:100510008403490018680028F0D13869834204D365
:100520001E60B261F660B66001E001F099F809F171
:100530000800BDE8F68B396990688A4228BF884276
:10054000F3D3C6609660B060F2600020B061EEE761
:100550002DE9FE4F04468B46A5692E4690469946E6
:100560003146FFF713FEA8F128020168406801EB4D
:10057000000AAAF1270111F007000EBF0021C1F106
:10058000080101F007010AEB0100A0F12F0706F1B5
:100590001000874238BF374607F1180001905946CE
:1005A000002000902046FFF719FE07F1080010F028
:1005B000070F18BF01F054F81B20786007F10801FD
:1005C00004F5E07090E80C5081E80C50C0F800B0E1
:1005D000C0F80480C0F80C9081600198009900E098
:1005E000001D07224260491C00F108025245F7D362
:1005F0000129D8BF01F034F8B74200F09580BF1B45
:10060000301D311DC05940084000C85147F001015C
:1006100071604FEAD70BF751BBF11F0F21D804EBE4
:10062000CB0000F12805A846102F38BF01F018F8BC
:10063000206820FA0BF1C90705D4012101FA0BF15A
:100640000843206006E0A868216988422CBF8046E4
:1006500001F006F8AE60C8F80C60C6F80880F560D6
:100660006FE0380A08BF002123D0B0F5803F28BFD3
:100670001F211ED2A0F58072120C02F008029040D9
:10068000A0F58051090C01F004018840A0F58043D9
:100690001B0CC2F10E0203F00203521AD21A984048
:1006A00002EBD032D01D27FA00F101F0010101EB7D
:1006B000420104EB8102002302F59870F16173613D
:1006C0003361626822FA01F3DB0707D4012303FADE
:1006D00001F1114361600660B0611DE002681F29ED
:1006E0001DBF4908C1F1190107FA01F1394600E0BF
:1006F00002465068C008C000B84216D002F110038C
:10070000C80F03EB8003490018680028F0D1206966
:10071000834204D31E60B261F660B56011E003B09D
:10072000BDE8F04F00F09CBF0BE0216990688A4261
:1007300028BF8842F3D3C6609560B060F2600020A5
:10074000B06103B0BDE8F08F2DE9F041714F05466F
:100750003868884608B9FFF728FDB96801EB08003A
:100760002F30491E20EA010188457DD205F5D87653
:10077000B06828B1326889188A4275D2884273D32A
:1007800000F07EFF01001CBF0C6811F1010F6BD05F
:100790003068201805F5D87230605368984238BF29
:1007A00018467060A86960BB286908B1814200D210
:1007B0002961316174610020F06105F12802386817
:1007C00068624FF0FF3028620020D260926002F130
:1007D000080353611361801C10322028F5D34E4862
:1007E000854208BFA4F1280228D055F8040CC0089F
:1007F00005EBC002A2F108000A19121A283A0146B4
:100800001CE005F5E070024600E092687AB31368D8
:1008100057683B449942F8D1137B1F0727D4AB6933
:100820001768BB4223D3D2F804C06744BB421ED230
:10083000A444C2F804C0E868A96922182846FFF752
:10084000CDFC1FE08068C0B103689342FAD1027BFF
:10085000130712D4026801604368E41844604346F9
:100860002846BDE8F041D2E40020BDE8F0812A69C5
:10087000914238BF29610A19E5E70023224628463C
:10088000FFF766FEE8688045EED2A0EB0800A96994
:10089000E86001EB0802AA6140F00100506048F0F6
:1008A0000300486001F10800BDE8F08138B4194B3D
:1008B0001A6882B94FF480525A604FF480344FF076
:1008C000FF329C60DA601A610422134C134D5A61A6
:1008D000C4F8BC211D6011F1400F17D28269AAB182
:1008E000C368283199420BD200F5E0710C68A2422E
:1008F00003D34D682C44A24202D389680029F5D164
:10090000C16999423CBF4FF0FF31C16132BC002048
:10091000704700007C240020781D00206859883C26
:100920002DE9F84F00258946090AC9F1000B08BFD7
:10093000002323D0B1F5803F28BF1F231ED2A1F58D
:100940008072120C02F008029140A1F580531B0C3A
:1009500003F004039940A1F58044240CC2F10E0277
:1009600004F00204D21A121BA14002EBD132D11DB5
:1009700029FA01F303F0010303EB4203074607F5ED
:10098000987858F8230030B31F2B0FBF4C465C08F3
:10099000C4F1190409FA04F4AC46594600E06400B5
:1009A0004268D208D200A2EB09028A4203D21100A7
:1009B000054600F06881426910304FEAD47B50F858
:1009C0002B00002A1CBF824294460028E7D18B46A8
:1009D0006046B0BBBDBB012000FA03F35B00584288
:1009E00003437868034000F04D81584203405B1E8A
:1009F000180B00F01000C340590901F00801CB406A
:100A00009A0802F00402D3405C0804F002040818BB
:100A1000E3401018C3F3400620183044F3401B187D
:100A200058F823000DE008464168C908C900A1EB49
:100A3000090159453CBF8B46054601690029F2D1A1
:100A400040690028F0D1002D00F01C81B868A0EBAF
:100A50000900834580F0168138698542C0F0108115
:100A60006868C008C00009EB0B01884218BF00F09D
:100A7000F7FD05EB0906B54280F00281EC68D5F878
:100A800018A0AC420CD0A8683969884222D3C1684A
:100A9000A94204BFA168A9421CD1C460A0601BE0A8
:100AA00005F11402146834B905F1100214689CB100
:100AB00001E01A46146804F114031968002902BF02
:100AC00004F1100318680028F3D139698A4228BF5D
:100AD000106001D200F0C4FDBAF1000F36D0E96910
:100AE00008EB81000268954209D10460200014D10E
:100AF000E8697968012282409143796026E038698B
:100B0000824508D3DAF81000A84214BFCAF814408E
:100B1000CAF8104001E000F0A3FDBCB1386984427E
:100B200012D3C4F818A0286930B13969884226BFA9
:100B30002061846100F094FD686938B139698842A8
:100B400002D36061846101E000F08AFDBBF1100F07
:100B50000CD2D94449F003006860291D281D50F8C3
:100B6000090040F0010041F8090088E049F0030065
:100B700068604BF0010070604FEADB0046F80BB094
:100B80001F281DD807EBC00101F12804396821FA9C
:100B900000F2D207A34605D4012202FA00F008436E
:100BA000386006E0A068396988422CBF834600F0AF
:100BB00057FDA660CBF80C60C6F808B0F4605EE0A4
:100BC0005FEA1B2008BF002123D0B0F5803F28BF7B
:100BD0001F211ED2A0F58072120C02F00802904074
:100BE000A0F58051090C01F004018840A0F5804374
:100BF0001B0CC2F10E0203F00203521AD21A9840E3
:100C000002EBD032D01D2BFA00F101F0010101EB13
:100C10004201F16100227261326108EB81007A6861
:100C200022FA01F3DB0707D4012303FA01F1114390
:100C300079600660B0611DE002681F291DBF490888
:100C4000C1F119010BFA01F1594600E00246506862
:100C5000C008C000584518D002F11003CC0F03EBB8
:100C60008403490018680028F0D13869834204D30E
:100C70001E60B261F660B66001E000F0F1FC13E1C5
:100C800000F0EEFC0DE18B46A3E6396990688A42DC
:100C900028BF8842F1D3C6609660B060F260002041
:100CA000B061ECE72DE9F84F064688467168484286
:100CB0000140491E080B00F01000C1404A0902F033
:100CC0000802D1408B0803F00403D9404D0805F019
:100CD00002051018E9401818C1F34004281806F559
:100CE000987A2044E14009185AF821104868C00851
:100CF000C0000D46A0EB080909E001464868C0089D
:100D0000C000A0EB080048453CBF81460D4608697D
:100D10000028F2D149690029F0D130698542C0F03C
:100D2000BE806868C00808EB090BC000584518BFB2
:100D300000F096FC05EB08008542009080F0AF8043
:100D4000EF68AC69AF420CD0A8683169884222D301
:100D5000C168A94204BFB968A9421CD1C760B86084
:100D60001BE005F11402176837B905F11002176886
:100D70009FB101E01A46176807F1140319680029AA
:100D800002BF07F1100318680028F3D131698A42C5
:100D900028BF106001D200F063FC002C31D0E9695B
:100DA0000AEB81000268954208D107608FB9E869B3
:100DB0007168012282409143716022E0306984426F
:100DC00005D32069A84214BF6761276101E000F0E4
:100DD00047FCB7B13069874211D3BC61286930B193
:100DE0003169884226BF3861876100F039FC686943
:100DF00038B13169884202D37861876101E000F03F
:100E00002FFCB9F1100F0BD24BF003006860291DC5
:100E1000281D50F80B0040F0010041F80B003DE0A8
:100E200048F00301696049F00100291D41F80800FC
:100E3000009840F80990D6F808804FEAD80BBBF12B
:100E4000200F28BF00F00CFCB8F1000F22D006EBF9
:100E5000CB00776900F12804A246B8F1100F38BF23
:100E600000F0FEFB306820FA0BF1C90705D4012120
:100E700001FA0BF10843306006E0A068316988424E
:100E80002CBF824600F0ECFBA760CAF80C70C7F8D4
:100E900008A0FC60C6F808900098706104E000F0BB
:100EA000DFFB0020BDE8F28F05F10800BDE8F28FFE
:100EB0002DE9FE4F0546AFF30080F52DDFF89C6766
:100EC00080F004810B2D31BF10250B35ED08ED00AE
:100ED0003068EC08E04010F0030F46D0C04300F04B
:100EE0000100041906F1280000EBC408E700D8F857
:100EF00008506868C008C000B84218BF00F0B0FBD6
:100F0000D5F80890454508BF00F0AAFB4D4508BF3D
:100F100000F0A6FB6868C008C000B84218BF00F027
:100F20009FFBC84507D13168012000FA04F421EA8B
:100F3000040434600DE03069814508D3D9F80C0011
:100F4000A84204D1C8F80890C9F80C8001E000F06C
:100F500087FB47F003006860291D281D05F1080480
:100F6000C05940F00100C851F8E0B168A94280F0D2
:100F7000BE80002800F0A1804FF0010808FA04F1BB
:100F8000490000FA04F4484201430C406042044026
:100F9000641E200B00F01000C440610901F008013C
:100FA000CC40A20802F00402D440630803F002031C
:100FB0000818DC401018C4F3400718183818FC4013
:100FC000241806F1280000EBC40AE700DAF80890BC
:100FD000D9F80400C008C000B84218BF00F040FBB8
:100FE000D9F808B0D14508BF00F03AFBD94508BF91
:100FF00000F036FBD9F80400C008C000B84218BFA2
:1010000000F02EFBDA4506D1316808FA04F421EA33
:10101000040434600DE03069834508D3DBF80C002C
:10102000484504D1CAF808B0CBF80CA001E000F0A4
:1010300017FB45F00300C9F804007F1B09F1040108
:1010400047F00100485109EB05000190C751B46811
:101050004FEAD40ABAF1200F28BF00F001FB34B3E5
:10106000CDF800A006F12800756900EBCA0AD34646
:10107000102C38BF00F0F4FA3168009821FA00F221
:10108000D30704D408FA00F00843306007E0DAF828
:101090000800316988422CBF834600F0E1FACAF8A3
:1010A0000850CBF80C50C5F808B0C5F80CA0B760D4
:1010B00009F108040198706150E07068C0B32946D6
:1010C0003046FFF7EFFD040011D047E015F1400F67
:1010D00028BF4FF0FF350AD20B35ED087068ED00E0
:1010E00028B129463046FFF71BFC040036D1B06812
:1010F000A8421DD3411B726910290AD3501970618F
:10110000B16041F001034360415045F00305556073
:101110000BE00021B1607161131D40F003015160CB
:10112000111D095841F00101195002F1080415E0A0
:10113000F06885420DD2401BB169F0604A19B26176
:1011400040F00100506045F003054D6001F10804D6
:1011500004E029463046FFF7F7FA0446AFF3008073
:101160002046FFF7EEBA002800D170472DE9FC4772
:10117000A0F10805AFF30080DFF8E0643269954222
:10118000C0F05982686800F00301012900F0538221
:10119000C1084FEAC109C10705EB090839D42C6819
:1011A00010F0030F00F04982604205449542A144CB
:1011B000C0F041827069854200F0C780E408202CAD
:1011C0005ED2D5F80CA0AF68554508BF00F048FACC
:1011D000BD4208BF00F044FA6868C008C000B0EB28
:1011E000C40F18BF00F03CFA06F1280000EBC40061
:1011F000874205D031698F423FD3F968A9423CD17B
:10120000BA452CD13068012101FA04F420EA040423
:101210003460454580F00F82D8F80440E00740F183
:101220000A82A00700F16881B069804540F0A08083
:10123000F068B5618144C6F80C9049F0010068601F
:101240007069854202D100207061B060F069484544
:1012500080F0F38100213046FFF728FBEDE1824565
:1012600006D03069824508D3DAF80800A84204D1D4
:10127000C7F80CA0CAF80870CBE700F0F1F9C8E78E
:10128000EC68AF69AC420BD0A868904223D3C16828
:10129000A94204BFA168A9421DD1C460A0601CE09E
:1012A00005F114031C6834B905F110031C68A4B1DE
:1012B00001E063461C6804F1140CDCF800100029FE
:1012C00002BF04F1100CDCF800000028F1D19342B9
:1012D00028BF196001D200F0C3F9002F99D0E96945
:1012E00006F5987000EB81000268954209D1046010
:1012F000200011D1E8697168012282409143716038
:1013000087E73069874205D33869A84214BF7C61FA
:101310003C6101E000F0A4F9002C3FF47AAF3169A0
:101320008C42AAD3A761286928B1884226BF2061D0
:10133000846100F095F9686900283FF46AAF31696B
:1013400088429AD36061846163E798F8040000F0F2
:10135000030003287FF45DAFC6F8089049F001014F
:10136000D8F8040040084000C8F8040069600AE0AA
:10137000706980450AD1B06875618144C6F80890EB
:1013800049F00100686045F8099056E1E408E4007E
:10139000A144E408202C3AD2D8F80CA0D8F8087060
:1013A000D04508BF00F05CF9B84508BF00F058F917
:1013B000D8F80400C008C000B0EBC40F18BF00F09C
:1013C0004FF906F1280000EBC400874207D03169CD
:1013D0008F42C0F08480F968414540F08080BA4572
:1013E00007D13068012101FA04F420EA04043460D2
:1013F00077E0824506D031698A4570D3DAF8080073
:1014000040456CD1C7F80CA0CAF8087069E0D8F85C
:101410000C40D8F8187044450DD0D8F80800316950
:10142000884222D3C168414504BFA16841451CD10F
:10143000C460A0601BE008F11402146834B908F11C
:10144000100214689CB101E01A46146804F11403F8
:101450001968002902BF04F1100318680028F3D1AD
:1014600031698A4228BF106001D200F0F9F8002FDC
:1014700037D0D8F81C1006F5987000EB8100026890
:1014800090450AD10460200012D1D8F81C00716880
:10149000012282409143716023E03069874205D385
:1014A0003869404514BF7C613C6101E000F0D8F828
:1014B000BCB131698C4212D3A761D8F8100028B1B1
:1014C000884226BF2061846100F0CAF8D8F8140071
:1014D00038B13169884202D36061846101E000F073
:1014E000BFF849F00100686045F8099070698542CD
:1014F0000BD1C6F80890A0E064086400C8F8044066
:1015000049F00100686045F809904FEAD907202F9B
:1015100022D206F1280000EBC704A046B9F1100F53
:1015200038BF00F09DF8306820FA07F1C90705D4EC
:10153000012101FA07F70743376006E0A068316927
:1015400088422CBF804600F08BF8A560C8F80C508C
:10155000C5F80880EC6070E05FEA192008BF002140
:1015600023D0B0F5803F28BF1F211ED2A0F5807286
:10157000120C02F008029040A0F58051090C01F015
:1015800004018840A0F580431B0CC2F10E0203F059
:101590000203521AD21A984002EBD032D01D29FA17
:1015A00000F101F0010101EB420106F5987202EB36
:1015B000810000226A612A61E961726822FA01F3FE
:1015C000DB0707D4012303FA01F1114371600560C1
:1015D000A8611DE002681F291DBF4908C1F119015A
:1015E00009FA01F1494600E002465068C008C0000F
:1015F000484526D002F11003CC0F03EB84034900C9
:1016000018680028F0D13069834204D31D60AA61B4
:10161000ED60AD6001E000F023F8306A401E3062FA
:101620000BD1D6F8C80100E080680028FCD14FF04B
:10163000FF30306201E000F013F8AFF30080BDE846
:10164000F387316990688A4228BF8842E3D3C56036
:101650009560A860EA600020A861DEE7781D0020A0
:10166000012000F023B88268521C8260426832B1C7
:101670000268531C036011704168491E4160704745
:101680000749086808B1002070470648C008C00034
:1016900008600549C908C900091A0160704700BF00
:1016A00038250020275C00202091002080B5AFF372
:1016B0000080024A11001820ABBEFBE726000200A2
:1016C00080B5DFF87C0901F05AF9DFF87829DFF8F6
:1016D000781901F05CF9DFF8740901F050F9DFF8CE
:1016E0006429DFF8641901F052F9DFF8640901F0A8
:1016F00046F9DFF85029DFF8501901F048F9DFF812
:10170000540901F049F9DFF83C29DFF84C1901F0E0
:101710003EF9DFF8480901F03FF9DFF82829DFF842
:10172000381901F034F9DFF8380901F035F9DFF83C
:101730001429DFF8241901F02AF9DFF8280901F04B
:101740002BF9DFF80029DFF8101901F020F9DFF894
:10175000FC0B01F029F901BD10B592B0012148221E
:10176000DFF804394820414319446C46200001F059
:101770005BF96946DFF8D80B01F0AAF9002012B036
:1017800010BD00000EB418B5A0B00200002023ABBD
:101790009121684602F086F804004FF47A73200025
:1017A000020092B26946DFF8AC0B02F0D6F82000D6
:1017B00021B010BC5DF810FB38B5DFF8841B0C6855
:1017C000DFF87C1B0968491CDFF8742B11600A21C3
:1017D000B4FBF1F201FB1244DFF8945B02F074FEFB
:1017E00045F8240031BD000038B584B004002068FD
:1017F000DFF8501B884240F0AC80DFF84C0B0068EB
:10180000401CDFF8441B0860DFF83C0B0068052132
:1018100090FBF1F201FB1200002840F09A800221B7
:10182000DFF8340B03F07FFA002801D0012000E03C
:101830000020C0B200281ED1DFF8200B03F00DFB02
:10184000DFF81C0B03F009FB03F04EFC01224FF400
:101850008051DFF8040B03F06FFAC82003F036FE66
:1018600000224FF48051DFF8F00A03F065FAC82037
:1018700003F02CFEEAE7DFF8FC0A0078012868D1C3
:10188000DFF8F40A0068132839DB01224FF4805195
:10189000DFF8C40A03F050FADFF8C80A007800281D
:1018A00016D101224FF40041DFF8AC0A03F044FAEC
:1018B000002504E0DFF8B00A03F01CFE6D1C012DCA
:1018C000F8DB01224FF480715FF0904003F034FAAE
:1018D000DFF8A40A0068142834DB0020DFF8981A27
:1018E0000860DFF8880A0068411CDFF8802A116070
:1018F0000B2827DB0120DFF86C1A087022E0002299
:101900004FF40041DFF8500A03F016FA00224FF4BA
:1019100080715FF0904003F00FFA00224FF4805185
:10192000DFF8340A03F008FA00224FF48041DFF8B0
:10193000280A03F001FA00224FF40051DFF8180AD8
:1019400003F0FAF9DFF8300A0068401CDFF8281AC3
:1019500008602068DFF8241A884240F02282DFF80D
:10196000200A0068401CDFF8181A08601420DFF80D
:10197000101A0968DFF8082A1268B2FBF0F200FBBF
:101980001210002840F0A480DFF8F80902F008FDEA
:101990000021002205E0DFF8D80950F822004118A4
:1019A000521C0A2AF7DB0A20B1FBF0F0DFF8E41939
:1019B0000860DFF8E0090068B0F5026F60D201202E
:1019C000DFF8C4190870DFF8C4090068401CDFF8AC
:1019D000BC190860DFF8B4090068332848D3DFF881
:1019E000B00903F087FD00222021DFF86C0903F025
:1019F000A3F9002280215FF0904003F09DF9DFF809
:101A00005C0903F02AFADFF8580903F026FA03F01C
:101A10008DFD00222021DFF8400903F08DF900221E
:101A200080215FF0904003F087F903F0AFFE03F0F0
:101A30008FFE03F094FE03F0B0FE00222021DFF8B9
:101A4000180903F079F9002280215FF0904003F03B
:101A500073F903F08BFE00222021DFF8FC0803F06D
:101A60006BF9002280215FF0904003F065F92FE0D0
:101A7000DFF818090168DFF8200903F03BFD27E0D3
:101A8000DFF810090068A0F621008B2814D200208E
:101A9000DFF8F8180860DFF804090068401CDFF878
:101AA000FC180860DFF8F40800680B2810D3012048
:101AB000DFF8D41808700BE00020DFF8E0180860A9
:101AC0000020DFF8C81808600020DFF8BC18087094
:101AD000DFF8CC080078002840F0B480DFF89408E4
:101AE0000078002840F0AE8000224FF40041DFF87B
:101AF000680803F021F900224FF480715FF09040F4
:101B000003F01AF900224FF48051DFF84C0803F07B
:101B100013F900224FF48041DFF83C0803F00CF980
:101B200000224FF40051DFF8300803F005F90022DD
:101B30004FF48041DFF8200803F0FEF8DFF8480892
:101B4000007801284CD1DFF8580900685A2824DBB6
:101B5000DFF83808006800280ED001224FF48051C9
:101B6000DFF8F40703F0E8F801224FF40051DFF842
:101B7000E80703F0E1F806E001224FF48051DFF8B6
:101B8000D80703F0D9F8DFF81809006864281FDBCC
:101B90000020DFF80C1908601AE0DFF8F007006891
:101BA00000280ED000224FF48051DFF8AC0703F07C
:101BB000C3F800224FF40051DFF89C0703F0BCF893
:101BC00006E000224FF48051DFF88C0703F0B4F8F0
:101BD000DFF8CC080068401CDFF8C418086031E06A
:101BE00000224FF48051DFF8700703F0A5F80022BF
:101BF0004FF48041DFF8600703F09EF8DFF87C09BE
:101C000000685A2810DB01224FF40051DFF8480722
:101C100003F092F8DFF86409006864280BDB002009
:101C2000DFF85819086006E000224FF40051DFF891
:101C3000280703F081F8DFF844090068401CDFF84A
:101C40003C190860DFF8900A0078012840F09B807A
:101C5000DFF8B00903F014FDDFF8A8090088DFF809
:101C6000A8194880DFF89C094088DFF89C19888013
:101C7000DFF890098088DFF89019C880DFF88409C0
:101C8000C088DFF884190881DFF878090089DFF857
:101C900078194881DFF86C094089DFF86C19888170
:101CA000002003900020029000200190002000906E
:101CB000DFF85409B0F90200DFF8B4190968C1EA85
:101CC00000400390DFF84009B0F90600DFF838194A
:101CD0008988C1EA00400290DFF82C09B0F90A00B7
:101CE000DFF824190989C1EA00400190DFF81809DA
:101CF000B0F90C000004009003A9DFF8580303F0CA
:101D00005BFD02A9DFF8540303F056FD01A9D44896
:101D100003F052FD6946D34803F04EFDCD4803F071
:101D200057FD97280BDBCB4803F057FDCB4803F05A
:101D300054FDCB4803F051FDCA4803F04EFDDFF8D7
:101D400030090068DFF8C0184870DFF8240900681F
:101D5000401CDFF81C1908603E20DFF8AC18C8737F
:101D60000D20DFF8A41808740A20DFF89C184874C6
:101D7000DFF89018DFF8D80500F03CFF012802DBFF
:101D8000C0B200F010F8DFF850090078002804D144
:101D90000120DFF84419087003E00020DFF838194B
:101DA000087005B030BD18B585B0040001224FF4AD
:101DB0008051DFF8A40502F0BFFF01224FF400417B
:101DC000DFF8940502F0B8FF0120DFF8A4190870CD
:101DD0006846DFF85019142200F036FE14F1300086
:101DE00040B2ADF804002000C0B2012806D158204E
:101DF000ADF80A0058208DF80E002AE02000C0B28D
:101E0000022806D15820ADF80A004F208DF80E00A8
:101E10001FE02000C0B2032806D14F20ADF80A0011
:101E200058208DF80E0014E02000C0B2042806D11E
:101E30004F20ADF80A004F208DF80E0009E0200079
:101E4000C0B2092805D12D20ADF80A002D208DF84B
:101E50000E004FF47A7312226946DFF8740901F01C
:101E60007CFD01224FF480715FF0904002F064FF2E
:101E70000020DFF804150860E4B2200003F07BF9CD
:101E80000020DFF8EC1808700120DFF8E814087073
:101E9000DFF840090368581CDFF838190860DFF8DC
:101EA000F404006840F6FC01B0FBF1F26420424308
:101EB000DFF8C0040178DFF84C0AFFF763FC06B0D6
:101EC00010BD10B50168DFF8102991420AD1DFF882
:101ED0000C19DFF8780400F06EFD0120DFF800191E
:101EE0000870ACE00068DFF8FC18884240F0A7807A
:101EF000002018E0C821DFF8102A1268DFF8083A3D
:101F00001B68B3FBF1F301FB1321DFF8002ADFF8B4
:101F1000003A1B5C5354DFF8F0190968491CDFF8DC
:101F2000E8291160401C0828E4DBDFF8DC090068C0
:101F300031E0DFF8D819014411F9071C412929D1F2
:101F4000DFF8C819014411F9061C542922D1DFF821
:101F5000BC19014411F9051C2B291BD1DFF8AC1960
:101F6000014411F9041C542914D1DFF8A0190144CB
:101F700011F9031C45290DD1DFF89019014411F91D
:101F8000021C532906D1DFF88419014411F9011C00
:101F9000542944D0401E082851DBDFF87019014451
:101FA00011F9071C4129C4D1DFF86019014411F966
:101FB000061C5429BDD1DFF85419014411F9051C40
:101FC0002B29B6D1DFF84419014411F9041C532917
:101FD000AFD1DFF83819014411F9031C4829A8D101
:101FE000DFF82819014411F9021C4F29A1D1DFF8AB
:101FF0001C19014411F9011C57299AD1DFF8140961
:10200000FFF7C0FB4FF480710022DFF80049200089
:1020100003F0EEFB0020DFF8F01808600FE0DFF8B7
:10202000F808FFF7AFFB4FF480710022DFF8DC48BF
:10203000200003F0DDFB0020DFF8CC18086010BDA5
:10204000A02400202C25002029CE0008A824002050
:10205000B0240020B824002063CE0008C024002053
:10206000C8240020D024002008C7000830B585B05F
:10207000002003F0F1FB00F015FA002006E04FF419
:102080002F61DFF8EC2242F82010401C0A28F6DB12
:1020900000F0AAFB00F00AFA00F072FA00F0B6FABB
:1020A00000F0E8FA00F066FB00F03EFB00F016FBE3
:1020B000DFF8D00202F074F903F05CFAC0B2002835
:1020C00037D101224FF48051A34802F035FE01229E
:1020D0004FF48041A04802F02FFE00224FF400513F
:1020E0009D4802F029FE40F2EF1003F0EFF90122C3
:1020F0004FF40051984802F01FFE00224FF4805127
:10210000954802F019FE00224FF48041924802F0F7
:1021100013FE40F2EF1003F0D9F9DFF80008016870
:10212000481CDFF8F8271060DFF8F40703F0E2F945
:10213000C7E7FFF711FB0222DFF8A016854801F080
:1021400073FC0822DFF8C817DFF8840601F06CFC86
:1021500000242AE001224FF480517F4802F0ECFD78
:10216000642003F0B3F900224FF480517A4802F062
:10217000E3FD642003F0AAF9C82003F0A7F90122C7
:102180004FF40051744802F0D7FD642003F09EF92B
:1021900000224FF40051704802F0CEFD642003F09D
:1021A00095F9C82003F092F9641C012CD2DBDFF80A
:1021B00074070268DFF8700700684FF47A7190FBCB
:1021C000F1F1DFF8680703F095F96846DFF860176A
:1021D000142200F039FC4FF47A7312226946DFF8BA
:1021E000F00501F0BAFB03F0C8F804215FF090405D
:1021F00002F099FD002801D0012400E0002408210C
:102200005FF0904002F08FFD002801D0012000E037
:1022100000200443E4B2002C36D0DFF80007016848
:10222000481CDFF8F8261060DFF8080703F062F9B1
:1022300001224FF48051484802F07EFD00224FF405
:102240000051454802F078FD40F2EF1003F03EF9EE
:1022500001224FF40051404802F06EFD00224FF47D
:1022600080513D4802F068FD40F2EF1003F02EF976
:10227000DFF8A8060168481CDFF8A0261060DFF828
:10228000B40603F037F9D3E7344802F0B0FD344820
:1022900002F0ADFD012220212F4802F04DFD642007
:1022A00003F014F9012280215FF0904002F044FD18
:1022B0000A2003F00BF9002280215FF0904002F029
:1022C0003BFD642003F002F9012280215FF0904081
:1022D00002F032FD0A2003F0F9F8DFF80405007877
:1022E0000028FAD0194800F093FB04000025A5420D
:1022F000F3DA1848406F202820D1DFF83C16134845
:1023000000F06FFB64230222DFF82C16DFF8C00414
:1023100001F023FBDFF8200690F900007E280DD1A4
:10232000DFF8140690F901007E2807D10120DFF8BC
:102330000C160870DFF8080603F0DCF86D1CD6E711
:102340002025002000100040E82400201C0100206F
:102350000817002050200020000400480022002020
:102360004C2200204525002010CC0008102500201C
:1023700038240020442500200C01002000140040D7
:10238000EC2400205021002040250020F4240020CF
:1023900044CD00081C2500207CCD0008F02400203E
:1023A0004325002000B5ADB01CA8442103F066FA17
:1023B0006846142103F062FA05A85C2103F05EFA76
:1023C00001201C905FF480301D9002202690032095
:1023D0002790012028900C20299007202A90022085
:1023E0002B9002202C901CA803F04CFA002801D05E
:1023F00000F0C4FA0F20009003200190002002900A
:1024000000200390002004900221684603F0D0FDD4
:10241000002801D000F0B2FA44F2450005900020F7
:102420000D9000200F90002011905FF080501990C7
:1024300003200690012007900820089007200990AB
:1024400002200A9004200B905FF080700C9005A889
:1024500003F03AFF002801D000F090FA4FF400702A
:1024600004F0B0F9002801D000F088FA03F09EFED5
:102470004FF47A71B0FBF1F0DFF8AC140860DFF8CC
:10248000A804006804F06EFA042004F06FFA002239
:1024900000215FF0FF3004F04FFA2DB000BD0000C6
:1024A000F824002080B5FFF77DFF01BD80B586B020
:1024B0006846182103F0E2F9DFF88804DFF8881491
:1024C00008605FF48020DFF8801448600020DFF8A7
:1024D000781488600020DFF87014C8600020DFF8EE
:1024E000681408610820DFF8601448610020DFF8F4
:1024F000581408760020DFF8501448760120DFF8E1
:102500004814C8610020DFF8401481F82000002042
:10251000DFF8341488620020DFF82C14C862002031
:10252000DFF8241481F830000020DFF81C14486321
:102530000020DFF8141481F83800DFF80C0401F0F3
:102540004CFE002801D000F019FADFF800040090DA
:1025500006200190032002907F2003900420049025
:10256000002005906946DFF8E00302F0BFF800287C
:1025700001D000F003FA07B000BD0000FC240020E9
:1025800080B5DFF8CC03DFF8CC130860DFF8C803B0
:10259000DFF8C01348600020DFF8B813886001201E
:1025A000DFF8B013C8600020DFF8A813086100202E
:1025B000DFF8A01348610020DFF89813886100203D
:1025C000DFF89013C8610020DFF888130862DFF895
:1025D000840304F0EBF9002801D000F0CFF90021CA
:1025E000DFF8700304F03CFE002801D000F0C6F9CB
:1025F0000021D84804F065FE002801D000F0BEF9A3
:1026000001BD000094240020F0000020E0B56846E1
:1026100000210022002380E80E00C34800684FF428
:102620007A7190FBF1F0CD49CD4A1160401ECC4942
:1026300048600020CA49886040F2E730C849C86055
:102640008020C7498861C64802F094FB002801D069
:1026500000F094F900200090002002906946C048E4
:1026600004F05EFE002801D000F088F907BD0000EC
:1026700014250020E0B5684600210022002380E8F0
:102680000E00A94800684FF47A7190FBF1F0B5494B
:10269000B54A1160401EB44948600020B2498860C4
:1026A00042F20F70B049C8608020AF498861AE48DF
:1026B00002F060FB002801D000F060F900200090DB
:1026C000002002906946A84804F02AFE002801D0A4
:1026D00000F054F907BD00001A01002080B5414800
:1026E0003B4908605FF4E1303949486000203849CF
:1026F000886000203649C8600020354908610C20F8
:10270000334948610020324988614FF40040304924
:10271000C8612F4801F0E4F8002801D000F02EF93C
:1027200001BD000014CE000880B52B488F49086019
:102730005FF4E1308D49486000208C4988600020BA
:102740008A49C8600020894908610C20874948618E
:102750000020864988614FF400408449C86183485D
:1027600001F0BEF8002801D000F008F901BD00001A
:102770004625002080B57E48006850F001007C4965
:1027800008607B48006810F001000090009800226B
:1027900005210C2004F0D0F80C2004F0DEF8002213
:1027A0000A210D2004F0C8F80D2004F0D6F800220C
:1027B00003210E2004F0C0F80E2004F0CEF8002211
:1027C00000210F2004F0B8F80F2004F0C6F801BD76
:1027D000D02000201825002000380140B823002018
:1027E000422500200048004080B586B0684614218C
:1027F00003F044F85F48006850F080005D490860CD
:102800005C48006810F08000059005985948006801
:1028100050F00100574908605648006810F0010068
:10282000059005985348006850F00200514908602F
:102830005048006810F002000590059800224FF4FF
:10284000F0715FF0904002F077FA00224FF222011F
:10285000494802F071FA0C200090002001900020FD
:10286000029069465FF0904002F080F920200090CD
:10287000002001900120029069465FF0904002F034
:1028800075F9802000900120019002200290002024
:10289000039069465FF0904002F068F94FF4B07021
:1028A00000900120019000200290002003906946D2
:1028B0005FF0904002F05AF9202000900120019032
:1028C000022002900020039069462B4802F04EF946
:1028D0004FF47040009001200190002002900020F1
:1028E00003906946244802F041F90220009000203C
:1028F00001900020029069461F4802F037F907B0A6
:1029000000BD000094CD0008E4240020501F0020EA
:1029100000000020F8CE000804CF000800250020A9
:1029200034CC0008040100200801002060CD00081C
:10293000ECCD000858CC0008F823002041250020E9
:1029400000CE000800000450502100204000201953
:1029500000540040B4210020826650000010004066
:1029600000220020001400404C22002050200020B3
:10297000481002404C1002400004004870471CB54B
:1029800004006946200004F009FD200016BD0B4636
:102990000146184604F012BD1CB50400694620002B
:1029A00004F050FD200016BD0021C0F8801C00215D
:1029B000C0F8841C704738B504001022D4F8840C89
:1029C000400104EB0005280000F02EF8D4F8840C38
:1029D000401C6421B0FBF1F201FB1200C4F8840C2E
:1029E00031BD38B504000D001022D4F8800C400130
:1029F00004EB0001280000F017F8D4F8800C401C0C
:102A00006421B0FBF1F201FB1200C4F8800C31BD6F
:102A1000D0F8841CD0F8800C081A64306421B0FB14
:102A2000F1F201FB1200704762B38B0708D0521E0F
:102A300011F8013B00F8013B00F024808B07F6D130
:102A4000830740F0208000BF103A07D330B4B1E8CC
:102A50003810103AA0E83810F9D230BC530724BF20
:102A6000B1E80810A0E8081044BF51F8043B40F852
:102A7000043BD20724BF31F8022B20F8022B44BFBD
:102A80000B7803707047121F17D35B0009D151F800
:102A9000043B20F8023B1B0C121F20F8023BF6D22D
:102AA0000BE051F8043B00F8013B1B0A20F8023B05
:102AB0001B0C121F00F8013BF3D238BF121D521E2F
:102AC00024BF11F8013B00F8013BF8D87047000023
:102AD00038B50D4604464FF4CE6102F0CFFE2046D5
:102AE00029464822FFF7A0FF04F526754FF0FF3076
:102AF00028614FF49670A8800020E88004F1480017
:102B000004F0A4FC04F0EEFE04F18801102064231C
:102B100001F1800213800B8053804B8093808B8067
:102B2000D380CB800831401EF2D12088642110FB75
:102B300001F1298004F525752A46642104F5936086
:102B400004F00EFF04F52472294604F5B86005F080
:102B500001F8002032BD30B400F54773B3F90040EE
:102B6000944211DA5B68D0F894525B1E03F01F03A5
:102B700000EBC30404F5497318682D1AA94206D363
:102B8000B3F90400904202DB30BC0120704730BC36
:102B90000020704778B400F54771B0F91840B1F9DA
:102BA0000030A34200F5257217DB4C68166800EB75
:102BB000C40505F54974761EA380266000F2244002
:102BC0004B685B1C03F01F034B60046813689C4256
:102BD0003CBF002484801433036000200880B2F9D5
:102BE0002000002802DD002111849181002072BCA8
:102BF000704700002DE9F24F2DED0E8BA0B0B1F91A
:102C00000010834600EE901A9FEDDD0AF8EEE00A10
:102C10002E9860EE800ACDED070A0BF58763B0F9B8
:102C200002102E9800EE901AF8EEE00A60EE800A8C
:102C3000CDED080A0BF23442B0F904102E9800EEE4
:102C4000901AF8EEE00A20EE800A8DED090ADFED19
:102C5000CD0AB0F906102E9800EE101AB8EEC00A90
:102C6000C0EE200ACDED0A0ADFEDC60AB0F9081061
:102C70002E9800EE101AB8EEC00AC0EE200ACDED74
:102C80000B0ADFEDC00AB0F90A1000EE101AB8EE18
:102C9000C00AC0EE200ACDED0C0A0BF5866107A82C
:102CA00004F03EFE0BF244430BF588620BF23C410C
:102CB00008A804F035FE0BF58A630BF24C420BF5C5
:102CC000896109A804F02CFE0BF224459FEDAE8A21
:102CD00095ED030A95ED061AD5ED090A20EE000AD6
:102CE00001EE010A00EEA00A05F04AF820EE080AFB
:102CF000BDEEC00A8DED040A0BF28A26049870809E
:102D00009DED070ADDED071A9DED081ADDED090AB4
:102D100020EE210A01EE010A00EEA00A05F030F8CB
:102D200020EE080ABDEEC00A8DED010A0BF25C43ED
:102D3000019830800BF58B620BF254410AA804F025
:102D4000EFFD0BF58D630BF264420BF58C610BA864
:102D500004F0E6FD0BF274430BF58E620BF26C414E
:102D60000CA804F0DDFD95ED0C0A95ED0F1AD5EDDC
:102D7000120A20EE000A01EE010A00EEA00A04F099
:102D8000FFFFFDEEC08A9DED0A0A9DED0B1ADDEDF9
:102D90000C0A20EE000A01EE010A00EEA00A04F07F
:102DA000EFFF286B04F0FCFFCDE9140114AFE86BD2
:102DB00004F0F6FFC7E90201A86C04F0F1FFC7E9CF
:102DC0000401E86804F0ECFFCDE90E010EAFA8693C
:102DD00004F0E6FFC7E902019FED6CDB686A04F0CE
:102DE000DFFFC7E9040100221AA8002100230EC05A
:102DF0000EC01AA900919FED670B0EAB14AA0BF140
:102E0000480102A804F0ECFB02A804F0EDFFDBF897
:102E1000480090ED009B806890ED00AB90ED02BB08
:102E200090ED04CB53EC192B51EC1B0B04F0EEFF8F
:102E300004460F4653EC1A2B51EC1C0B04F0E6FF32
:102E400002460B462046394605F0B2F853EC1D2BDE
:102E500004F0DCFF05F01EF900EE100A05F04EF953
:102E6000B0EE40EA53EC192B51EC190B04F0CEFFF5
:102E700004460F4653EC1C2B51EC1C0B04F0C6FF10
:102E800022463B4605F068F953EC1D2B04F0BEFFCB
:102E90000022DFF8F43905F05FF905F0FBF800EEE9
:102EA000900AB0EE608A53EC1B2B51EC1C0B04F023
:102EB000ADFF04460F4653EC192B51EC1A0B04F0EE
:102EC000A5FF22463B4605F047F953EC1D2B04F0C5
:102ED0009DFF05F0DFF800EE100AF0EE480A05F05D
:102EE000F7F9B0EE408A1EEE100A04F059FF9FED8C
:102EF0002B9B53EC192B04F089FFDFF89029DFF8A6
:102F0000903905F01BFA05F03DFB074618EE100A54
:102F100004F046FF53EC192B04F078FFDFF86C291E
:102F2000DFF86C3905F00AFA05F02CFB5A380090EE
:102F300010F1B40FBCBF00F5B4700090B7800098DA
:102F4000F080BBF910004142B942BFBF87420098F0
:102F5000BBF91610884225DABBF80802401CABF812
:102F600008024FF04F0ABBF94200C742A1BFB84266
:102F7000BBF944000099884216DB4FF0010915E0C7
:102F8000000000396F1283420000C84200000000B8
:102F9000000000407B14AE47E17A943F000000003F
:102FA000008066404FF0580A4FF000090BF20A20EB
:102FB000B6F90810BBF8082220F811200BF188019F
:102FC0000498B6F9082021F812000BF584780198CE
:102FD000B6F9082028F812000BF5C470B6F90830CD
:102FE00018EE902A20F813200BF52577B6F9082063
:102FF000FB88521F02F03F0230F812209A1AFA8022
:1030000018EE900A8218FA8046F2676012B212FB3C
:1030100000F0401400EBD07000B203900024B6F929
:103020000830BBF90000BA881B1A03F03F0331F8DF
:103030001310511AB98004984118B98009B2BBF92C
:10304000000091FBF0F008EE100A2E98696DB0F9BF
:103050000600002902DD002808D501E0002805DD72
:10306000A9656C650BF5906239685160696D40180F
:1030700068650199BBF98004462928DB0BF590614E
:10308000401C0BF545720880B2F90830002B22DD98
:10309000B9F1000F1FD0BBF93E20B7F908309A42B2
:1030A00011DBBBF93C3002B29A420CDA00B20228C2
:1030B00011DD3A684868121A042A0CD2A96DDFF8AB
:1030C000D407814207DB5846FFF764FD03E0002880
:1030D000C8BFABF88044B6F908103889C91E01F0A2
:1030E0003F0138F81120821A3A81019882183A81FA
:1030F0000BF5C472788932F81110411A798118EEF3
:10310000900A411879810199B7F9200082291CDBC6
:10311000396820B979620BF54571087109E0B86A20
:10312000081A062805D90BF54570796204713C84AC
:10313000BC813868398CB862019AA2F164004118E8
:10314000B88D3984401CB88537E0002835DD049AF5
:10315000642A32DA60282FDB3B68796A5B1A022B1B
:103160002ADD46F2610210FB02F2901500EBD070EE
:1031700000B20A28B7F90C10A8BF0920814202DA70
:10318000B8813868386141F27B41B7F9200010FB03
:1031900001F1C81400EBD07000B2BBF91A1008306E
:1031A0008142B8BF0846396840180BF52571CA69D5
:1031B0009042B8BF1046F8613C840BF54571086831
:1031C000B7F92C300BEB4002B2F9C202181A029088
:1031D000A2F8C2320868401C086028280BF5457028
:1031E000A8BFCBF81443017901290AD102980A2813
:1031F000A4BF09210291B7F90C0002998142B8BF1E
:103200000290BBF9040001998842BEBF0846BBF991
:103210000610884252DAB7F9181088424EDB0BF5D7
:103220004570B0F90810042948DCC068401E0BF551
:10323000497200F01F0002EBC0013A680868121AD8
:10324000062A03D2B1F90410042937DC0198388327
:10325000386878610199019A6439AF2A07DA0D203C
:103260004143DFF8343681FB03C358111CE0C82A00
:1032700012DAA2F1AF00C0EBC000DFF81C2680FB21
:103280000232D21002EBD2720D325143DFF808063F
:1032900081FB00C0401107E001EB81008000DFF8F6
:1032A000F81580FB01214811BBF91A1000EBD07012
:1032B0008142B8BF084679694018F8613868F969F1
:1032C000884208BF3C8338682828C0F0CA820BF5C2
:1032D0004571B1F90800BBF90210049A9142C0F29D
:1032E00010810BF54571401C088100B205280CD1F6
:1032F0000BF590623868536900F1640183425161B3
:103300003CBF0BF5936004F037FB0BF54571087972
:1033100040B93968B86A091A192903D20BF5457200
:1033200001211171BBF9380038B10098BBF91610B2
:10333000884209DA01984F2804DC0BF54571B1F990
:10334000088005E0A04603E00BF54570B0F9088061
:10335000B6F908000BF20A22014632F81130069342
:10336000113901F03F0132F811209A1A0A2A07DDBB
:1033700053106FF0050102EB9372A1EBA20205E07E
:10338000C2F11102511002EB91729210BBF92E1092
:10339000ADF810100BF54571B1F90830BDF91010FA
:1033A000891A8B4242DB0BF54573D7F800E0B3F97D
:1033B0000810AEEB010101F1010ECDF814E00BF5A0
:1033C000497CD968491E01F01F010CEBC103196843
:1033D000AEEB010CBBF932E0ACF1010CF445A4BF3B
:1033E000BBF934E0E64521DBBBF92CC0B3F904306E
:1033F000ACEB02029342A2BF4A1CFB699A42A2BFF5
:10340000B5F90420BBF936309A420FDBAA68914225
:10341000BCBF05998A4209DA401C00F03F003081A8
:103420003868401C386020B0072025E20BF5457154
:10343000B1F90820042A57DD3B689B1A5B1C0593F1
:103440000BF549710BF54573DB68DDF814C0BBF96A
:1034500032E05B1E03F01F0301EBC3010B68ACEB12
:10346000030CACF1010CF445A4BFBBF934E0E64514
:103470003ADBB1F90410BBF92CC06145A4BFBDF91A
:1034800010C0624530DB0BF54572B2F90820BBF97C
:1034900030C05118614527DB04920BF20A21821AD1
:1034A00002F03F02DDF818C031F81210049AACEBBC
:1034B000010C02EBD271BCEB610F15DAB5F90420F7
:1034C000BBF936108A420FDBA9688B42BCBF059A54
:1034D000914209DA401C00F03F0030813868401CFE
:1034E000386020B00820C7E10BF54571B1F908003C
:1034F00004280CDB39680BF590600F318160C481C2
:1035000005E00028C4BF5846FFF744FBA0463868D2
:103510002968884207D2B5F904000199884202DA85
:10352000A9803868A8603868F969884205D200988F
:10353000BBF916108842C0F2EB80B8F1000F40F3DF
:10354000E780029800286DDDBAF14F0F0AD1B9F17A
:10355000000F04461AD0BBF9400000EBD07004EB1A
:10356000600413E0BBF91600009988420EDB9DED64
:10357000020AB8EEC00A10EE100A04F011FCC74AA5
:10358000C74B04F043FC04F0FDFF0446BBF9080000
:103590000399814210DABBF9000020188045C0F27F
:1035A000A1803089401C00F03F0030813868401C09
:1035B000386020B003205FE1BBF900106118884536
:1035C00055DA039ABBF90A309A4280F28B80101ABE
:1035D00000EE900AF8EEE00A9FEDA91A60EE810A6B
:1035E000DFEDA81AB8EEC80AC0EEA11AF0EE400A44
:1035F00040EE610ABDEEE00ABBF90C2010EE100AA5
:1036000090426FDA01EBD171B8EB610F6ADB308960
:10361000401C00F03F0030813868401C386020B00A
:10362000042029E1BAF14F0F05D1B9F1000F04D000
:10363000BBF9404001E0BBF93A40BBF908000399EF
:1036400081420FDABBF90000201880454ADB30893F
:10365000401C00F03F0030813868401C386020B0CA
:10366000012009E1BBF90010611888450ADB3089A7
:10367000401C00F03F0030813868401C386020B0AA
:103680000C20F9E0039ABBF90A309A422ADA101AA0
:1036900000EE900AF8EEE00A9FED791A60EE810ADA
:1036A000DFED781AB8EEC80AC0EEA11AF0EE400AB3
:1036B00040EE610ABDEEE00ABBF90C2010EE100AE4
:1036C00090420FDA01EBD171B8EB610F0ADB308960
:1036D000401C00F03F0030813868401C386020B04A
:1036E0000220C9E00BF54571B1F90800BBF90020D3
:1036F000BBF94610891888420ADB3089401C00F06B
:103700003F0030813868401C386020B00920B3E0A9
:10371000B7F90800BBF922108842A2BF0098BBF994
:1037200016108842A2BF686D42F21171884213DB05
:10373000BBF92620BBF924105846FFF70CFA0128E4
:103740000AD13089401C00F03F0030813868401CAD
:10375000386020B010208FE02E990BF5B86004F08F
:1037600035FA002816DD042805DC3089401C00F0FD
:103770003F0030816FE0B6F908100BF20A220846CC
:1037800032F810300F3800F03F0032F810001B1AEA
:103790000C2B5CDD0BF5906538686969884221D295
:1037A0000BF593642E9A0199204604F021F9012823
:1037B00018D1204604F074F900280ADD3089401C35
:1037C00000F03F0030813868401C386020B00A208B
:1037D00052E03968A868814204D2E88BE8813868F1
:1037E000401E28613968A86881423AD22E98B0F903
:1037F000081001F51C51103144F62160814203D3B9
:10380000A889401CA88105E0B5F90C000028C4BFB8
:103810000021A981B5F90C00042822DBB6F90810B3
:103820000BF20A22084632F810300F3800F03F0041
:1038300032F810001B1A0C2B13DCB5F90E20C82A25
:103840000FDB3B6828691B1A9B1F092B09D2491CF7
:1038500001F03F0131813868401C386020B00520FC
:103860000AE03089401C00F03F0030813868401C7D
:10387000386020B05FF00000BDEC0E8BBDE8F28F29
:10388000CDCC4C3E000048430000F0BF182D4454FE
:10389000FB210940A18601001F85EB519A99999956
:1038A0009999E93F08B584B00023039300290EBF1E
:1038B00001930190491E0291009301A904AB0748AE
:1038C0007844183004F07CFE019909B100220A7096
:1038D000002858BF039805B000BD00BF8BDDFFFF77
:1038E00010B50400002C01D1012035E0A0690028AA
:1038F000FFD1606F002805D1002084F870002000FF
:1039000005F04EFE242060672068006840084000F3
:1039100021680860200000F0E3F8012801D10120AF
:103920001AE0606A002802D0200000F03DFA20680A
:10393000406830F49040216848602068806830F02A
:103940002A00216888602068006850F00100216822
:103950000860200000F095FA10BD2DE9FC4106003A
:103960000D0014001F00706F20285AD1002D03D0C5
:10397000200080B2002801D1012053E096F97000A8
:10398000012801D102204DE0012086F870000020BE
:10399000F0672120706705F01FFF8046A6F85040B1
:1039A000A6F85240B068B0F5805F04D130690028B5
:1039B00001D1002401E02C000025002086F87000D1
:1039C00011E0207831680885641C07E0002CF8D1EC
:1039D0002888C005C00D31680885AD1CB6F85200B6
:1039E000401EA6F85200B6F8520000280AD00097F0
:1039F000434600228021300000F077FA0028E5D00D
:103A000003200FE00097434600224021300000F0E1
:103A10006CFA002801D0032004E020207067002009
:103A200000E00220BDE8F68110B504001300A06F8D
:103A3000202853D1002903D0180080B2002801D1DA
:103A400001204CE094F97000012801D1022046E0E9
:103A5000012084F870006165A4F858300020E06708
:103A60002220A067E06E002821D0DFF81403E16E69
:103A7000C862DFF81003E16E0863DFF80003E16E4F
:103A800048630020E16E88639BB2626D206810F18C
:103A90002401E06E05F028FF002808D01020E06720
:103AA000002084F8700020206067012017E00020CB
:103AB00084F870002068006850F480702168086005
:103AC0002068806850F00100216888602068806864
:103AD00050F0400021688860002000E0022010BD06
:103AE00038B5040000252068A7498842FFD0A168A6
:103AF0002069014360690143E0690143206802686D
:103B0000A24802401143206801602068416831F4F6
:103B10004051E068014320684160A16920689A4AE9
:103B2000904201D0206A01432068806830F4306000
:103B300001432068816020689549884215D19548E5
:103B4000006810F00300002805D0022805D006D335
:103B5000032806D007E001205CE002205AE00420A0
:103B600058E0082056E0102054E020688A49884236
:103B700016D18848006810F00C00002806D00428F0
:103B800008D0082804D00C2806D007E0002041E027
:103B900002203FE004203DE008203BE0102039E017
:103BA00020687E49884216D17A48006810F03000BB
:103BB000002806D0102808D0202804D0302806D0AD
:103BC00007E0002026E0022024E0042022E0082074
:103BD00020E010201EE020686B49884219D16D4812
:103BE000006810F44060002809D0B0F5806F0AD05A
:103BF000B0F5006F05D0B0F5406F06D007E00020AB
:103C000008E0022006E0042004E0082002E0102082
:103C100000E0102021685C4A91423DD140B200286A
:103C200006D0022808D0042808D008280AD00CE0C2
:103C300002F0BFFA02000AE0594A08E002F067FA0F
:103C4000020004E04FF4004201E000220125002AB6
:103C500000F08D806168032041438A4205D361688A
:103C60004FF480504143914201D201257FE04FF44F
:103C70008073606840080021E3FB02016268002352
:103C800005F002FFB0F54071464A914202D2216828
:103C9000C8606CE001256AE0E169B1F5004F37D1F9
:103CA00040B2002808D0012809D002280AD00428F0
:103CB0000AD008280BD00DE002F07BFA0CE002F0ED
:103CC00085FA09E0364807E002F021FA04E04FF4F3
:103CD000004001E000200125002848D06168490823
:103CE00011EB40016068B1FBF0F080B2B0F110015F
:103CF0004FF6F072914209D24FF6F0710140C0F3D5
:103D00004200014389B22068C16030E001252EE005
:103D100040B2002808D0012809D002280AD004287F
:103D20000AD008280BD00DE002F043FA0CE002F0B4
:103D30004DFA09E01A4807E002F0E9F904E04FF40F
:103D4000004001E000200125002810D0616810EB40
:103D500051006168B0FBF1F080B2B0F110014FF694
:103D6000F072914202D22168C86000E00125002073
:103D7000206600206066280040B232BD1B4000086B
:103D8000CF3F00081140000800800040F369FFEFBA
:103D900000380140881002400044004000480040C4
:103DA0000024F40000FD0F0090F82410C90707D587
:103DB00001684A6832F40032816A0A4301684A6045
:103DC00090F82410890707D501684A6832F48032D8
:103DD000C16A0A4301684A6090F82410490707D570
:103DE00001684A6832F48022016B0A4301684A6024
:103DF00090F82410090707D501684A6832F4004298
:103E0000416B0A4301684A6090F82410C90607D53F
:103E100001688A6832F48052816B0A4301688A60C3
:103E200090F82410890607D501688A6832F4005298
:103E3000C16B0A4301688A6090F82410490613D5C3
:103E400001684A6832F48012016C0A4301684A60D2
:103E5000016CB1F5801F07D101684A6832F4C002D5
:103E6000416C0A4301684A6090F82410090607D59E
:103E700001684A6832F40022816C0A43006842609B
:103E8000704738B504000020E06705F0A5FC050088
:103E90002068006800070DD57FF07E4000902B0061
:103EA00000225FF40011200000F01FF8002801D06C
:103EB000032019E02068006840070DD57FF07E40A0
:103EC00000902B0000225FF48001200000F00DF82C
:103ED000002801D0032007E0202060672020A06791
:103EE000002084F87000002032BD2DE9F04105006B
:103EF0000E0090461F00069C2868C0693040B04202
:103F000001D1012000E00020414649B2884241D160
:103F100014F1010FF0D005F05FFCC01B844201D307
:103F2000002C14D12868006830F4D070296808602B
:103F300028688068400840002968886020206867F9
:103F40002020A867002085F87000032023E028685F
:103F500000684007D0D52868C0690005CCD54FF46B
:103F60000060296808622868006830F4D070296809
:103F70000860286880684008400029688860202020
:103F800068672020A8672020E867002085F8700077
:103F9000032000E00020BDE8F0810168096831F0ED
:103FA000C0010268116020214167704701680968FB
:103FB00031F490710268116001688968490849000C
:103FC000026891602021816700210166704780B5F9
:103FD0000100886A09680968890616D40021A0F8DA
:103FE0005A100168096831F4807102681160016833
:103FF000896849084900026891600168896831F060
:1040000040010268916020218167FDF75AFF01BDE0
:1040100080B5806A05F04FFE01BD38B5846A606FD7
:10402000A56F21688968090607D5212805D10020D8
:10403000A4F852002000FFF7B0FF20688068400617
:1040400007D5222D05D10020A4F85A002000FFF743
:10405000ADFFE06F50F01000E067200005F02CFE8F
:1040600031BD0000826832F47C12114381607047D8
:10407000826832F0E072114381607047806810F00E
:10408000E070704710B410F1600414EB81042168F3
:10409000DFF80C04014012F0F8420A431A4352F0D0
:1040A0000042226010BC7047603010EB8100006855
:1040B00010F0F8407047603010EB8100016821F08B
:1040C00000410A4302607047C06810F4406F01D19C
:1040D000012000E00020704730B410F130030800E8
:1040E000800910F00C00C3181C681F2511F01F0078
:1040F0008540AC43C2F3846011F01F0110FA01F156
:104100002143196030BC7047C06C10F0C00F01D162
:10411000012000E00020704730B414300B00DB0DAC
:1041200013F004031818036807240D002D0D15F073
:104130001F05AC40A343090D11F01F0112FA01F154
:104140001943016030BC704710B4D0F8B0404B0345
:104150005B0B9C43DFF84C3312F01802D34019403C
:104160004903490B2143C0F8B01010BC7047826866
:10417000DFF834130A40826070478068400F10F007
:10418000010070478268DFF824130A4052F0805221
:10419000826070478068000F10F0010070478268ED
:1041A000DFF808130A4052F001028260704780680D
:1041B00010F0010070478268DFF8F0120A4052F0F8
:1041C0000402826070478068800810F00100704728
:1041D0008068C00810F0010070477CB5040000261C
:1041E00000200090002C01D10120D8E02069002897
:1041F00002D094F920000128606D002807D120002A
:1042000005F018F90020A065002084F8500020680F
:10421000FFF7B3FF002802D02068FFF7A8FF20684F
:10422000FFF7B8FF002811D12068FFF7ABFFDFF8D8
:1042300080020068DFF87C12B0FBF1F0009002E031
:104240000098401E009000980028F9D12068FFF7E0
:10425000A1FF002808D1606D50F010006065A06DCE
:1042600050F00100A06501262068FFF7ACFF616DEA
:10427000C90600F18D80002840F08A80606D30F41E
:10428000807050F0020060652068FFF790FF002802
:104290000AD1DFF82402FFF78AFF002804D1616801
:1042A000DFF81802FFF7DEFE94F91900616B51EA9E
:1042B0004031E0680143A068014394F9200051EACD
:1042C000004194F92000012803D1606A401E51EAA0
:1042D0004041A06A002805D0A26A12F47072E06A18
:1042E000024311432068C268DFF8D4010240114341
:1042F0002068C1602068FFF766FF05002068FFF7AF
:1043000067FF0543002D29D194F9180094F9301066
:10431000490051EA80312068C268DFF8A8010240F4
:1043200011432068C16094F93800012810D1206839
:1043300001696FF38A01E06B0143206C0143606CFB
:104340000143A06C014351F001012068016105E0C7
:104350002068006940084000216808612069012840
:1043600009D12068006B00090001E169491E08437A
:104370002168086305E02068006B000900012168DE
:104380000863606D30F0020050F00100606504E0E9
:10439000606D50F0100060650126300040B276BDBF
:1043A00038B504002068FFF70EFF002874D194F997
:1043B0005000012801D1022071E0012084F8500052
:1043C000200000F099FB0500280040B200285FD1D2
:1043D000616DDFF8FC06014051F480716165606D2C
:1043E000C00404D5A06D30F00600A06501E00020F7
:1043F000A0651C2021680860002084F85000206817
:10440000406830F01C00216848606069082806D1C7
:104410002068406850F008002168486005E0206886
:10442000406850F0040021684860606B002805D1A6
:104430002068406850F01000216848602068C0681B
:10444000800121D5606D30F4005050F480506065DB
:10445000606908280CD12068406830F0200021688D
:1044600048602068406850F04000216848600BE0D8
:104470002068406830F0400021684860206840684B
:1044800050F02000216848602068FFF794FE04E0A7
:10449000002084F8500000E00225280040B232BD20
:1044A00000F0FF03FFFF0700C0FFFF5FC0FFFF7FBB
:1044B00014010020400D03000000045000030450CC
:1044C00007C0F0FFFDBFFFFF0068006C70472DE9DB
:1044D000F04105000026286807682868D0F80480A5
:1044E000B8070FD55FEA88700CD5686DC00603D495
:1044F000686D50F400606865280005F0DEFB02205E
:1045000029680860780702D55FEA487004D4380744
:104510003BD55FEA087038D5686DC00603D4686D76
:1045200050F4007068652868FFF7CEFD002826D09B
:104530002868C068800422D42868006800071ED557
:104540002868FFF740FE002811D12868406830F045
:104550000C0029684860686D30F480706865686D8B
:10456000C0040CD4686D50F00100686507E0686D08
:1045700050F010006865A86D50F00100A865280093
:10458000FDF71AF90C2029680860B80602D55FEA21
:10459000886004D4780645D55FEA486042D5686DE6
:1045A000C00603D4686D50F4005068652868FFF7B2
:1045B000ABFD04002868FFF787FD2968C968002C57
:1045C00005D18A0128D4002826D0880424D428685C
:1045D0000068400620D588021ED42868FFF7F8FD41
:1045E000002811D12868406830F0600029684860D0
:1045F000686D30F480506865686DC0050CD4686DD6
:1046000050F00100686507E0686D50F010006865C3
:10461000A86D50F00100A865280005F04FFB602050
:104620002968086038060CD55FEA086009D5686D0E
:1046300050F480306865280005F041FB802029682F
:104640000860F8050DD55FEAC8500AD5686D50F4CA
:1046500000306865280005F033FB4FF4807029684E
:104660000860B8050DD55FEA88500AD5686D50F42A
:1046700080206865280005F024FB4FF4007029684D
:104680000860F8061CD55FEAC86019D5686B002879
:1046900001D1012604E02868C068C00700D50126C2
:1046A000012E0AD1686D50F480606865A86D50F0E5
:1046B0000200A865280005F005FB102029680860A5
:1046C000780511D55FEA48500ED5686D50F48040EA
:1046D0006865A86D50F00800A8654FF480602968EF
:1046E0000860280005F0EFFABDE8F081F8B5060093
:1046F0000F00002500200090F868DFF8D8138842EA
:10470000FFD196F95000012801D10220DEE10120FD
:1047100086F850003068FFF756FD002840F0CC8145
:104720007868062818D27868022806D012D30428A0
:1047300009D005D3052809D00CE00C2078600BE0E7
:104740001220786008E01820786005E04FF480704F
:10475000786001E0062078603A6879683068FFF791
:10476000BBFC3068FFF72FFD04003068FFF730FD19
:104770000443002C40F0B780BA6839683068FFF70E
:10478000CBFC78693168C968C1F3C101C9B24B007B
:1047900010FA03F33869042805D03A68396930689B
:1047A000FFF770FC9FE000213068FFF77DFC4003BD
:1047B00006D100213068FFF777FCC0F3846007E082
:1047C00000213068FFF770FC90FAA0F0B0FA80F09A
:1047D0003968490303D13968C1F3846104E0396859
:1047E00091FAA1F1B1FA81F1884204D100220021AD
:1047F0003068FFF760FC01213068FFF755FC40038B
:1048000006D101213068FFF74FFCC0F3846007E058
:1048100001213068FFF748FC90FAA0F0B0FA80F070
:104820003968490303D13968C1F3846104E0396808
:1048300091FAA1F1B1FA81F1884204D1002201215B
:104840003068FFF738FC02213068FFF72DFC400389
:1048500006D102213068FFF727FCC0F3846007E02F
:1048600002213068FFF720FC90FAA0F0B0FA80F047
:104870003968490303D13968C1F3846104E03968B8
:1048800091FAA1F1B1FA81F1884204D1002202210A
:104890003068FFF710FC03213068FFF705FC400388
:1048A00006D103213068FFF7FFFBC0F3846007E007
:1048B00003213068FFF7F8FB90FAA0F0B0FA80F01F
:1048C0003968490303D13968C1F3846104E0396868
:1048D00091FAA1F1B1FA81F1884204D100220321B9
:1048E0003068FFF7E8FB3068FFF761FC002840F014
:1048F0009080FA6839683068FFF726FCF868DFF8BE
:10490000D411884240F085803868400303D138686C
:10491000C0F3846004E0386890FAA0F0B0FA80F048
:10492000401C10F01F000A2836D23868400303D11B
:104930003868C0F3846104E0386890FAA0F0B0FAF7
:1049400080F13868400303D13868C0F3846004E024
:10495000386890FAA0F0B0FA80F03A68520303D1B8
:104960003A68C2F3846204E03A6892FAA2F2B2FAB8
:1049700082F2491C890611F0F8410123401C10F015
:104980001F0013FA00F00143521C12F01F02032013
:10499000424351EA025138E03868400303D1386895
:1049A000C0F3846104E0386890FAA0F0B0FA80F1B6
:1049B0003868400303D13868C0F3846004E0386885
:1049C00090FAA0F0B0FA80F03A68520303D13A6846
:1049D000C2F3846204E03A6892FAA2F2B2FA82F276
:1049E000491C890611F0F8410123401C10F01F00FA
:1049F00013FA00F00143521C12F01F020A3A03207E
:104A0000424351EA025151F00071BA683068FFF731
:104A100083FB3868DFF8C010084252D0DFF8BC00D2
:104A2000FFF72CFB01003868DFF8B42090421DD15D
:104A300008021BD43068DFF8AC20904241D151F419
:104A40000001DFF89800FFF713FBDFF89C00006817
:104A5000DFF89810B0FBF1F10C2041430091009871
:104A600000282ED00098401E0090F8E73868DFF844
:104A7000802090420DD1C8010BD43068DFF864204B
:104A800090421ED151F08071DFF85000FFF7F0FA2C
:104A900017E03868DFF85C20904212D1480210D449
:104AA0003068DFF8402090420BD151F48001DFF8EC
:104AB0002C00FFF7DDFA04E0706D50F02000706507
:104AC0000125002086F85000280040B2F2BD000009
:104AD000FEF1FFFF00007F4000000880000304504B
:104AE000000052C70000045014010020400D0300D4
:104AF000000084CB0100008038B504002068FFF777
:104B000056FB002830D1206880686FF39E10002883
:104B100009D0606D50F010006065A06D50F001008C
:104B2000A065012021E02068FFF739FB04F054FE66
:104B3000050020680068C00716D42068FFF737FB1F
:104B4000002802D12068FFF72AFB04F045FE401B35
:104B50000328EED3606D50F010006065A06D50F03A
:104B60000100A065012000E0002032BD78B4020001
:104B700000243BE0072604E0DFF8D0319A42F9D167
:104B8000042614F00303DBB29B009E403543DFF89C
:104B9000C0312600B60843F82650DFF8B8311B684C
:104BA00083434D68ED0300D50343DFF8A8512B6024
:104BB000DFF8A4311B6883434D68AD0300D5034380
:104BC000654D2B60654B1B6883434D68ED0200D536
:104BD0000343624D2B60624B1B6883434D68AD02FB
:104BE00001D5184303005E480360641C0868E04078
:104BF000002800F0968008680123A3401840002890
:104C0000F3D04B68012B08D04B68022B05D04B68C2
:104C1000112B02D04B68122B17D195680326230065
:104C2000DBB25B009E40B543CE682300DBB25B0085
:104C30009E403543956053680125A540AB434D68C0
:104C4000C5F30015A5402B435360D5680326230008
:104C5000DBB25B009E40B5438E682300DBB25B0095
:104C60009E403543D5604B68022B02D04B68122B17
:104C700017D12300DB0802EB83031D6A0F2614F013
:104C80000703DBB29B009E40B5430E6914F0070397
:104C9000DBB29B009E4035432300DB0802EB83031D
:104CA0001D62156803262300DBB25B009E40B543FE
:104CB0000E7916F003062300DBB25B009E403543FD
:104CC00015604B68DB0090D5264B1B6853F0010341
:104CD000244D2B60234B1B6813F001030093009BB2
:104CE0001B4B2500AD0853F825500F2614F0030385
:104CF000DBB29B009E40B543B2F1904F01D100263C
:104D00003FE7194B9A4201D101263AE7174B9A42E5
:104D100001D1022635E7164B9A427FF42DAF0326C8
:104D20002FE771BC7047006989B2084201D00120A9
:104D300000E0002040B2704752B2002A02D089B28F
:104D4000816101E089B28162704700000010004873
:104D5000080001400004014004040140080401402F
:104D60000C040140601002400004004800080048A4
:104D7000000C004810B50400002C01D1012035E0E2
:104D800094F93D00002805D1002084F83C00200063
:104D900004F0D3FB022084F83D00211D206800F0C0
:104DA00049F9012084F84800012084F83E000120E0
:104DB00084F83F00012084F84000012084F841007D
:104DC000012084F84200012084F84300012084F887
:104DD0004400012084F84500012084F846000120A9
:104DE00084F84700012084F83D00002010BD90F9B0
:104DF0003D10012901D001202EE0022180F83D1054
:104E00000168C96851F001010268D1600168DFF8EA
:104E10008420914208D00168B1F1804F04D001682C
:104E2000DFF87420914210D101688A68DFF86C10B5
:104E30000A40062A0FD0B2F5803F0CD001680968FD
:104E400051F001010068016005E00168096851F056
:104E5000010100680160002070470168C9684908C5
:104E600049000268D1600168096A41F211121142D9
:104E70000BD10168096A40F24442114205D1016830
:104E800009684908490002681160012180F83D1055
:104E900000207047002C0140004001400700010045
:104EA00010B504002068006980071AD52068C06822
:104EB000800716D57FF00200216808610120207765
:104EC0002068806910F0030F03D0200004F0FCFE7E
:104ED00005E0200004F0F9FE200004F0F7FE0020B9
:104EE00020772068006940071AD52068C06840070D
:104EF00016D57FF004002168086102202077206821
:104F0000806910F4407F03D0200004F0DDFE05E04E
:104F1000200004F0DAFE200004F0D8FE0020207704
:104F20002068006900071AD52068C068000716D5F8
:104F30007FF0080021680861042020772068C0699C
:104F400010F0030F03D0200004F0BEFE05E02000A7
:104F500004F0BBFE200004F0B9FE0020207720689A
:104F60000069C0061AD52068C068C00616D57FF053
:104F7000100021680861082020772068C06910F4BB
:104F8000407F03D0200004F09FFE05E0200004F0E5
:104F90009CFE200004F09AFE002020772068006923
:104FA000C0070AD52068C068C00706D57FF0010099
:104FB000216808612000FCF717FC206800690006E2
:104FC0000AD52068C068000606D57FF080002168F9
:104FD0000861200004F07BFE20680069C0050AD546
:104FE0002068C068000606D57FF4807021680861DB
:104FF000200004F06DFE2068006940060AD5206894
:10500000C068400606D57FF0400021680861200096
:1050100004F05FFE2068006980060AD52068C06839
:10502000800606D57FF0200021680861200004F08A
:1050300051FE10BD0368DFF87020904202D0B0F13D
:10504000804F03D133F070034A681343DFF85820D0
:1050500090420AD0B0F1804F07D0DFF85020904244
:1050600003D0DFF84C20904203D133F44073CA6878
:10507000134333F080034A69134303608A68C262B2
:105080000A688262DFF82020904207D0DFF81C20F7
:10509000904203D0DFF81820904201D109690163E2
:1050A0000121416170470000002C01400040014097
:1050B00000440140DFF8DC03006880B24FF6FF7166
:1050C000884202D15FF4802006E0DFF8C80301685F
:1050D000DFF8C40310EA812000F1FE6010F57F20A4
:1050E000DFF8B8130860704700B585B00020019064
:1050F00001200290DFF89C03006880B24FF6FF7138
:10510000884202D15FF4802006E0DFF8880301685E
:10511000DFF8840310EA8120C00A801E0390022079
:105120000490DFF87003006880B24FF6FF71884288
:1051300002D15FF4802006E0DFF858030168DFF851
:10514000580310EA812000F1FE6010F57F20DFF89F
:105150004C13086004F025FE694601A804F0A6FE81
:10516000002804D0DFF8380300F0C4F9FEE704F0AB
:105170002AFE05B000BD30B58DB0040000200990B6
:1051800001200A90C348006880B24FF6FF71884240
:1051900002D15FF4802004E0BE480168BE4810EAF6
:1051A0008120C00A801E0B9002200C90B948006834
:1051B00080B24FF6FF71884202D15FF4802004E094
:1051C000B4480168B44810EA812000F1FE6010F58F
:1051D0007F20B249086004F0E4FD08A909A804F0A2
:1051E00065FE002803D0AE4800F084F9FEE70025F4
:1051F00003A804F067FFAB4804F06BFF03900AE0DC
:1052000003A804F079FF0068A74941F825002D1D87
:1052100003A804F075FFA34804F079FF079007A9DD
:1052200003A804F084FF0028EAD1012502A804F0B5
:1052300049FF9E4804F04DFF02900AE002A804F0E6
:105240005BFF0068984941F825002D1D02A804F075
:1052500057FF964804F05BFF069006A902A804F0E9
:1052600066FF0028EAD1022501A804F02BFF904830
:1052700004F02FFF01900AE001A804F03DFF006850
:10528000894941F825002D1D01A804F039FF8848FF
:1052900004F03DFF059005A901A804F048FF00288F
:1052A000EAD10325684604F00DFF824804F011FF9F
:1052B00000900AE0684604F01FFF00687A4941F850
:1052C00025002D1D684604F01BFF7A4804F01FFFDF
:1052D000049004A9684604F02AFF0028EAD1764821
:1052E000026800236D480168002004F0F5FC6B485B
:1052F0000068001D694908605FF0FF3200236748BD
:105300000168002004F0E8FC64480068001D63495F
:105310000860240414F47F042200E3175F48016846
:10532000002004F0D9FC5D480068001D5B4908605E
:105330005FF0FF32002359480168002004F0CCFCE4
:1053400056480068001D5549086000240EE0564884
:1053500050F82420D31751480168002004F0BCFC09
:105360004E480068001D4D490860641CB4F5167F66
:10537000EDDB04F028FD0DB030BDF8B584B00020A1
:1053800000200020002000200020002000204B48AA
:1053900000F0B0F83F48006880B24FF6FF718842D5
:1053A00002D15FF4802004E03A4801683A4810EAEC
:1053B000812000F1FE6010F57F20384908603748F1
:1053C000006801683E4800F095F8344800680830ED
:1053D00032490860314800680168090C49B239480F
:1053E00000F088F82B48006880B24FF6FF718842C1
:1053F00002D15FF4802004E026480168264810EAC4
:10540000812000F1FE6010F57F202449086000240F
:105410003CE02248006802681100120C1F48006836
:10542000001D1E4B18601D48006800680300000C3A
:105430001A4D2D682D1D194E3560184D2D682E689A
:105440003500360C154F3F683F1DDFF850C0CCF8D3
:105450000070124F3F683F683F0CDFF840C0DCF837
:1054600000C01CF1040CDFF834E0CEF800C03FB2FD
:10547000039736B202962DB2019500B200901BB28E
:1054800012B289B2104800F035F8641C972CC0DBCA
:1054900005B0F0BDE075FF1F00FCFF03D82400201D
:1054A0009CCE0008B8240020A40D0020C0240020B9
:1054B000C8240020D02400201C25002028CD00086E
:1054C000ECCE0008ACCE0008C0CB000838B5040014
:1054D00004F082F9050014F1010F03D0044890F99B
:1054E0000000241804F078F9401BA042FAD331BD23
:1054F0001B0100200EB418B5A0B00200002023ABA1
:1055000091216846FEF7CEF904004FF47A7320002B
:10551000020092B269460448FEF71FFA200021B04B
:1055200010BC5DF810FB0000D0200020E0B5DFF8D3
:105530000802DFF8081208606B208DF80400402094
:105540008DF805004FF47A700090022301AADFF86D
:10555000F00190F90000010089B2DFF8E001006875
:1055600001F08AFA002804D0DFF8D001006801F0C9
:10557000F2FC07BDF8B5DFF8C001DFF8C011086024
:10558000D020DFF8C0110870642002900120019043
:10559000DFF8B401009001237522DFF8A40190F92F
:1055A0000000010089B2DFF89401006801F0E6FB19
:1055B000DFF894010178DFF89401FFF79BFFDFF833
:1055C00088010078122801D0002057E06B208DF868
:1055D0000C0000208DF80D004FF47A70009002232B
:1055E00003AADFF85C0190F90000010089B2DFF83E
:1055F0004C01006801F040FA002804D0DFF83C01BB
:10560000006801F0A8FC1B208DF80C0008208DF824
:105610000D004FF47A700090022303AADFF82001F6
:1056200090F90000010089B2DFF81001006801F074
:1056300023FA002804D0DFF80401006801F08BFC95
:105640001C208DF80C0008208DF80D004FF47A70A6
:105650000090022303AADFF8E80090F9000001009F
:1056600089B2DFF8D800006801F006FA002804D0FB
:10567000DFF8C800006801F06EFC012005B000BD35
:1056800010B586B004003B208DF804004FF47A700A
:105690000090012301AADFF8A80090F900000100A2
:1056A00089B2DFF8940001F0E7F9002803D0DFF8B1
:1056B000880001F050FC4FF47A7000900E2302AA8B
:1056C000DFF87C0090F90000010089B2DFF8680083
:1056D00001F090FA002803D0DFF85C0001F03BFCF9
:1056E0009DF808009DF8091051EA002121809DF8DD
:1056F0000A009DF80B1051EA002161809DF80C0012
:105700009DF80D1051EA0021A1809DF810009DF830
:10571000111051EA0021E1809DF812009DF813104C
:1057200051EA002121819DF814009DF8151051EADD
:105730000021618106B010BDB4210020DC240020CE
:105740001801002060240020E0240020BCCE0008C6
:105750001648006830F48070144908607047144897
:105760000068400840001249086070470F48006810
:10577000C008C00050F003000C4908600D480068E4
:1057800050F004000B49086030BF704709480068BA
:1057900030F002000749086070470648006830F0A2
:1057A00010000449086070470000000000700040CD
:1057B0000470004010ED00E038B504000D0020003A
:1057C00004F0BFFC2A000100200004F0CAFC31BD37
:1057D00080B504F0EBFC006802BD10B504002000A9
:1057E00004F077FC0100200004F0E5FC10BD00008F
:1057F00062F30F2262F31F42401810F0030308D037
:10580000C91A1FD3DB0748BF00F8012D28BF20F8B5
:10581000022D130030B414461546103928BF20E974
:105820003C00FAD8490728BF20E90C0048BF40F8DF
:10583000042D890028BF20F8022D48BF00F8012D53
:1058400030BC7047C91818BF00F8012DCB0728BF1E
:1058500000F8012D7047000010B50024032001F06E
:1058600067F8002004F0BAFC002801D0012401E010
:1058700003F0B8FD200040B210BD0000002204F08B
:10588000DDBC0000F8B50500002D01D101208EE33C
:10589000DFF85809046814F00C04DFF85C090668A6
:1058A00016F003062878C00640F1C280002C05D00F
:1058B0000C2C40F08680012E40F08380DFF8CC096C
:1058C0000068800704D5A869002801D101206EE393
:1058D000DFF8B8090068000705D5DFF8B0090068EF
:1058E00010F0F00005E0DFF8A0090068000910F0F2
:1058F000F000296A88423ED2286A00F07FFC002826
:1059000001D0012053E3DFF88409006850F008005B
:10591000DFF878190860DFF87409016831F0F001E8
:10592000286A0143DFF864090160DFF86409006850
:1059300030F47F40E96950EA0120DFF8541908602B
:1059400000F0E5FBDFF84C19DFF8A0281268C2F37D
:105950000312895C11F01F01C840DFF89418086039
:10596000DFF89008006804F039FC010049B2002912
:105970005ED040B21BE3DFF81409006850F0080065
:10598000DFF808190860DFF80409016831F0F00158
:10599000286A0143DFF8F4080160DFF8F4080068C2
:1059A00030F47F40E96950EA0120DFF8E41808602C
:1059B000002CC5D1286A00F021FC0028C0D00120AD
:1059C000F5E2A869002846D0DFF8C008006850F06A
:1059D0000100DFF8B818086003F0FEFE0700DFF8EA
:1059E000AC080068800706D403F0F6FEC01B03284D
:1059F000F5D30320DBE2DFF89408006850F00800DC
:105A0000DFF888180860DFF88408016831F0F001D9
:105A1000286A0143DFF874080160DFF87408006841
:105A200030F47F40E96950EA0120DFF8641808602B
:105A30002878C00779D5082C03D00C2C22D1032E4E
:105A400020D1DFF84808006880036ED56868002818
:105A50006BD10120ABE2DFF8340800684008400059
:105A6000DFF82818086003F0B7FE0700DFF81C080D
:105A700000688007DCD503F0AFFEC01B0328F5D318
:105A8000032094E26868B0F5803F08D1DFF8FC0796
:105A9000006850F48030DFF8F417086024E068688C
:105AA000B0F5A02F10D1DFF8E407006850F4802093
:105AB000DFF8D8170860DFF8D407006850F48030AA
:105AC000DFF8C81708600FE0DFF8C007006830F49F
:105AD0008030DFF8B8170860DFF8B007006830F4EE
:105AE0008020DFF8A8170860686800280ED003F04F
:105AF00073FE0700DFF894070068800315D403F0F5
:105B00006BFEC01B0B28F5D3032050E203F064FEAC
:105B10000700DFF878070068800306D503F05CFE15
:105B2000C01B0B28F5D3032041E2287880071AD543
:105B3000042C03D00C2C33D1022E31D1DFF84C07CA
:105B40000068400504D5E868002801D101202EE254
:105B5000DFF83C07006830F0FE40296950EA016038
:105B6000DFF82C170860287800076DD568690028D1
:105B700053D0DFF81407006850F00100DFF8081771
:105B8000086003F029FE0600DFF8FC0600688007C5
:105B90005AD403F021FE801B0328F5D3032006E22C
:105BA000E868002822D0DFF8E406006850F480702E
:105BB000DFF8D816086003F00FFE0600DFF8CC0609
:105BC0000068400506D403F007FE801B0328F5D3C8
:105BD0000320ECE1DFF8B806006830F0FE402969E8
:105BE00050EA0160DFF8A8160860BCE7DFF89C0601
:105BF000006830F48070DFF89416086003F0ECFD64
:105C00000600DFF8880600684005ACD503F0E4FD27
:105C1000801B0328F5D30320C9E1DFF86C06006878
:105C200040084000DFF86016086003F0D5FD06006C
:105C3000DFF854060068800706D503F0CDFD801B11
:105C40000328F5D30320B2E12878400740F1928081
:105C50000026DFF844060068C0000FD4DFF83806DD
:105C6000006850F08050DFF830160860DFF8280632
:105C7000006810F08050009000980126DFF81C06A4
:105C80000068C00516D4DFF81406006850F4807070
:105C9000DFF80816086003F09FFD0700DFF8FC0539
:105CA0000068C00506D403F097FDC01B0328F5D398
:105CB00003207CE1A868012808D1DFF8E40500682A
:105CC00050F00100DFF8D815086023E0A868052827
:105CD00010D1DFF8CC05006850F00400DFF8C015E3
:105CE0000860DFF8BC05006850F00100DFF8B0156F
:105CF00008600FE0DFF8A805006840084000DFF802
:105D0000A0150860DFF89805006830F00400DFF89F
:105D100090150860A868002810D003F05DFD07000A
:105D2000DFF87C050068800719D403F055FDC01B1F
:105D300041F289318842F3D3032038E103F04CFD6E
:105D40000700DFF85C050068800708D503F044FD14
:105D5000C01B41F289318842F3D3032027E176B298
:105D6000012E07D1DFF83005006830F08050DFF8F1
:105D7000281508602878800630D5686A002816D073
:105D8000DFF82005006850F00100DFF81815086002
:105D900003F022FD0600DFF80C05006880071DD423
:105DA00003F01AFD801B0328F5D30320FFE0DFF882
:105DB000F404006840084000DFF8E814086003F0CD
:105DC0000BFD0600DFF8DC040068800706D503F051
:105DD00003FD801B0328F5D30320E8E0A86A002810
:105DE00000F0E480A86A022840F0AF80DFF80804E1
:105DF000006810F00301EA6A914222D110F07001AC
:105E00002A6B521EB1EB021F1BD110F4FE416A6BCC
:105E1000B1EB022F15D110F07841AA6BB1EBC26F34
:105E20000FD110F4C001EA6B5208521EB1EB425F71
:105E300007D110F0C060296C4908491EB0EB416FD2
:105E40005FD00C2C5BD0DFF844040068400101D522
:105E50000120ACE0DFF83404006830F08070DFF837
:105E60002C14086003F0B8FC0400DFF8200400687C
:105E7000800106D503F0B0FC001B0328F5D30320F6
:105E800095E0DFF874030168DFF81C040140E86A5C
:105E90000143286B401E51EA0011686B51EA002152
:105EA000E86B4008401E51EA4051286C4008401EF3
:105EB00051EA4061A86B51EAC061DFF83C03016020
:105EC000DFF8C803006850F08070DFF8C013086086
:105ED000DFF82403006850F08070DFF81C130860BE
:105EE00003F07AFC0400DFF8A403006880015DD4AD
:105EF00003F072FC001B0328F5D3032057E00120B8
:105F000055E0DFF88803006880014FD4DFF87C0398
:105F1000006850F08070DFF874130860DFF8D80272
:105F2000006850F08070DFF8D012086003F054FC75
:105F30000400DFF858030068800137D403F04CFCFC
:105F4000001B0328F5D3032031E00C2C2CD0DFF804
:105F50003C03006830F08070DFF830130860DFF831
:105F60002C030068000107D4DFF88C020068800869
:105F70008000DFF884120860DFF87C020168DFF837
:105F80002C030140DFF87002016003F025FC0400DF
:105F9000DFF8F8020068800108D503F01DFC001B43
:105FA0000328F5D3032002E0012000E00020F2BD29
:105FB00070B504000D00002C01D10120A6E0DFF82F
:105FC000F002006810F00700A84211D2DFF8E002EA
:105FD0000068C008C0002843DFF8D4120860DFF86A
:105FE000D002006810F00700A84201D001208DE027
:105FF0002078C0073CD56068032805D17A4800683E
:10600000800119D4012081E06068022805D176481A
:106010000068800310D4012078E06068002805D172
:1060200071480068800707D401206FE06E4800685F
:10603000400501D4012069E06C48016889088900A5
:10604000606801436948016003F0C6FB06006748C9
:10605000006810F00C006168B0EB810F08D003F00D
:10606000BBFB801B41F289318842F0D303204DE015
:106070002078800707D55D48016831F0F001A068FD
:1060800001435A480160DFF82802006810F0070059
:10609000854211D2DFF818020068C008C00028430A
:1060A000DFF80C120860DFF80802006810F0070043
:1060B000A84201D0012029E02078400707D54B48AD
:1060C000016831F4E061E0680143484801602078EC
:1060D000000708D54548006830F46050216950EA4F
:1060E000C1004249086000F012F8DFF8A8113F4AE9
:1060F0001268C2F30312895C11F01F01C8403C49C9
:1061000008603C48006804F069F840B270BD0022A5
:1061100000203649096811F00C01374B1B6813F059
:106120000303002903D00C2915D1012B13D12E4ACA
:106130001268120704D4544A1268C2F3032203E01F
:10614000294A1268C2F303125B4B53F8222000293C
:1061500008D1100006E0042901D1584802E00829BE
:1061600000D157480C2920D12348006810F00300C3
:10617000022802D0032802D003E0504A01E0504A2E
:10618000FFE71D480068C0F30211491C1A48006867
:10619000C0F306204243B2FBF1F017490968C1F38E
:1061A0004161491C4900B0FBF1F07047104800689C
:1061B000704780B5FFF7FAFF42493E4A1268C2F3C2
:1061C0000222895C11F01F01C84002BD80B5FFF7B3
:1061D000EDFF3C49374A1268C2F3C222895C11F0D4
:1061E0001F01C84002BD000000100240081002401C
:1061F00014010020100100200C10024038B50400EA
:10620000002525480068C00002D500F0D5FA13E04B
:106210002148006850F080501F4908601E480068FF
:1062200010F080500090009800F0C6FA1A490968F2
:1062300031F08051184A1160B0F5007F07D1812CF0
:1062400010D3A12C01D302250CE001250AE0812CFA
:1062500001D3032506E0802C01D1022502E0702C39
:1062600000D1012512480068C008C0002843104929
:1062700008600F48006810F00700A84201D0012014
:1062800000E0002032BD00009410024000100240E7
:1062900004100240CCCE00085810024000700040AC
:1062A00090100240981002408C809D01FFFFEEFE8E
:1062B00000200240081002403CCB00080024F400FB
:1062C00000127A001CCF00082DE9FC4104000026D2
:1062D0000025206800052AD5606C00280FD0B0F595
:1062E000000F03D0B0F5400F0FD00FE0DFF8300300
:1062F000006850F48030DFF82813086007E00021C0
:10630000201D00F097F9060001E000E001263000B2
:1063100040B200280AD1DFF81403016831F44001CB
:10632000606C0143DFF80403016000E03500206881
:10633000800340F183800027DFF8E8020068C00096
:106340000FD4DFF8E002006850F08050DFF8D4127C
:106350000860DFF8D002006810F0805000900098CC
:106360000127DFF8C402006850F48070DFF8B8122B
:10637000086003F031FA8046DFF8AC020068C0051F
:1063800006D403F029FAB0EB08000328F4D303265F
:10639000300040B2002845D1DFF89402006810F4C4
:1063A000407000281AD0A16D884217D0DFF8800213
:1063B000006830F44070DFF87812096851F48031D9
:1063C000DFF86C221160DFF86812096831F480315F
:1063D000DFF85C221160DFF858120860C00710D5A2
:1063E00003F0FAF98046DFF848020068800708D415
:1063F00003F0F2F9B0EB080041F289318842F2D3A0
:106400000326300040B200280AD1DFF824020168D8
:1064100031F44071A06D0143DFF81402016002E025
:10642000350000E035007FB2012F07D1DFF8F4011D
:10643000006830F08050DFF8EC1108602078C00769
:1064400009D5DFF8E801016889088900206A01435D
:10645000DFF8D80101602078800709D5DFF8CC018A
:10646000016831F00C01606A0143DFF8C00101608E
:106470002078400709D5DFF8B401016831F0300118
:10648000A06A0143DFF8A40101602078800609D5E5
:10649000DFF89801016831F44061E06A0143DFF8F8
:1064A0008C0101602068800509D5DFF88001016852
:1064B00031F44021E06B0143DFF870010160206896
:1064C000400509D5DFF86401016831F44011206C02
:1064D0000143DFF8580101602078400609D5DFF854
:1064E0004C01016831F44051206B0143DFF83C015D
:1064F00001602078000609D5DFF83001016831F429
:106500004041606B0143DFF8240101602068C00551
:1065100009D5DFF81801016831F44031A06B01435F
:10652000DFF8080101602068000324D5DFF8FC00D3
:10653000016831F04061A06C0143DFF8F0000160B8
:10654000A06CB0F1006F08D1DFF8D400006850F4FF
:106550008010DFF8CC1008600DE0A06CB0F1806F07
:1065600009D10121201D00F065F80100080040B2AA
:10657000002800D00D002068400324D5DFF8AC00CF
:10658000016831F04061E06C0143DFF8A000016078
:10659000E06CB0F1006F08D1DFF88400006850F4BF
:1065A0008010DFF87C1008600DE0E06CB0F1806FC7
:1065B00009D10121201D00F03DF80100080040B282
:1065C000002800D00D002068400417D5DFF85C00DB
:1065D000016831F04051206D0143DFF85000016047
:1065E000206DB0F1805F09D10221201D00F022F85A
:1065F0000100080040B2002800D00D00206800040F
:1066000009D5DFF82800016831F08041606D014351
:10661000DFF818000160280040B2BDE8F6810000F4
:106620000C100240581002400070004088100240D8
:1066300090100240F8B505000C000026594800688B
:1066400010F0030F13D05748006810F003002968BA
:1066500088420AD12868002807D052480068C0F351
:106660000210401C6968884230D001262EE028685C
:10667000012804D019D303280DD006D315E04848CB
:106680000068800700D4012610E0454800684005F6
:1066900000D401260AE042480068800304D4404840
:1066A0000068400300D4012600E00126300040B21B
:1066B00000280BD13B48016831F073012868014381
:1066C0006868401E51EA001136480160300040B24F
:1066D000002861D13248006830F08060304908609D
:1066E00003F07AF807002E480068000105D503F092
:1066F00073F8C01B0328F6D30326300040B20028ED
:106700004AD1002C0CD12848016828480140A868CB
:1067100051EA0021E86851EAC061234801601EE0A7
:10672000012C0ED12048016821480140A86851EA97
:10673000002128694008401E51EA40511A48016072
:106740000DE0194801681B480140A86851EA002182
:1067500068694008401E51EA4061134801601048D2
:10676000006850F080600E49086003F035F80400BE
:106770000B480068000105D403F02EF8001B032825
:10678000F6D30326300040B2002805D10648016840
:10679000A869014304480160300040B2F2BD000026
:1067A000001002400C10024010100240FF80FF0752
:1067B000FF809FFFFF80FFF9DFF89000006810F472
:1067C000C0607047B0F5007F2BD1DFF88000006813
:1067D00010F4C060B0F5007F35D0DFF870000068BD
:1067E00030F4C06050F40070DFF860100860DFF82B
:1067F0006000016832204143DFF85800B1FBF0F03F
:10680000401C00E0401EDFF850100968490501D522
:106810000028F7D1DFF840000068400513D50320B9
:1068200012E0DFF82800006810F4C060B0F5806F57
:1068300009D0DFF81800006830F4C06050F48060C0
:10684000DFF808100860002070470000007000406A
:106850001401002040420F001470004010F00700A7
:106860004A490A684FF6FF010A40494951EA0021A6
:106870000A4346480260704744480068C0F302205B
:1068800070470000010049B2002908D4012210F02D
:106890001F018A403F4940B2400941F8202070471B
:1068A000020052B2002A04D409013B4A40B21154FA
:1068B00007E00901394A40B210F00F00104400F817
:1068C000041C704710B410F00700D0F10703052B2B
:1068D00001D3042301E0D0F10703041D072C01D2EA
:1068E000002000E0C01E012414FA03F35B1E1940CF
:1068F0008140012313FA00F0401E1040084310BCF1
:10690000704780B5411EB1F1807F01D301200EE0B8
:10691000401E234908600F215FF0FF30FFF7C0FFE2
:1069200000202049086007201F490860002002BDA0
:1069300080B5FFF793FF01BD70B504000D00160090
:106940000020FFF799FF32002900FFF7BBFF01008D
:10695000200040B2FFF7A4FF70BD80B540B2FFF742
:1069600091FF01BD80B5FFF7CCFF02BD042806D121
:106970000D48006850F004000B49086005E00A4823
:10698000006830F004000849086070470CED00E032
:106990000000FA0500E100E000E400E018ED00E08E
:1069A00014E000E018E000E010E000E010B50400A2
:1069B000002C01D101205EE094F84100002805D1AF
:1069C000002084F84000200002F073FD242084F8A9
:1069D0004100206800684008400021680860606845
:1069E00030F07060216808612068806830F40040F1
:1069F00021688860E068012805D1A06850F4004053
:106A00002168886004E0A06850F404402168886030
:106A1000E068022803D14FF40060216848602068D4
:106A2000406840F0007050F40040216848602068E1
:106A3000C06830F400402168C86021696069014382
:106A4000A06951EA00212068C160E169206A014320
:106A5000206801602068006850F00100216808602B
:106A600000206064202084F8410000202063002082
:106A700084F84200002010BD2DE9F84304000D0009
:106A80009046994694F84100202840F0B08094F94F
:106A90004000012801D10220AAE0012084F8400032
:106AA00002F09AFE06000096192301224FF40041DD
:106AB000200000F0A8FA002801D0012098E0089FEB
:106AC000212084F84100102084F8420000206064F6
:106AD000C4F82480A4F82A9000206063608DB0F58B
:106AE000807F0ED3FF202085DFF8840200905FF0C6
:106AF0008073228DD2B2290089B2200000F095FB6C
:106B00001BE0608D2085DFF8680200905FF0007365
:106B1000228DD2B2290089B2200000F086FB0CE061
:106B2000FF202085002000905FF08073228DD2B27C
:106B3000290089B2200000F078FB608D002838D051
:106B400032003900200000F08DFA002801D0012029
:106B50004EE0606A007821688862606A401C60626A
:106B6000608D401E6085208D401E2085608D002830
:106B7000E3D0208D0028E0D100963B000022802148
:106B8000200000F040FA002801D0012030E0608DA4
:106B9000B0F5807FC4D2608D2085002000905FF02A
:106BA0000073228DD2B2290089B2200000F03DFB93
:106BB000C3E732003900200000F080FA002801D03D
:106BC000012015E020202168C86120684168DFF8B5
:106BD000A401014020684160202084F84100002089
:106BE00084F84200002084F84000002000E00220E9
:106BF000BDE8F2832DE9F84304000D009046994664
:106C000094F84100202840F0B08094F94000012819
:106C100001D10220AAE0012084F8400002F0DCFD4E
:106C200006000096192301224FF40041200000F0D5
:106C3000EAF9002801D0012098E0089F222084F87A
:106C40004100102084F8420000206064C4F82480D1
:106C5000A4F82A9000206063608DB0F5807F0ED389
:106C6000FF202085DFF8100100905FF08073228DF7
:106C7000D2B2290089B2200000F0D7FA1BE0608D63
:106C80002085DFF8F40000905FF00073228DD2B20F
:106C9000290089B2200000F0C8FA0CE0FF2020850E
:106CA000002000905FF08073228DD2B2290089B25B
:106CB000200000F0BAFA608D002838D03200390088
:106CC000200000F024FA002801D001204EE02068C6
:106CD000406A616A0870606A401C6062208D401ED4
:106CE0002085608D401E6085608D0028E3D0208D5A
:106CF0000028E0D100963B0000228021200000F017
:106D000082F9002801D0012030E0608DB0F5807F4D
:106D1000C4D2608D2085002000905FF00073228D2A
:106D2000D2B2290089B2200000F07FFAC3E7320016
:106D30003900200000F0C2F9002801D0012015E040
:106D400020202168C86120684168DFF828000140E0
:106D500020684160202084F84100002084F842002F
:106D6000002084F84000002000E00220BDE8F2830B
:106D70000020008000E800FE002400802DE9FE4F86
:106D80000500884692469B4695F84100202840F031
:106D9000D0800C9C002C05D0DDF83490484680B2A1
:106DA000002804D14FF4007068640120C2E095F916
:106DB0004000012801D10220BCE0012085F84000FC
:106DC00002F00AFD06000096192301224FF400414B
:106DD000280000F018F9002801D00120AAE00E9F39
:106DE0005B465246222085F84100402085F842004B
:106DF000002068646C62A5F82A9000206863019600
:106E000000979BB292B2414689B2280000F0A6F8E2
:106E1000002804D0002085F8400001208AE0688D19
:106E2000B0F5807F0ED3FF202885DFF80C0100909D
:106E30005FF080732A8DD2B2414689B2280000F0FB
:106E4000F4F90DE0688D2885DFF8EC0000905FF024
:106E500000732A8DD2B2414689B2280000F0E5F9CC
:106E600000963B0000220421280000F0CCF8002806
:106E70002DD12868406A696A0870686A401C686297
:106E8000288D401E2885688D401E6885688D0028E5
:106E90002ED0288D00282BD100963B000022802187
:106EA000280000F0B0F8002813D1688DB0F5807F7D
:106EB00011D3FF202885002000905FF080732A8D79
:106EC000D2B2414689B2280000F0AFF910E00120AB
:106ED00030E001202EE0688D2885002000905FF0D2
:106EE00000732A8DD2B2414689B2280000F09DF984
:106EF000688D0028B4D132003900280000F0DEF897
:106F0000002801D0012015E020202968C8612868E8
:106F10004168DFF82800014028684160202085F89A
:106F20004100002085F84200002085F84000002044
:106F300000E00220BDE8FE8F0024008000E800FE93
:106F400080B50168896902681268436B002B01D023
:106F5000436B984701BD406C704700002DE9FC4130
:106F6000040017009846089D099EDFF8E80200908B
:106F700000234246D2B289B2200000F056F9320016
:106F80002900200000F06EF8002801D0012026E042
:106F90001FFA88F8B8F1010F03D1FFB220688762A9
:106FA00011E0380080B2000AC0B221688862320065
:106FB0002900200000F056F8002801D001200EE042
:106FC000FFB22068876200962B000022402120003B
:106FD00000F019F8002801D0012000E00020BDE8F1
:106FE000F68101688969890702D5002102689162EA
:106FF00001688969C90705D40168896951F00101EF
:107000000068816170472DE9F04105000E0090464F
:107010001C00069F286880693040B04201D10120E1
:1070200000E00020414649B2884218D114F1010F16
:10703000F0D002F0D1FBC01B844201D3002CE9D177
:10704000686C50F020006864202085F84100002022
:1070500085F84200002085F84000012000E0002073
:10706000BDE8F08170B505000C0016002868806945
:10707000800721D432002100280000F091F8002878
:1070800001D0012019E014F1010FEFD002F0A4FBB0
:10709000801B844201D3002CE8D1686C50F02000A2
:1070A0006864202085F84100002085F84200002017
:1070B00085F84000012000E0002070BD70B505009B
:1070C0000C0016002868806980061ED4320021005A
:1070D000280000F065F8002815D102F07DFB801B28
:1070E000844201D3002CEDD1686C50F0200068641C
:1070F000202085F84100002085F84200002085F816
:107100004000012002E0012000E0002070BD70B5C9
:1071100005000C0016002868806940073ED4320044
:107120002100280000F03CF8002816D1286880696A
:10713000800614D402F050FB801B844201D3002C43
:10714000E9D1686C50F020006864202085F8410087
:10715000002085F84000012021E001201FE0286880
:107160008069400704D5288D002801D0002016E052
:1071700020202968C861286841683748014028688C
:10718000416000206864202085F84100002085F8D7
:107190004200002085F84000012000E0002070BD82
:1071A00070B505000C00160028688069C0063AD545
:1071B00028688069800618D414F1010FF8D002F015
:1071C0000BFB801B844201D3002CF1D1686C50F082
:1071D00020006864202085F84100002085F84200E6
:1071E000002085F8400001201EE010202968C861B9
:1071F00020202968C8612800FFF7F3FE286841684D
:107200001548014028684160686C50F004006864CB
:10721000202085F84100002085F84200002085F8F4
:107220004000012000E0002070BD70B4039C0568A0
:107230006D680A4E56EA5456B54389B28905890DE0
:107240002943D2B251EA0241194321430068416007
:1072500070BC70470020008000E800FEFF63FF0361
:1072600090F84120202A2AD190F94020012A01D10A
:10727000022025E0012280F84020242280F84120CD
:10728000026812685208520003681A6002681268A5
:1072900032F4805203681A6002681268114302686F
:1072A00011600168096851F0010102681160202134
:1072B00080F84110002180F84010002000E00220FA
:1072C000704790F84120202A27D190F94020012AC8
:1072D00001D1022022E0012280F84020242280F8FF
:1072E0004120026812685208520003681A6002685E
:1072F000126832F4706252EA012201680A60016881
:10730000096851F0010102681160202180F84110E4
:10731000002180F84010002000E0022070470000AB
:1073200030B490F93C20012A01D1022030E0012242
:1073300080F83C20022280F83D20026854680268F0
:1073400093680268134DAA4203D134F470044A686A
:10735000144334F070040A681443026854600268ED
:107360000C4CA24207D00268B2F1804F03D00268F1
:10737000094CA24205D133F0800389680B430168B0
:107380008B60012180F83D10002180F83C10002026
:1073900030BC7047002C01400040014080B502F035
:1073A00066FF02BD38B504460D46AC4205D02068E4
:1073B00020188047241DAC42F9D131BDF8B50546EF
:1073C0000E461746AFF300801A49086800B91A48FC
:1073D0001A4A90422EBF002404460C300860AFF3D6
:1073E00000800CB90120F2BD26606560A760002016
:1073F000F2BD80B50F49124800F001F801BDF8B5A3
:107400000E46054637683C0004D1F1BD88470DE0C3
:1074100007463C46AC42F8D00C3C61680800F9D005
:107420000020606020680028F0D0884730688742DC
:10743000F0D0EDE728250020482500201C2700205B
:107440004825002080B502F019FF02BD10B50446A2
:10745000102002F01BFF08B102F02AFF206000227A
:10746000DFF84C34C0E9002381689FED0C0B81EDFF
:10747000000B816881ED020B806880ED040B84EDC8
:10748000020B84ED040B84ED060B84ED080B84EDF8
:107490000A0B84ED0C0BA26310BD0000000000007D
:1074A000000000002DE9F0412DED108B0D46174630
:1074B00082B00646984695ED009B97ED00ABB0EE86
:1074C000408AF0EE608A51EC1A0B53EC192B00F055
:1074D0006FFDCDE9000195ED02BBD7E9020153EC48
:1074E0001B2B00F065FD41EC1D0BD7E9040195ED68
:1074F00004CB53EC1C2B00F05BFDB46B41EC1E0B7A
:107500006CB3DDE9002351EC180B81F0004103F06E
:1075100093FA41EC1F0B5AD2DDE9000153EC182B12
:1075200003F08AFA53D251EC1F0B53EC1D2B03F0DE
:1075300083FA4CD251EC1D0B53EC182B03F07CFA60
:1075400045D251EC1F0B53EC1E2B03F075FA3ED2C3
:1075500051EC1E0B53EC182B03F06EFA37D2601C63
:1075600003F082FA41EC180B204603F07DFA53EC4D
:10757000192B00F04BFC53EC1A2B00F0EDFD53ECF3
:10758000182B00F0DBFEC5E90001204603F06CFA81
:1075900053EC1B2B00F03AFCD7E9022300F0DCFD92
:1075A00053EC182B00F0CAFEC5E90201204603F097
:1075B0005BFA53EC1C2B00F029FCD7E9042300F004
:1075C000CBFD53EC182B00F0B9FEC5E9040144458E
:1075D000BCBF641CB46302B0BDEC108BBDE8F0818D
:1075E0002DE9FC412DED088B04460D469846B0EE82
:1075F00040AAF0EE60AA9AB016469FEDAE0B42F29A
:10760000107305F108012846FFF74CFFD6E9040185
:10761000D5E9062300F0CCFC9FEDA8BB53EC1B2B57
:1076200000F0F4FB53EC1A2B00F0F0FBD5E9042337
:1076300041EC120BD6E90201B0EE428AF0EE628A0A
:1076400000F0B6FC53EC1B2B00F0E0FB53EC1A2BC4
:1076500000F0DCFBD5E9022341EC110BD6E9000177
:10766000B0EE482AF0EE682AB0EE418AF0EE618A68
:10767000B0EE429AF0EE629A00F09AFC53EC1B2BAB
:1076800000F0C4FB53EC1A2B00F0C0FB41EC100BD4
:10769000B0EE492AF0EE692AB0EE481AF0EE681A08
:1076A0000EA802F0A5FE02462968684602F058FFBF
:1076B0002868694603F0E9F9012102A803F000FAFD
:1076C0000021684603F0FCF90321684603F013FA31
:1076D00000989FED7E9B80ED009B9FED7A8B00983C
:1076E00080ED029B9FED790B009880ED048B0AA83A
:1076F00098ED043B98ED022B98ED001B02F050FE34
:107700000246296802A802F02BFF296812A802F09D
:10771000C3FF12AA02A906A802F022FF012114A8A1
:1077200003F0CEF9012104A803F0CAF908A902A8C0
:1077300003F0F8F96A4602A904A803F001FA01214E
:1077400002A803F0BDF908A902A803F0EBF904A808
:1077500003F046FA039E012EB0EE40AAF0EE60AAB6
:1077600011DB029F97ED000B51EC100B53EC102B2B
:1077700000F04CFB53EC192B00F0EEFC0837761EA2
:1077800041EC190BEED1B0EE490AF0EE690A03F0B4
:1077900051FA51EC1A0B53EC102B00F0CFFD41ECD9
:1077A000100B03F0CBFAB0EE409AF0EE609A012194
:1077B00002A803F085F998ED000B98ED04AB98ED65
:1077C00002BB53EC102B51EC100B00F01FFB2646B4
:1077D00007460C4653EC1B2B51EC1B0B00F016FB21
:1077E0003A46234600F0B8FC07460C4653EC1A2BE9
:1077F00051EC1A0B00F00AFB3A46234600F0ACFCB1
:1078000041EC100B03F016FA53EC102B51EC180B53
:1078100000F0A2FC41EC100B53EC102B00F0F6FA38
:107820002C4A2D4B00F08AFD41EC100B03F08CFA32
:1078300053EC102B29482A4900F0E8FA53EC192B95
:1078400000F0E4FA04AC41EC100B214616A802F05B
:1078500041FD2A68014612A802F082FE286812A99A
:1078600003F013F9012114A803F02AF9012118A843
:1078700003F026F92968304602F02AFF012104A806
:1078800003F01EF9012108A803F01AF901210CA840
:1078900003F016F90121684603F012F9012110A83E
:1078A00003F00EF91AB0BDEC088BBDE8F3810000BF
:1078B0000000F03F0000000000002440399D52A26B
:1078C00046DF913F000000000000F0BF0000000014
:1078D000000000007C14AE47E17A84BF9A99999920
:1078E0009999B93F1D4890ED000AB0EE001ADFEDFE
:1078F0001A0A20EE200AD0ED010A80ED050A60EE9A
:10790000810A30EE801A70EE600AC0EE810A80EEC5
:10791000010AC0ED020A80ED030A80ED040A7047F7
:10792000DFF838C0D0ED000A9CED030A92ED001A92
:1079300020EE200ADCED040A00EE810ADCED020AEA
:1079400093ED001A00EEC10A81ED000A83ED000AF2
:107950000068106070470000C3F5C840D8000020E0
:1079600070B50D46044616464FF49471FDF786FF38
:10797000A5812660204670BDD0F8241100EBC1001F
:10798000002242627047000038B4D0F82421046815
:10799000256800F1240101EBC20319686D1A052D59
:1079A00008D2B3F90420B0F906108A420CDB32BCCD
:1079B00000207047521C202A28BF002200F1240119
:1079C000C0F8242101EBC20321681960DFED5D0AD4
:1079D000C188998090ED050AB4EE600AF1EE10FAC4
:1079E000ACBF012000209871012032BC704700001C
:1079F000F8B51646044600272279B4F90A00012A90
:107A00000D463ED1854242DAC82827713FDBE0802F
:107A10009FED4D1A00EE100AB4F91C0001EE900A19
:107A2000F8EEE11ADFED490A61EE811AB8EEC00AFC
:107A300061EEA01AC1EE801AB4F91E00C4ED041A5A
:107A400001EE900AF8EEE11A61EE811A61EEA01AD9
:107A5000C1EE801AB4F92000C4ED051A01EE900AB7
:107A6000F8EEE11A21EE811A61EE200A80EE800A1A
:107A700084ED060A2046FFF787FF012807D101277A
:107A800005E0A84203DA01212171208102276581E6
:107A90003088A0837088E083B08820843846F2BDA7
:107AA0002DE9F00302460025D2F824010026A9465C
:107AB000202140F2EE2340F255189FED250A176869
:107AC00002EBC00404F1240C3C68DCF800700028D0
:107AD00014BF401E1F20E41B4C2C2AD29CF80640E9
:107AE000761C012C08BF6D1CBCF90440022EA14479
:107AF00018DD00EE905A01EE106AF8EEE00AB8EEDA
:107B0000C11AC0EE810AF4EE400AF1EE10FAA2BFEB
:107B1000B9F57A7F99FBF6FCC44508DBBDE8F003B4
:107B20000120704708BF022D01D1994505DA491E91
:107B3000C5D1BDE8F00300207047BDE8F003022086
:107B400070470000FFFFFFBE000000390000C84280
:107B5000C3F5283F70B50D4604461646AC21FDF727
:107B60008DFE01202560A06066600020206101205C
:107B7000E06500206066204670BDB0F84C10436898
:107B800000EBC102491C42F80C3F836853608AB283
:107B9000082AA8BF0021A0F84C10704770B4024614
:107BA00012681368B1F84C4000200822641E48BFD8
:107BB000083401EBC40555F80C6F9E1B652E03D2EB
:107BC0006D682818521EF1D170BC70477CB50D4607
:107BD0000446A168B5F90600012937D1002829D447
:107BE0006168B1F90020002A02DDA16D491CA16580
:107BF000B0F57A7F62DB216940185A4920618842DA
:107C00000DDB21680A68E168511A01EBD171A26DA0
:107C1000491091422DD3544988424FDB29E004F1A9
:107C200008012046FFF7BAFF216940184E498842F3
:107C300044DB29E0206942F211718842A4BF04F1BB
:107C40000800FFF79AFF4FF0FF3028E000281DD50D
:107C50006168B1F90020002A02DDA16D491CA1650F
:107C6000424A90422ADA2169414E4018B0422061CE
:107C700001DA012076BD04F108012046FFF78EFFEE
:107C800021694018B04219DA022076BD20693949CD
:107C90008842BCBF04F10800FFF76FFF0120A0601D
:107CA00020680168E160B5F9060020616068B0F9FC
:107CB00000100029CCBF01200020A065E16DB5F9BE
:107CC0000A00012921D1002813D4B0F57A7F45DBC1
:107CD000616E401828496066884221DA04F15C012F
:107CE0002046FFF75BFF616E40182449884235DB70
:107CF00022E0606E42F211718842A4BF04F15C0080
:107D0000FFF73BFF4FF0FF3021E0002816D5174961
:107D1000884223DA616E401810F5402F606601DA60
:107D2000052076BD04F15C012046FFF737FF616E48
:107D3000401810F5582F11DA062076BD606E0D49F7
:107D40008842BCBF04F15C00FFF717FF0120E0652B
:107D5000206801682166B5F90A006066002076BDDA
:107D600000000000010006000100090019FCFFFFEF
:107D70000080F2FFF0D8FFFF01000C0001800D0031
:107D8000B5EEC00AF1EE10FA02D4B1EEC00A7047A7
:107D90006FF0004C00EE10CA02F0E8BF7047000020
:107DA000C0F3C75181B1FF2906D0C110400721F0AF
:107DB000E04101F16051704741020CBF40F4E00125
:107DC0006FF000410020704700F0004100020AD02F
:107DD000B0FA80FC00FA0CF001F16051A1EB0C51FB
:107DE00001EBD0214005704710B5044620680169B9
:107DF000491E01612268106928B90023002201216F
:107E0000204602F0C5FF204610BD0000B0B581EA53
:107E1000030C0CF0004C40F2FF7515EA11541DBF25
:107E200015EA1357AC42AF4239E0E41923EA45534F
:107E300043F48013C90241F0004141EA505EC70299
:107E40001100A7FB020200284FF00000EEFB01200A
:107E50004FF00001E3FB072118BF42F00102401878
:107E600000214941E3FB0E01A4F580640F0302D217
:107E700052004041494154F101046CDD470872F160
:107E8000004250F1000051EB0451A1F580115CBF9C
:107E900041EA0C01B0BD4CEA05510020B0BD05EA35
:107EA0001357AC4214BFAF4241E050EA410E1CBF31
:107EB00052EA430E02E061460020B0BD24423C4439
:107EC0001BD15FEA070EF6D0090302BF014600206E
:107ED000AEF1140EB1FA81F7AEEB070401FA07FE1A
:107EE0000C37C7F1200100FA07F7C8404EEA000E30
:107EF00023EA455343F48013A2E733F00043B3FA77
:107F000083F704BFB2FA82FE77440B3FE41BB7F15C
:107F1000200E2FBF02FA0EF3BB40C7F1200E22FA4B
:107F20000EFE38BF43EA0E03BA40641C82E750EAF3
:107F3000410E14BF52EA430E6FF000014FF40017D8
:107F400017EB430F8ABF194617EB410FB5E74CEA11
:107F500005510020B0BDD4F10104B4F120070FDABF
:107F6000C4F12007520828BF42F0010210FA07F5B9
:107F700001FA07F7E1BF2A43E0403843E1400FE050
:107F8000352C98DCC7F1200452EA400220FA07F2AF
:107F900018BF42F0010231FA07F0A1400A43002164
:107FA00072F1004250F1000051EB0C01B0BD000035
:107FB00070B44FF0004591EA030F40F1D5806B405B
:107FC000841A71EB030603D2001BB14112197341ED
:107FD0004FF4001C1CEB410F34BF7CEB430442E028
:107FE0000C0DA4EB1356352E4FDC45EAC323DB0AF8
:107FF00045EAC121C912B6F120050DDD63FA05F687
:10800000EB4086EA0305124218BF45F00105C0188F
:1080100051F100010CD213E062FA06F5F24055402E
:10802000F3415A40B340F3405A408018594107D3B6
:1080300049085FEA30005FEA350528BF45F00105D1
:1080400001F58011420875F1004250F1000041EB4A
:1080500004514E0016F5001F70BC38BF7047002059
:10806000090D090570471CEB410F10D252EA430677
:108070000BD0BCEB410F05D80C0DAB43661E342E64
:10808000B6DD02E0AB438018594170BC704770BC4C
:108090007047000001F000428B1AA3F16051B1F566
:1080A000801F0ADBB1F17F6F1FD242EAC102C1001B
:1080B00071F1004142EB507070470B15C3F1090399
:1080C000212B10D2890241EA9051800201284941B6
:1080D00041F0004121FA03F0C3F12003994071F10E
:1080E000004150417047100070476FF0000013EBE3
:1080F000103F5CBF000E42EAC050704710EE101AED
:108100004FF07E5201EE902AC80F31F0004120D08E
:1081100000EE101A914212D871EEC00A0D4A31EEEB
:10812000801A61EE200AF1EEE00A914286BF80F0EB
:10813000040080EE800A80EE200A02F0F1BE4900C1
:1081400011F1807F9CBF6FF0004100EE101A42F2E7
:108150000D867047F404353F70B44FF0004591EA46
:10816000030F7FF52DAF6B40841A71EB030604D229
:108170006E40001BB141121973414FF4001C1CEBFF
:10818000410F34BF7CEB430682E00C0DA4EB135689
:10819000362E7BDC012E45EAC32341DC43EA5253F1
:1081A00012BFD20292025B08240545EAC12141EACE
:1081B0005051D2EBC020994125D407D1B0FA80F6B6
:1081C00010FA06F162D00020203608E0B1FA81F6FC
:1081D000B140C6F1200220FA02F21143B0404FEA4A
:1081E000F474B4EB465434F001064FEA74040AD830
:1081F000D6F50016760D04F00044F04061FA06F260
:108200005040F1404840C00A40EA415021F000414E
:1082100028BF5FEA500550F1000044EBD12135E062
:10822000DB0A45EAC121C90AB6F120050EDD42EAA2
:108230000242120CC5F1200603FA06F6EB4042EAB0
:1082400006056D42984161F100010DE062FA06F504
:10825000F240554063FA06FC82EA0C02F3405A40B1
:108260006D42904161EB030111F4801F05D1641E42
:10827000620502D06D004041494121F4801143085C
:1082800075F1004350F1000041EB045170BC7047A0
:108290001CEB410F15D223F0004352EA43060BD0EA
:1082A0004FEA4C0CBCEB410F04D80C0D661E342E6B
:1082B000B7DDEBE7801A994150EA410608BF00217B
:1082C000E4E708BF1CEB430F28BF6FF00001DDE7B8
:1082D00052EC101AB0EEC00AC80F49005200F0EE7E
:1082E000E00A28BF0C3011F1807F38BF12F1807F87
:1082F0000CD28A4238BF80F00400124214D034BF3E
:1083000080EE800A80EE200A02F00ABE11F1807F22
:1083100008BF80F0040098BF12F1807F08D88A421D
:1083200014BF00224FF07E5200EE102A02F0F8BD7A
:108330006FF0004100EE101A70470000F0B540F2F7
:10834000FF7581EA030C0CF0004C15EA11541DBFB7
:1083500015EA1357AC42AF42E5E0BC41C1F313014B
:10836000C3F31303801A994143F4801304D2641EAB
:108370004000494180185941C90241EA5051B1FBBE
:10838000F3F603FB1611A2FB0675D7EBC020A9413B
:1083900002D2761E80185941C90241EA5051B1FB00
:1083A000F3FE03FB1E11A2FB0E75D7EBC020A94103
:1083B00003D2AEF1010E80185941890241EA905171
:1083C000760546EA8E2EB1FBF3F603FB1611A2FBEF
:1083D0000675D7EB8020A94102D2761E801859413C
:1083E000C90241EA50514EEA060EB1FBF3F603FB17
:1083F0001611A2FB0675D7EBC020A94102D2761E4A
:1084000080185941C90241EA5051B1FBF3F703FB0F
:108410001711A2FB0735D3EBC020A94167F1000774
:108420000CBF004247F0010766F3D5274FEA1E3123
:10843000B80814F5806412DDBD0775F1004250EBF9
:108440000E5051EB045111F5801F5CBF41EA0C0145
:10845000F0BD4CF07F6141F0E0410020F0BDBD0770
:108460006D0840EA0E5041F48011D4F10104B4F1DA
:1084700020060ADAC4F120060200E04001FA06F301
:10848000E1401843B24015430EE0342C13DCC6F132
:10849000200445EA40056D0820FA06F2154321FA4A
:1084A00006F0A1400D43002175F1004250F100009B
:1084B00051EB0C01F0BD00205FEA0C01F0BDCFB91B
:1084C00092185B41B3FA83F704BFB2FA82F6BF1980
:1084D0000B3FB7F120062FBF02FA06F3BB40C7F1EE
:1084E000200622FA06F638BF3343BA401CB1E4191D
:1084F000641E33E77F4231F00041B1FA81F404BFDA
:10850000B0FA80F6A4190B3CB4F120062FBF00FA94
:1085100006F1A140C4F1200620FA06F638BF314327
:10852000A0403C1B1AE7AC421ABF05EA1357AF4202
:1085300012E050EA41061CBF52EA4306BFE750EA88
:108540004107304661461CBF41EA0551F0BD52EA81
:10855000430C08BFC143F0BD00204FF4001616EBDA
:10856000410F98BF16EB430F08BF16EB410F24BF16
:10857000C14305E016EB430F0CBF61464CEA0551C1
:10858000F0BD0000C1F30A5340F2FE329B1A14DD25
:10859000D3F120034FEAE17208DDC90241EA5051EC
:1085A00041F00040D84080185040704703F2E1305D
:1085B00010B1D24382F000407047002070470000A5
:1085C0002DE9F0439FB000BF66A6269CDFF8E48A41
:1085D00002918DF83B4000210B914FF0FF3704468C
:1085E00091461D460AE019F8011B0298A047002891
:1085F000029000F0A4800B98401C0B9099F80000AA
:1086000050B12528EFD10020002105900691079058
:10861000089109900A9103E00B98A7E041F001014D
:1086200019F8010F2028F9D023280CD02B2804D0CA
:108630002D2805D0302809D083E041F00201EFE772
:1086400041F00401ECE741F00801E9E741F01001D5
:10865000E6E700200D900AE00D98404505DA00EBB2
:10866000800302EB4302303A0D9209F1010999F8B7
:108670000020A2F130000A28EED399F800002E283D
:1086800018BF0C9726D119F8010F2A2808D128689D
:10869000286009F1010950F8042B28600C9219E0B8
:1086A0002D280CBF19F8010B002000220C920BE0C2
:1086B00040B90C9A424505DA02EB820203EB420311
:1086C000303B0C9309F1010999F80030A3F1300215
:1086D0000A2AEDD3ADF83810304699F8001002F0B0
:1086E00071FC08B119F8010B8DF83A009DF83A00B9
:1086F000682804BF99F80010682903D162208DF81A
:108700003A0008E06C2804BF99F800006C2804D1F6
:1087100071218DF83A1009F1010910A804902A4638
:1087200019F8013B6946204600F060F838B910AAF4
:108730006946204600F08CF900287FF55FAF384687
:1087400014E02A2885D12A682A6052F8040B2A608E
:1087500000280D9003D540420D9041F0040109F12D
:1087600001098AE7686A6C747A4C00001FB0BDE8A2
:10877000F083622820D0682811D06A2803D06C28A2
:1087800027D0712825D10868C01D20F00700086097
:10879000D0E9002308300860194610467047002AC7
:1087A0000A680A60106803D0121D0A6000B217E060
:1087B000121D0A6080B217E0002A0A680A60106879
:1087C00003D0121D0A6040B20AE0121D0A60C0B256
:1087D0000AE0002A0A680A60106803D0121D0A60C5
:1087E000C1177047121D0A600021704770B51C4602
:1087F0000D46B4F125002E69114600F017811C3892
:108800006AD0001F022867D9133843D0093863D0D3
:10881000801E16D0401E1ED0401E02285CD9001FAC
:1088200019D0401F00F08380401E33D0401E00F05E
:10883000CD80C01E00F0D880801E2BD0C01E29D055
:10884000FAE06869421C6A610A680A6052F8043BEF
:108850000A603354FAE095F83A000122FFF789FFE5
:10886000C5E900010023994204DA6869411C696185
:108870002D210DE0288F810704D56869411C6961AD
:108880002B2105E0C00722D56869411C69612021C0
:1088900031541CE095F83A000022FFF76AFFC5E961
:1088A000000195F83800010711D5D5E90023002013
:1088B000834208BF82420AD044F02000782806D1C3
:1088C000686930213154401C411C6961345421468F
:1088D00068693044E86083E00868C01D20F0070044
:1088E0000860D0E9002308300860C5E90023D5E915
:1088F0000001C80F04D06869411C69612D210DE099
:10890000288F810704D56869411C69612B2105E026
:10891000C00704D56869411C696120213154686928
:108920003044E8602146284600F0C4F98EE005F1A5
:108930003A02507820B14FF0FF340FF648205EE045
:108940001078622808D0682824D06A2812D06C28B1
:108950002ED071280ED02BE00A680A6052F8040B62
:108960000A6020B94FF0FF340FF6302047E0E96A83
:1089700001706BE00A680A6052F8040B0A6020B9C3
:108980004FF0FF340FF6142039E0EA6AD317C0E93C
:1089900000235BE00A680A6052F8040B0A6020B901
:1089A0004FF0FF340FF6F41029E0E96A01804DE042
:1089B0000A680A6052F8040B0A6020B94FF0FF34CD
:1089C0000FF6D8101BE0E96A01603FE00A680A6010
:1089D00052F8040B0A600021C5E90001EE6078211D
:1089E000284600F0BBF831E00868086050F8044BF6
:1089F0000860EC603CB94FF0FF340FF6B81002F09D
:108A0000EDFA201A70BD2E6B002E04D5204602F020
:108A100005FB044608E032460021204602F01AFB1E
:108A2000002814BF041B3446AC610FE06869411C88
:108A300069612521315409E06969481C6861252272
:108A40007254210002D0411C69613454002070BD71
:108A50002DE9FC410F460646796B7869BC6A091A14
:108A6000386A091AB869091A786A091AF869091A74
:108A700097F838000C1B410790460FD42021002C9A
:108A80008DF800100ADD254601236A463946304636
:108A900000F060FC00285DD16D1EF5D17B69424677
:108AA0003946304600F056FC002853D130208DF86E
:108AB00000003D6A002D09DD01236A463946304633
:108AC00000F048FC002845D16D1EF5D1BB69FA685D
:108AD0003946304600F03EFC00283BD130208DF86E
:108AE00000007D6A002D08DD01236A4639463046C4
:108AF00000F030FC70BB6D1EF6D1F868B969FB69F7
:108B000042183946304600F025FC18BB30208DF85D
:108B10000000BD6A002D08DD01236A463946304653
:108B200000F018FCB0B96D1EF6D197F83800410777
:108B30000DD52021002C8DF8001008DD01236A4698
:108B40003946304600F006FC20B9641EF6D10020FC
:108B5000BDE8F6814FF0FF30BDE8F6812DE9FC4716
:108B600007468A463E69BAF16F0F08BF082405D050
:108B70004AF02001782914BF0A2410243C25D7E9A3
:108B80000023BAF1640F18BFBAF1690F90469946F5
:108B900006D100218B4203DAD8F1000869EB4909BC
:108BA0000020814508BF80451FD1386BE8B9082CEB
:108BB0004CD197F83800010748D530203B2586F87E
:108BC0003B0043E000280ED597F8380000F0140071
:108BD000102808D17A6B7869121A386A121A511A59
:108BE0000029C8BF3962BDE8F3878DF800A0404670
:108BF00049462246E31700F047FF3032D0B26D1EDF
:108C00003A28019504DB9DF80000A0F151018A1873
:108C10007255404649462246E31700F035FF80462C
:108C200089460020814508BF804503D0F868711946
:108C30008842DCD3082C09D197F83800010705D504
:108C4000715D302902D06D1E30207055C5F13C0198
:108C5000B9617019F860386B8142B3DA411A396230
:108C60004FF6EF70398F01403987BDE8F3872DE962
:108C7000D04306460F4614464FF00008DFF83894FC
:108C800012E0E00707D542464B4630463946FFF72B
:108C9000BDF806460F464046494642464B46FFF75A
:108CA000B5F8641080468946002CEAD13046394632
:108CB000BDE8D0832DE9F34F054641F020048DB087
:108CC000D5E90089612C02AE09D0286B002848BF85
:108CD000062003D408BF672C01D101202863D5E901
:108CE000002358004015401C0ED119030CD003205E
:108CF000A8619DF8380061381A2802D20FF2D061BD
:108D000011E00FF2D0610EE058004015401C0FD169
:108D100019030DD10320A8619DF8380061381A2885
:108D200014D30FF2B861E8680322F9F77DFED3E1AE
:108D3000194621F00043B3F5801F10460DD20027DD
:108D4000BB4208BFBA42019703D111E00FF288611C
:108D5000E9E701AA02F0AAF90AE0DFF8607307EB7D
:108D60001352DFF85C3301921940DFF8583319438E
:108D7000C5E90001612C0ED1E86830210170811C29
:108D8000E9609DF8381061290CBF782158214170A5
:108D90006869801C6861D5E900AB2BF000430020B6
:108DA0002AF00002834204BF8242002300F05A816D
:108DB000612C40F0A980286B00284CBF2120401C6A
:108DC00000904046009F7F1C49460022002301F08E
:108DD00033FED94601988DF8082038BF89F0004944
:108DE000001F0190002FD0460DF1090040F349818A
:108DF00040F2FF71DFF8D0B20C910646404649467A
:108E00000022002302F08AF980F03A814800400DE8
:108E100000F11C0210D0002A0EDD0C98824205DB06
:108E200009F0004040EA0B01002013E0A44808408C
:108E300040EA025140460DE029F00043002028F0AE
:108E40000002834208BF82420FBF40461C224046B8
:108E500002F07CF980468946FFF794FBFF1F002F44
:108E6000044609DD01F000FE02460B464046494635
:108E7000FFF79EF880468946F01D072104E004F0C4
:108E80000F0200F8012D2411002C01DD491EF6D53A
:108E9000491E5CBF002200F8012DF9D5ECE000204E
:108EA000194602AA0A4400E05B1E12F80149491E55
:108EB0008442F9D00F2804D10DF10900425C521C04
:108EC0004254002904D50198001D02AE5B1C01909C
:108ED000591E12D49DF838007218147804F1300825
:108EE0005FFA88F4392CC4BFA0F13A04A044491EAB
:108EF00002F80189F1D58DF83800286B002840F17F
:108F0000B080591E2963ACE0404649460022002348
:108F100001F092FD019938BF89F0004947F297505E
:108F200041436A4A91FBF2F20192D2F1070204DD59
:108F300040464946FFF79BFE0AE052420020644942
:108F4000FFF795FE02460B4640464946FFF7F6F905
:108F50008046662C286BDFF87CB106BF019F0A377C
:108F600006273F18142FC8BF142730208DF808009B
:108F700089460DF1090000E03046002F34DD064639
:108F80004046494602F080F901460A4606F10803C8
:108F900004200A26B2FBF6F606EB860EA2EB4E0282
:108FA000303203F8012C0A22B6FBF2F202EB820EF9
:108FB000A6EB4E063036401E03F8026DE9D1083F9D
:108FC000002F03F10806D7DD084602F071F90246CA
:108FD0000B4640464946FEF7EBFF00225B46FEF794
:108FE00015FF80468946CBE70DF10901401A0DF1C6
:108FF000090604E00199491E401E0191761C317852
:109000003029F7D0662C02D10199491C03E0652C68
:109010000CBF012100212B6BCB189842B8BF431E17
:10902000002B1ED4834204DAF05C3528A8BF392017
:1090300000DA30201946721E02EB010800E05B1EC8
:1090400018F80199491E8145F9D0392802D1705C80
:10905000401C7054002904D50198401C16465B1C26
:109060000190019800B200901BB29DF83810324672
:10907000284600F035F82FE0C61D002F3FF7BEAEA2
:1090800030460DF10901401A009903468842C8BFD5
:109090000B46002B0DF109063FF52FAF8342BFF6BB
:1090A000FEAE0DF10900C05C07287FF7F8AE0F2077
:1090B000F6E60000CBCCCC0C0000244002FCFFFF05
:1090C000FFFF0F800000E03F0000F07FA08601005E
:1090D0000000F03F84D797410FB0BDE8F08F00004B
:1090E0002DE9F84783B006468A461746984602F0AF
:1090F000EDF8B8F1000F406A356B90F8009002DC93
:109100004FF00108B6A7BDF930404AF020006628AC
:1091100008BF641C15D0672840F0848014F1040F48
:10912000C0F28680AC4280F2838096F83800641CDE
:10913000010702D4A845B8BF454620B22D1A48BF42
:1091400000250FFA84FAF068B169BAF1000F25DC46
:109150004A1C30234354002D03DC96F838000107E5
:1091600003D5F06800F80290521C15EB0A0FB8BF47
:109170006C4220B2441941424445B8BFA046B26196
:1091800071620FFA88F5F561F068B3692A463946CD
:109190001844F9F749FC641BB462C4E022B290455C
:1091A000084417DA42463946F9F73EFCB0694044B4
:1091B000B061AAEB0801002D716203DC96F838104B
:1091C0000A0705D5F16801F80090F069401CF061CC
:1091D000B562A8E03946F9F727FCB069002D504484
:1091E000A8EB040803DC96F838100A0703D5F168E9
:1091F00001F80090401CB0610FFA88F08542F068D9
:10920000B369B8BFA8460FFA88F207EB0A01184401
:10921000F9F70AFCB0690FFA88F10844B061681ADE
:10922000706280E0BAF1610F14D14FF0700A16E05D
:10923000A84504DA96F838100A0758BF45466D1E4F
:1092400048BF0025BAF1670F14BF4FF0450A4FF031
:10925000650A04E0BAF1410F08BF4FF0500AB16946
:10926000F368481CB061002D17F8012B5A5403DC39
:1092700096F838100A071BD5F168431CB36101F852
:109280000090002D14DDA8F101080FFA88F0854246
:10929000F068B8BFA8460FFA88F239461844F9F7C3
:1092A000C3FBB0690FFA88F108446D1AB0617562AA
:1092B000F068B1690844002C80F800A003D42B2189
:1092C0004170811C03E02D2141706442811C00200B
:1092D0006A460AE023460A2493FBF4F404EB84056F
:1092E000A3EB450302F8013B401C24B2002CF1DC47
:1092F000012806DC4AF02002652A04BF302201F86A
:10930000012B48B9302001F8010B07E0401E1DF881
:109310000020303201F8012B0028F7DCF068B26938
:109320001044091AF16196F8380000F01400102872
:109330000DD17169B0694118706A4118F06941181E
:10934000B06A4118706B8142BCBF411A316204B0EF
:10935000BDE8F087F8B505460E4617461C460020C6
:1093600074B117F8011BB068A847B06030B1F06A5B
:10937000401CF0620020641EF3D1F2BD4FF0FF30BC
:10938000F2BD00007072696E74665F733A20256EDC
:1093900020646973616C6C6F776564007072696ECC
:1093A00074663A2062616420256E20617267756D73
:1093B000656E74007072696E74665F733A206261E4
:1093C0006420257320617267756D656E74000000FE
:1093D0006E616E004E414E00696E6600494E460059
:1093E0003000000080B5DFF8A803006850F00100ED
:1093F000DFF89C130860DFF89803006810F00100A4
:1094000000900098DFF88C03006850F08050DFF87F
:1094100084130860DFF87C03006810F0805000902F
:109420000098002200210520FDF786FA0520FDF7AF
:1094300094FA01BD10B586B0040001A81421FCF710
:109440001DFA2068DFF85013884230D1DFF84C0352
:10945000006850F40050DFF844130860DFF83C0364
:10946000006810F4005000900098DFF830030068A6
:1094700050F00100DFF824130860DFF820030068D3
:1094800010F0010000900098022001900B20029043
:109490000020039001A95FF09040FBF767FB0022DA
:1094A00002211220FDF748FA1220FDF756FA06B005
:1094B00010BD10B586B0040001A81421FCF7DEF938
:1094C0002068DFF8DC12884235D1DFF8D00200686E
:1094D00050F00200DFF8C4120860DFF8C002006834
:1094E00010F00200009000984FF44070019012209C
:1094F000029001200390032004900420059001A90C
:10950000DFF8A002FBF732FBDFF88802006850F4B6
:109510000010DFF880120860DFF87802006810F4AD
:10952000001000900098002202211F20FDF704FA8D
:109530001F20FDF712FA06B010BD80B501689A4AE7
:10954000914214D19348006850F01000914908608E
:109550009048006810F0100000900098002202214E
:109560003620FDF7E9F93620FDF7F7F917E0006836
:109570008E49884213D18748006850F02000854901
:1095800008608448006810F02000009000980022D5
:1095900002213720FDF7D0F93720FDF7DEF901BDB4
:1095A00010B586B0040001A81421FCF767F9206803
:1095B0007F49884273D17648006850F480407449EE
:1095C00008607348006810F4804000900098734869
:1095D000006850F00200714908607048006810F09F
:1095E000020000900098C02001900220029000200C
:1095F0000390032004900720059001A96948FBF718
:10960000B5FA6C486C49086002206B49486000203C
:109610006949886000206849C860802066490861FF
:109620000020654948610020634988612020624923
:10963000C8614FF44050604908625F4800F0D2F8BA
:10964000002801D0F9F79AF95B48E0665A4884622D
:109650005A485B490860022059494860102058491F
:10966000886000205649C860802055490861002064
:109670005349486100205249886120205049C861FF
:1096800000204F4908624E4800F0ACF8002801D095
:10969000F9F774F94A48A0664948846276E0206880
:1096A0004849884272D13B48006850F480203949CB
:1096B00008603848006810F480200090009837480F
:1096C000006850F00200354908603448006810F026
:1096D0000200009000984FF4406001900220029038
:1096E00000200390032004900720059001A92D4835
:1096F000FBF73CFA3448354908600220334948609A
:1097000000203249886000203049C86080202F49FD
:10971000086100202D49486100202C4988612020E3
:109720002A49C861002029490862284800F05AF8EF
:10973000002801D0F9F722F92448E0662348846222
:10974000234824490860022022494860102021490A
:10975000886000201F49C86080201E4908610020E1
:109760001C49486100201B49886120201949C861B3
:10977000002018490862174800F034F8002801D08A
:10978000F9F7FCF81348A0661248846206B010BDD1
:109790006010024058100240000004504C1002407B
:1097A0000054004000040048001000400014004035
:1097B0000038014058000240982200204400024036
:1097C000E022002000480040300002402823002012
:1097D0001C0002407023002001480068704700BF51
:1097E00024250020002801D101206DE00168374ABE
:1097F00091420AD2026836498A181421B2FBF1F16B
:10980000890041643349016409E0026832498A18D9
:109810001421B2FBF1F18900416430490164022155
:1098200080F8251001680A686FF30E128368C1681A
:109830000B4301690B4341690B4381690B43C169C8
:109840000B43016A0B431A4301680A608168B1F552
:10985000804F30D0016C1F4A914216D120490968CF
:109860000F2290F8443013F01C039A4091431C4A95
:1098700011601B490968426890F8443013F01C03DA
:109880009A401143164A116015E0164909680F22E3
:1098900090F8443013F01C039A409143114A116030
:1098A00010490968426890F8443013F01C039A404C
:1098B00011430C4A11600021C163012180F8251079
:1098C000002180F8241000207047000008040240A6
:1098D000F8FFFDBF00000240F8FBFDBF000402409E
:1098E000A8000240A804024070B50400002594F9C5
:1098F0002400012801D1022037E0012084F824004F
:1099000094F9250001282AD1022084F8250000209E
:10991000E06320680068400840002668306020004E
:1099200000F099F8206B002806D02068006850F0FD
:109930000E00216808600BE02068006830F0040029
:10994000216808602068006850F00A0021680860FB
:109950002068006850F001002168086003E00020E2
:1099600084F824000225280040B270BD10B5016CB7
:10997000096802681268042390F8444014F01C043B
:10998000A340194219D0530717D501680968890601
:1099900005D40168096831F00401026811600421EE
:1099A00090F8442012F01C029140026C5160016B4F
:1099B00000294FD0016B88474CE0022390F84440C7
:1099C00014F01C04A34019421FD093071DD5016851
:1099D0000968890608D40168096831F00A0102683B
:1099E0001160012180F82510022190F8442012F026
:1099F0001C029140026C5160002180F82410C16A61
:109A0000002927D0C16A884724E0082390F8444001
:109A100014F01C04A34019421CD011071AD5016888
:109A2000096831F00E0102681160012190F84420AC
:109A300012F01C029140026C51600121C1630121AE
:109A400080F82510002180F82410416B002901D0F6
:109A5000416B884710BD30B4012490F8445015F094
:109A60001C05AC40056C6C60046863608368102B57
:109A700004D103689A600068C16003E003689960DC
:109A80000068C26030BC7047B3BBD9B1B2F5803F4B
:109A90007DD2022A1ED98C46B1FBF2F102FB11C322
:109AA0001B0443EA1043B3FBF2FC02FB1C3380B2FD
:109AB00040EA0343B3FBF2F002FB103240EA0C40F1
:109AC00000237047022A05D98446B0FBF2F002FB5E
:109AD00010C270474AB105D100F0010249085FEA9F
:109AE0003000704700220023704701F0F3BB0B00E9
:109AF0000200002100207047904271EB030CF6D366
:109B0000B3F5803F2FD2F0B5B3FA83F7B1FA81F401
:109B1000A7F10F0E3D1B5340CEF1200602FA0EF2C4
:109B2000F3415340B5F10F0746D80F3C2C44414058
:109B3000C4F12006A040F1414140B1FBF3F603FB24
:109B40001611A2FB0645001BA94102D2761E801801
:109B5000594180EA010221FA0EF362FA0EF2002165
:109B60005A403046F0BD30B4B1FBF3FC03FB1C118E
:109B7000A2FB0C45001BA94103D2ACF1010C8018DB
:109B8000594130BC02460B46604600217047B2F195
:109B9000807F65D3F0B5B2FA82F7B1FA81F4C7F1EC
:109BA0000F063D1B22FA06F307F1110EF241203594
:109BB0005A40B5F10F07B8D94140C4F12006A04082
:109BC000F1414140B1FBF3FC03FB1C11A2FB0C452E
:109BD000001BA94103D2BCF1010C801859410F2F81
:109BE00012D30F3FC90341EA5041B1FBF3F603FB27
:109BF0001611A2FB0645D4EBC030A94102D2761E55
:109C00008018594146EACC3C07B34140C7F12006D1
:109C1000B840F1414140B1FBF3F603FB1611A2FB42
:109C20000645001BA94102D2761E8018594180EAE0
:109C3000010221FA0EF3C7F1200462FA0EF20CFAC7
:109C400007F05A402CFA04F13043F0BD80EA0102DB
:109C500021FA0EF3002162FA0EF260465A40F0BD7E
:109C60008C46B1FBF2F102FB11C31B0243EA106305
:109C7000B3FBF2FC02FB1C331B024CEA002043EA5C
:109C80001063B3FBF2FC02FB1C331B024CEA002006
:109C900043EA1063B3FBF2FC02FB1C331B024CEAE9
:109CA000002043EA1063B3FBF2FC02FB1C324CEAD7
:109CB0000020002370477047704770477047704717
:109CC00070477047704770477047704770477047DC
:109CD00070477047704700002DE9F8430700884639
:109CE00014001D000026DFF8A00190F900000128F3
:109CF00001D1022053E00120DFF88C1108704CF2F2
:109D0000503000F068F88146484640B2002840D103
:109D10000020DFF874114860DFF87001006840052A
:109D20000CD5DFF86801006830F48060DFF85C1162
:109D300008600220DFF85011087703E00020DFF808
:109D40004811087722002B0040463C00002C04D12B
:109D5000110000F079F801260AE0012C01D0022C54
:109D600006D1110000F078F8022C01D15FF48026B2
:109D70004CF2503000F02FF88146002E07D0DFF86B
:109D80001001006830EA0606DFF80401066000F002
:109D900052F90020DFF8F0100870484640B2BDE8E4
:109DA000F28300203A49096800290AD53C493D4A16
:109DB00011603D493B4A116035490968002900D5C9
:109DC000012040B270473248006850F000403049EE
:109DD00008600020704738B50400FFF7FDFC05005F
:109DE0002C480068C00309D514F1010FF8D0FFF723
:109DF000F3FC401BA042F3D3032024E02548006875
:109E000025490840002816D01F49496801431E4AC9
:109E1000516010F0404F06D020490A6810F04041D0
:109E20000A431E490A60810003D020F040401949CE
:109E30000860012007E017480068C00702D501202C
:109E400014490860002032BD114A126852F0010224
:109E50000F4B1A600160704710B440240C4A12681E
:109E600052F480220A4B1A60EFF3108372B60A682C
:109E70000260001D091D641E2200D2B2002AF6D124
:109E800083F3108810BC7047B80000200020024007
:109E90001420024010200240FAC3020018200240A1
:109EA0002301674508200240AB89EFCDF8B50400D7
:109EB0000D00DFF8000290F90000012801D1022016
:109EC00088E00120DFF8EC1108704CF25030FFF709
:109ED00082FF0600300040B2002875D10020DFF874
:109EE000D4114860DFF8D001006880051ED5DFF886
:109EF000C801006830F40070DFF8BC110860DFF8BA
:109F0000B801006840050CD5DFF8AC01006830F4FA
:109F10008060DFF8A41108600320DFF8981108774B
:109F20001AE00120DFF88C11087715E0DFF88801CE
:109F3000006840050CD5DFF88001006830F48060CF
:109F4000DFF8741108600220DFF86811087703E079
:109F50000020DFF8601108772068012810D16068C0
:109F600000F039F84CF25030FFF735FF0600DFF80B
:109F70004C01006830F00400DFF84011086021E077
:109F80005FF0FF302860A76800E07F1CA168E068F0
:109F900041188F4216D26168380000F02FF84CF259
:109FA0005030FFF718FF0600DFF810010168DFF8F6
:109FB00010010140DFF804010160300040B20028C8
:109FC000E3D02F6000F037F80020DFF8E8100870C9
:109FD000300040B2F2BDC00707D5DFF8E0000068EE
:109FE00050F00400DFF8D4100860DFF8D0000068FB
:109FF00050F48030DFF8C41008607047DFF8BC1000
:10A00000096831F47E71C00010F4FF600843DFF886
:10A01000AC100860DFF8A400006850F00200DFF820
:10A020009C100860DFF89400006850F48030DFF87E
:10A030008C1008607047DFF87C0090F91C0001006C
:10A0400049B2012903D0010049B2032915D1DFF833
:10A050006810096851F40061DFF85C201160DFF8D6
:10A060005810096831F40061DFF84C201160124982
:10A07000096851F40071104A1160010049B20229C7
:10A0800002D040B2032811D10B48006850F4805030
:10A09000094908600848006830F4805006490860A3
:10A0A0000548006850F480600349086000200149B9
:10A0B00008777047B80000200020024014200240BA
:10A0C00005FCFFFF10B50400200001F004F920009A
:10A0D00010BD38B50400200001F001F90500200092
:10A0E00001F001F9006801F002F92A0001686846F0
:10A0F00001F001F9006832BD80B501F003F902BD3D
:10A1000010B50400200001F002F9200010BD38B5A0
:10A110000400200001F0E3F80500200001F0E3F85E
:10A120002A000168684601F0E6F8006832BD80B593
:10A1300001F0F6F8002801D1012000E00020C0B2B3
:10A1400002BD38B50400200001F0C9F80500200068
:10A1500001F0C9F82A000168684601F0EAF80068D1
:10A1600032BD73B50400150001A801F0E9F806003E
:10A17000280001F0E7F80500300001F0E4F82B00BA
:10A1800002683100200001F0E2F805000121200002
:10A1900001F0F7F8300001F0D6F80560280001F072
:10A1A000D2F8006801F0A3F8056073BD80B501F036
:10A1B00000F9001D02BD13B50400002101A801F043
:10A1C000FCF80100200001F0FEF80100200001F081
:10A1D00020F90199200001F03DF916BD38B50400C1
:10A1E0000025134890F9000000281DD04FF47A7024
:10A1F0000F4991F90010B0FBF1F00E490968B1FB6D
:10A20000F0F0FCF7AFFB00280CD1102C08D2002294
:10A2100021005FF0FF30FCF78FFB0748046004E08B
:10A22000012502E0012500E00125280040B232BDF1
:10A230001B010020140100201001002000B500BF08
:10A24000130096469446103928BFA0E80C50FAD85F
:10A250005FEA417C28BF0CC048BF40F8042BC90707
:10A2600028BF20F8022B48BF00F8012B00BD10B515
:10A270000400200001F0F9F8200010BD10B5040022
:10A28000200001F0F6F8200010BD000010B50446D3
:10A2900001E001F0F2F82046F6F70AFE28B903487B
:10A2A00000680028F5D08047F5E710BD3025002074
:10A2B0001CB504460020DFF81417C4E90001CDE9FD
:10A2C00000000322694604F1080001F0D8F8204696
:10A2D00016BD000070B52DED048B05460E4688B006
:10A2E000B0EE408AF0EE608A002105F1080000F02F
:10A2F000E7FB7468032C4ED153EC182B0020DFF8D9
:10A30000C016FDF783FD41EC190BB0EE490AF0EEE3
:10A31000690A00F025FD8DED040B324604A902A860
:10A3200001F0BCF87468012C9FED8B8B11DB366853
:10A3300096ED000B51EC100B53EC102BFDF766FD66
:10A3400053EC182BFDF708FF0836641E41EC180B80
:10A35000EED1B0EE480AF0EE680A00F06BFC8DED2D
:10A36000060B06AA02A9684601F0B6F8694605F18F
:10A37000080001F0CFF80121684600F0A1FB01219F
:10A3800002A800F09DFBB0EE490AF0EE690A00F069
:10A39000E1FC85ED000B08B02846BDEC048B70BDD8
:10A3A00010B52DED068B044682B084ED000B002025
:10A3B000CDE90000B0EE418AF0EE618AB0EE429A3B
:10A3C000F0EE629AB0EE43AAF0EE63AA0322694669
:10A3D00004F1080001F053F8A06880ED008B80EDD7
:10A3E000029B80ED04AB02B02046BDEC068B10BD95
:10A3F00010B52DED0A8B0446B0EE408AF0EE608A6F
:10A4000094B09FED550B84ED000BB0EE41BAF0EE29
:10A4100061BAB0EE429AF0EE629A8DED000B032223
:10A42000694604F1080001F02AF89FED99AB53EC5E
:10A43000182B51EC1A0BFDF7E9FC41EC1C0BB0EEAC
:10A440004C0AF0EE6C0A00F08BFCB0EE408AF0EEA5
:10A45000608AB0EE4C0AF0EE6C0A00F07BFC9FEDD7
:10A460003E3B9FED3D2BB0EE481AF0EE681A0CA86B
:10A47000FFF796FF53EC1B2B51EC1A0BFDF7C6FCB4
:10A4800041EC1B0BB0EE4B0AF0EE6B0A00F068FCDF
:10A49000B0EE408AF0EE608AB0EE4B0AF0EE6B0A46
:10A4A00000F058FC9FED2C3BB0EE482AF0EE682AF5
:10A4B0009FED291B08A8FFF773FF53EC192B51ECF4
:10A4C0001A0BFDF7A3FC41EC190BB0EE490AF0EEB4
:10A4D000690A00F045FCB0EE408AF0EE608AB0EE0A
:10A4E000490AF0EE690A00F035FCB0EE483AF0EEA9
:10A4F000683A9FED192B9FED181B10A8FFF750FF2E
:10A50000014608AA04A800F02BF80CAA04A9684682
:10A5100000F026F89DED000B84ED000B02A904F17C
:10A52000080000F0F7FF012102A800F0C9FA01219C
:10A5300006A800F0C5FA012112A800F0C1FA012115
:10A540000AA800F0BDFA01210EA800F0B9FA14B073
:10A550002046BDEC0A8B10BD00000000000000008A
:10A5600070B52DED028B8AB004460D461646FFF7F6
:10A570009FFE06F1080105F1080000F0DDFFD5E9B6
:10A580000023D6E90001B0EE408AF0EE608AFDF7C4
:10A590003DFC53EC182BFDF70BFDC4E9000106F15F
:10A5A0000802294604A800F079FF05F108023146A7
:10A5B00006A800F073FF06AA04A902A800F0E6FFAF
:10A5C00006F1080205F1080108A800F0B9FA08AA86
:10A5D00002A9684600F0DAFF694604F1080000F0BD
:10A5E00099FF0121684600F06BFA012108A800F0EC
:10A5F00067FA012102A800F063FA012106A800F021
:10A600005FFA012104A800F05BFA0AB0BDEC028BEE
:10A6100070BD38B584B004460D46FFF749FE95ED90
:10A62000000BDFF8AC1384ED000B0020CDE9020134
:10A6300005F1080202A9684600F030FF694604F1FE
:10A64000080000F067FF0121684635E010B50446B8
:10A650002DED028B04F1080104F1080000F06CFFFD
:10A66000B0EE408AF0EE608A94ED000B53EC102BB4
:10A6700051EC100BFDF7CAFB53EC182BFDF76CFDEA
:10A68000BDEC028B41EC100BBDE8104000F0D2BADB
:10A69000000000000000E03F38B584B004460D46DD
:10A6A0006846FFF7B6FF2846FFF7D0FF6946204609
:10A6B00000F094F9012102A800F002FA05B030BDC3
:10A6C0004A68032A04BF083000F081BF70470000C9
:10A6D0002DE9F84F2DED068B0D4684B0044603237B
:10A6E0000322002100F054FB074627609FEDB59B35
:10A6F000A86895ED000B90ED00AB53EC102B51ECDE
:10A70000100BFDF783FB0646884653EC1A2B51ECE1
:10A710001A0BFDF77BFB32464346FDF71DFD53EC5C
:10A72000192BFDF773FB9FEDAB8B53EC182BFDF74B
:10A7300013FD41EC1A0B38690228A4BF204600F033
:10A7400055FF2168086880ED00ABAE68D6E90023AC
:10A75000D6E90201FDF75AFB07468946D5E90023F1
:10A76000D6E90401FDF752FB02460B46384649463E
:10A77000FDF71EFC53EC192BFDF748FB41EC1A0BBF
:10A78000206801690229A4BF204600F02FFF20683D
:10A79000016881ED02ABAE68D6E90023D6E9040179
:10A7A000FDF734FB07468946D5E90023D6E90201C7
:10A7B000FDF72CFB3A464B46FDF7CEFC53EC192B2C
:10A7C000FDF724FB41EC1A0B206801690229A4BFA4
:10A7D000204600F00BFF2068016881ED04ABD5F83E
:10A7E00008802668D8E90023D8E90201F768FDF758
:10A7F0000DFB82468B46D5E90001D8E90423FDF71D
:10A8000005FB52465B46FDF7A7FC53EC192BFDF701
:10A81000FDFA41EC1A0B30690228A4BF204600F073
:10A82000E5FE2168086800EBC700012380ED00AB5E
:10A8300001222146684600F0F3FEA86895ED000B62
:10A8400090ED02AB53EC102B51EC100BFDF7DEFA40
:10A8500006460F4653EC1A2B51EC1A0BFDF7D6FAAD
:10A8600032463B46FDF778FC53EC192BFDF7CEFA48
:10A8700053EC182BFDF770FCCDE9020102A96846E4
:10A8800000F0D7FE022301222146684600F0C8FEF0
:10A89000AE68D6E90223D6E90401FDF7B7FA074608
:10A8A0008946D5E90023D6E90001FDF7AFFA024653
:10A8B0000B4638464946FDF77BFB53EC192BFDF759
:10A8C000A5FACDE9020102A9684600F0B2FE002314
:10A8D00002222146684600F0A3FEAE68D6E90023B6
:10A8E000D6E90401FDF792FA07468946D5E9002327
:10A8F000D6E90201FDF78AFA02460B463846494678
:10A90000FDF756FB53EC192BFDF780FACDE9020158
:10A9100002A9684600F08DFE012302222146684606
:10A9200000F07EFEAE68D6E90223D6E90401FDF709
:10A930006DFA07468946D5E90023D6E90001FDF7FF
:10A9400065FA3A464B46FDF707FC53EC192BFDF729
:10A950005DFACDE9020102A9684600F06AFE022311
:10A9600002222146684600F05BFEA86895ED000BC8
:10A9700090ED04AB53EC102B51EC100BFDF746FAA5
:10A9800004460D4653EC1A2B51EC1A0BFDF73EFA18
:10A9900022462B46FDF7E0FB53EC192BFDF736FA68
:10A9A00053EC182BFDF7D8FBCDE9020102A968464C
:10A9B00000F03FFE04B0BDEC068BBDE8F18F000057
:10A9C0000000E03F00000000000000400000F03FF9
:10A9D0000000F0BF000000000000F0BF38B52DED12
:10A9E000020B84B004460D46FFF762FCD5E9000176
:10A9F000DDE90423FDF7A2FCC4E90001002168465B
:10AA000000F05EF8AA68E9680123684600F026FEB7
:10AA100004AA694602A800F05FFD02A92046FFF7DC
:10AA20004FFE012102A800F04BF80121684600F01A
:10AA300047F807B030BD00004FF4001C1CEB410F7D
:10AA400094BF1CEB430F09E041EA030C50EA4C0CA5
:10AA500052EA0C0C03D2994208BF9042704714BFCF
:10AA60008B42824270470000C11768B14840401ACB
:10AA7000B0FA80F29040D21CC907C2F5846241EA64
:10AA8000025202EBD0214005704738B50D4604460E
:10AA900004F1080005F1080195ED000B84ED000BB1
:10AAA00088420BD0012100F00BF8A968A1600021B9
:10AAB000E868E06005F1080000F002F8204632BDC9
:10AAC00038B50400C9B2002910D0206800280DD084
:10AAD000012505E0206800EBC50000F0DFFD6D1CDE
:10AAE00060688542F6D3206800F0D9FD00206060E0
:10AAF0000020206031BD70B505000C00002C10D086
:10AB000000220021200000F0CFFD2860002605E093
:10AB1000286800EBC60000F0D5FD761CA642F7D3EE
:10AB20006C6070BD38B50D4604460021FFF7C8FFC4
:10AB30002A6869680123204600F090FD204632BD56
:10AB40002DE970430E4604461546032100F0C8FD6A
:10AB50002D6836682468D6E90223D5E90401FDF79B
:10AB600055F980468946D6E90423D5E90201FDF767
:10AB70004DF902460B4640464946FDF719FAC4E92D
:10AB80000001D6E90423D5E90001FDF73FF980462D
:10AB90008946D6E90023D5E90401FDF737F90246D5
:10ABA0000B4640464946FDF703FAC4E90201D6E9DF
:10ABB0000023D5E90201FDF729F980468946D6E947
:10ABC0000223D5E90001FDF721F902460B46404674
:10ABD0004946FDF7EDF9C4E90401BDE870830000C2
:10ABE00070B52DED028B056846689FED108B002433
:10ABF0000FE095ED000B53EC102B51EC100BFDF713
:10AC000005F953EC182BFDF7A7FA41EC180B641C5F
:10AC10000835B442EDDBB0EE480AF0EE680ABDEC50
:10AC2000028BBDE8704000F005B800BF00000000D6
:10AC30000000000051EC100B00B500F003F841ECEF
:10AC4000100B00BD40F2FF7C0B0D4DD0634566D26A
:10AC500030B421EA035141F4801103F2FD3C5FEA74
:10AC60005C0C01D300184941890041EA90718000D1
:10AC70004FF440140023E202D50AB1F5100107D4C5
:10AC80006D081DD2091B641900184941491BF7D5ED
:10AC90006D080AD20919641B00184941491BEFD5F8
:10ACA0006D08F7D301E0520817D0C01861419B1A14
:10ACB000AC4100184941801AA941F4D452080AD085
:10ACC000C01AA1419B186C4100184941801AA94142
:10ACD000E9D45208F4D15B1C6C4161084FEA33009F
:10ACE00001EB0C5130BC704750EA0103FBD030B48B
:10ACF000B1FA81F311B9B0FA80F41B190B3BB3F12F
:10AD000020042FBF00FA04F19940C3F1200420FA77
:10AD100004F438BF21439840D3F101039DE7634514
:10AD200014BF50EA410CDEE711F5801FDBD8D94390
:10AD300000F01CB8704741EC100B01BD80B551EC20
:10AD4000100B00F0DBFCF6E780B551EC100B00F0C7
:10AD50004DFDF0E780B551EC100B00F08FFFEAE7F6
:10AD600080B551EC100B00F08BFFE4E70FB581B01C
:10AD700000F088FF0549212205E00FB581B000F001
:10AD800081FF02492222425001B00FBD3C25002024
:10AD900070B5040015001E005D48007800280BD037
:10ADA00000205B4A1070002004E00022594B43F859
:10ADB0002020401C0128F8DB49B200290AD00229D2
:10ADC00001D049D3A1E054480068401C52490860B2
:10ADD00000209BE050480068401C4F4908604F48E5
:10ADE0000068401C4D490860012824D1002100E082
:10ADF000491C00291FD5474850F821000028F7D0EA
:10AE0000444850F821008068A842F1D1414850F8E8
:10AE10002100C068B042EBD13E4850F8210000222A
:10AE20003C4B43F821203D490968491E3B4A1160CB
:10AE3000012101616AE039480068401E3749086015
:10AE40001420FFF723FA002804D03200290000F074
:10AE50001BFF00E0002059E02F480068401E2E49EB
:10AE600008602D480068002821D02C480068401C4C
:10AE70002A490860012814D1002500E06D1C002D2E
:10AE80000FD52100234800EB850000F00CFF20685F
:10AE90000028F3D121480068401E204908600020A6
:10AEA00034E01E480068401E1C49086023E01B482F
:10AEB0000068401C19490860002515E0154850F845
:10AEC000250000280FD0134850F82500002806D090
:10AED000104850F8250000F0F9FE00F0E0FB0020DB
:10AEE0000C4941F825006D1C002DE7D40B48006883
:10AEF000401E0A4908602068002804D0206800F03D
:10AF0000E5FE00F0CCFB00202060002070BD00BFFB
:10AF10001901002004250020082500200C25002010
:10AF20001AA210EE101A43F2A40CC3F6896CF2ECCC
:10AF3000060A614509DB00EE803A70EE800A83EE76
:10AF4000200A40F0020010EE101A4900D1F1E6414B
:10AF50000BD860EE000A20EE203A03EE010A01EE63
:10AF6000A02A42EE202A80EE220A400810F0020FAA
:10AF700018BFB1EE400A02EB8002D2ED000A30EEBB
:10AF8000200A28BFB1EE400A70470000D7B3DD3F6A
:10AF90006AD5033F2B94A93DB82A593F0000803F52
:10AFA000000080BF00000000920A063FDB0FC93F8F
:10AFB000920A863FDB0FC93F920A0640DB0F4940E9
:10AFC000368D27400278C9B28A421AB11CBF10F8E8
:10AFD000012FF9E718BF00207047000080B500B9C5
:10AFE00006A005490B681BB122220021984701E009
:10AFF000F6F736FB222002BD34250020636F6E7306
:10B00000747261696E742068616E646C65723A2056
:10B01000626164206D6573736167650000F101030F
:10B02000810704D010F8011B89B18107FAD10268A9
:10B03000B2F10131914311F0803F04BF50F8042F69
:10B04000F6E710F8011B11B110F8011BFBE7C01A5D
:10B0500070470000C9B2830706D0521E22D310F8F1
:10B06000013B9942F7D11FE0083A13D302F10402E1
:10B0700041EA012141EA014150F8043B121F21BF7E
:10B080004B40A3F1013C2CEA030C1CF0803FF3D0B1
:10B09000C9B2001F083210F8013B521E28BF91EAC6
:10B0A000030FF8D818BF0120401E704710B5144692
:10B0B00000F002F8226010BDC1F30A5343B14A0008
:10B0C00012F5001F28D2A3F2FE32A1EB0251704705
:10B0D00050EA410C20D001F0004C31EA0C01B1FAE9
:10B0E00081F204BFB0FA80F3D2180B3AB2F1200318
:10B0F0002CBF00FA03F1914041EA0C013EBFC2F1BE
:10B10000200C20FA0CF319439040524240F2FD33D8
:10B11000D21A01EB03517047002270474FF4001C14
:10B120001CEB410F94BF1CEB430F09E041EA030CF9
:10B1300050EA4C0C52EA0C0C03D28B4208BF8242FC
:10B14000704714BF9942904270470000124254D495
:10B1500040F2FF7C1CEA11530FD0634531D09B189D
:10B1600063453CBF01EB0251704701F0004141EAE9
:10B170000C510020FFF701BE704750EA410320D078
:10B1800001F0004C91EA0C011CD0B1FA81F30B3BA9
:10B190009A420DD9D21A994051EA0C01C3F1200C00
:10B1A00020FA0CFC61449840531C40F2FF7CD7E726
:10B1B000914041EA0C01C2F1200C20FA0CF3194332
:10B1C00090407047B0FA80F31533202BE0D3202A4B
:10B1D000EED3203A203B9A4209D9D21A00FA03F161
:10B1E00041EA0C010020531C40F2FF7CB8E700FA52
:10B1F00002F141EA0C0100207047524240F2FF7C0C
:10B200001CEA11530DD06345DBD0B2EB030C3CBFFD
:10B21000A1EB025170470CF1010221EA035141F404
:10B22000801150EA410CCCD001F0004C352A27DCCB
:10B2300030B481EA0C01B2F1200309DAC2F1200333
:10B24000044601FA03F5D0402843D1409C400CE06D
:10B25000C3F12002450020FA03F418BF44F00104B2
:10B2600021FA03F091400C43002174F1004550F1A4
:10B27000000051EB0C01244230BC7FF47BAF7047DF
:10B280006146002076E70000400D491840EA812021
:10B290000CD2490DA1F58061491C40F0004005DB4E
:10B2A000D1F11F0154BFC840C0177047002070473C
:10B2B000014648B1B0FA80F18840C91CC1F58461EB
:10B2C000090501EBD0214005704700000048704798
:10B2D00080000020704780B500F0FFFC02BD80B503
:10B2E00000F002FD02BD80B5FFF7F9FF02BD80B599
:10B2F00000F0FBFC02BD10B50400200000F0F6FCDD
:10B30000200010BD80B5006800F0F4FC02BD10B54F
:10B310000400206800F0E9FC00682060200010BDF7
:10B3200000680968884201D1012000E00020C0B215
:10B33000704710B50400200000F0DEFC200010BDB6
:10B3400000687047704780B500F0DAFC02BDF8B5C0
:10B3500004001D00200000F0D5FC06002800FFF7C7
:10B36000F1FF0500300000F0F8FC00F0FAFC0700E7
:10B37000200000F0FAFC2A00390000F0FAFC30004E
:10B38000F2BD70B504000D00200000F0FEFC0600C8
:10B39000200000F001FD0068361A761EAE4201D290
:10B3A000F6F75EF9200000F0F7FC01686D18056003
:10B3B00070BD80B500F0F5FC02BD10B50468FFF764
:10B3C000A6FF200010BD73B5050001A8FFF7B8FF68
:10B3D00004002000FFF7B7FF0068FFF788FF0600B2
:10B3E0002000FFF784FF006830602000FFF77FFF38
:10B3F0000068FFF7A8FF06002000FFF7A4FF006821
:10B400003060280000F0C8FC0168491E016020007F
:10B4100076BD70B505000C002000FFF768FF00F056
:10B42000C1FC2000FFF78FFF00F0BCFC200000F003
:10B4300094FC00F096FC0600280000F096FC310019
:10B4400000F0B4FC280000F090FC0122210000F084
:10B45000B1FC70BD1CB50C00FFF7ABFF0200210072
:10B460006846FFF748FF006816BD80B500F0A6FCEF
:10B4700002BD80B500F0B3FC02BDF6F7F1B870B5BF
:10B480000D46044616460021FFF71AFB00232A4604
:10B490003146204600F0E2F8204670BD2DE9F0412B
:10B4A000154688466968044600F01AF90026002708
:10B4B0000DE028683844D8E90023D0E90001FCF702
:10B4C000A5FC22683A44761CC2E90001083760688E
:10B4D0008642EED3BDE8F0812DE9F0410D460646E7
:10B4E0006968904600F0FCF8002400270DE0286809
:10B4F0003844D8E90023D0E90001FCF71FFF326887
:10B500003A44641CC2E90001083770688442EED3F3
:10B51000BDE8F08138B504460D46AC420AD00121A1
:10B52000FFF7CEFA2868206000216868606028462E
:10B53000FFF7C6FA204632BDF8B52DED028B044662
:10B540000D469FED108B0026002711E020682A6829
:10B5500038443A44D0E90001D2E90023FCF756FC14
:10B5600053EC182BFCF7F8FD41EC180B761C083750
:10B5700060688642EAD3B0EE480AF0EE680ABDEC95
:10B58000028BF1BD00000000000000002DE9F04139
:10B590000F4604467968154600F0A2F80026B0462A
:10B5A00010E038684044761CD0E900232868404405
:10B5B000D0E90001FCF7D0FD2268424408F10808F8
:10B5C000C2E9000160688642EBD3BDE8F08138B57E
:10B5D00004000D00AC4207D0280000F011FC01006F
:10B5E0002A68200000F00EFC200032BD38B50400AF
:10B5F00020680069012812D02068C368206882682A
:10B6000000212000FFF7C4FB050021682800FFF798
:10B61000DEFF20680069401E21680861256031BD99
:10B6200030B40C68E568016005FB0232426030BC52
:10B63000704738B505460C46286801680A69022A31
:10B64000A8BFFFF7D3FF286894ED000B0168686876
:10B650000A6802EBC00080ED000B32BD2DE9F0411D
:10B6600005000C0016001F00002C15D00022002140
:10B67000200000F019F828605FF0000809E03100B0
:10B68000286800EBC80000F0E2FB18F1010806EBA7
:10B69000C706A045F3D36C60BDE8F0817047002871
:10B6A00018BF00F0E7BB704710B504000020002C65
:10B6B00007D0B4F1005F01D3F5F7D2FFE000FEF749
:10B6C000E5FD10BD80B50100082000F0D5FB002885
:10B6D00004D000220023C0E9002300E0002001BDC7
:10B6E00038B504000D0000212000FFF7E9F929001A
:10B6F0002000FFF700FA200032BD0000D0B52DED8C
:10B70000048B41EC180B48004015401C01D1090383
:10B7100019D151EC180B20F0000221F00043002059
:10B72000834208BF82420ED0C80F1ABF43EC182BC9
:10B730000824002451EC180B00224FF07953FFF736
:10B740007BF905D234BB51EC180BBDEC048BD0BD9A
:10B750009FED229B51EC190B53EC182BFCF728FCA6
:10B7600006460F4653EC182B51EC190BFCF7F4FC72
:10B7700032463B46FCF74AFBFFF764FA41EC190BF3
:10B7800051EC180B174A184BFFF756F907D253EC38
:10B79000192B0FE081F0004141EC180BD3E7012297
:10B7A0000D4BFFF749F90ED284F0020451EC190B4E
:10B7B00053EC182BFCF7C2FDBDEC048B2246BDE810
:10B7C000D04000F05DBBFFF7D1FABDEC048B4FF029
:10B7D000FF306FF00041D0BD0000F03F00000000DE
:10B7E0000000F03FCE3B7F669EA0E63F41EC100B91
:10B7F000480080B54015401C0ED148004015401C43
:10B8000001D1090305D151EC100BC80F18BF9FEDF2
:10B81000080B51EC100B04BD002100910022034BDA
:10B8200051EC100B00F030FC04BD00BF0000F03FF5
:10B830000000000000000000F8B52DED068B41EC83
:10B84000180B154653EC182BDFF8A003DFF8A013F4
:10B85000FCF7DCFA41EC190B21F00041DFF89423EE
:10B86000DFF89433FFF7E8F86AD253EC192B9FED19
:10B87000B90B03F0004251EC100B0C46144353EC8F
:10B88000102B51EC190B2346FCF766FCFCF77AFEF3
:10B89000040051D0FFF7E8F80022D84BFCF7B6FAC5
:10B8A00041EC190B53EC192B4FF0A040D449FCF795
:10B8B000ADFA02460B4651EC180BFCF779FB064635
:10B8C0000F4653EC192B4FF0C040CE49FCF79EFABF
:10B8D00002460B4630463946FCF76AFB06460F46E1
:10B8E00053EC192B4FF00050C749FCF78FFA024672
:10B8F0000B4630463946FCF75BFB06460F4653ECD9
:10B90000192B0020C149FCF781FA02460B4630464C
:10B910003946FCF74DFB06460F4653EC192B4FF00A
:10B920000050BB49FCF772FA02460B4630463946D6
:10B93000FCF73EFB41EC180B04F003046519BAE078
:10B9400051EC180B48004015401C51EC180B0DD160
:10B9500048004015401C02D1090340F04181BDEC74
:10B96000068B4FF0FF306FF00041F4BD21F0004135
:10B970000022914208BF904205D1002D00F0308195
:10B980009FEDBC8B2CE153EC192B9FED720B03F058
:10B99000004251EC100B0C46144353EC102B51ECAD
:10B9A000190B23460026FCF7D7FB4B0043EAD07364
:10B9B0004200B34208BFB24241EC190B19D040F229
:10B9C0003344A4EB5352352A04DB00F0000001F0AD
:10B9D00000410CE0202A03DD203AD140914000E0F4
:10B9E00001D1002003E0012AA4BFD040904041ECE7
:10B9F000190B51EC190B20F0000231F0004308BF85
:10BA0000B24251D053EC192B00207C49FCF7FEF9CF
:10BA100041EC1A0B53EC1A2B4FF0A0407849FCF77D
:10BA2000F5F902460B4651EC180BFCF7C1FA064635
:10BA30000F4653EC1A2B4FF0C0407249FCF7E6F961
:10BA400002460B4630463946FCF7B2FA06460F4628
:10BA500053EC1A2B4FF000506B49FCF7D7F9024614
:10BA60000B4630463946FCF7A3FA06460F4653EC20
:10BA70001A2B00206549FCF7C9F902460B463046EF
:10BA80003946FCF795FA06460F4653EC1A2B4FF051
:10BA900000505F49FCF7BAF902460B46304639467A
:10BAA000FCF786FA41EC180B51EC190BFCF76AFD18
:10BAB00000F00300451951EC180B21F00041002261
:10BAC0004FF07953FEF7B8FF05F0010405D2002CC2
:10BAD00000F07E809FED678B7AE053EC182B51ECE1
:10BAE000180BFCF793F9002C41EC190B36D053ECF2
:10BAF000192B48484849FCF789F9484A484BFCF754
:10BB00002BFB53EC192BFCF781F9464A464BFCF70B
:10BB100023FB53EC192BFCF779F9444A444BFCF70F
:10BB20001BFB53EC192BFCF771F9424A424BFCF713
:10BB300013FB53EC192BFCF769F96FF051023F4BE3
:10BB4000FCF70AFB53EC192BFCF760F900223C4B85
:10BB50003AE000BF000000000000E03F53EC182B6B
:10BB6000FCF754F906460F4653EC192B3548364975
:10BB7000FCF74CF9354A364BFCF7EEFA53EC192B2F
:10BB8000FCF744F9334A344BFCF7E6FA53EC192B33
:10BB9000FCF73CF9314A324BFCF7DEFA53EC192B37
:10BBA000FCF734F92F4A304BFCF7D6FA53EC192B3B
:10BBB000FCF72CF92D4A2E4BFCF7CEFA32463B46C9
:10BBC000FCF724F953EC182BFCF7C6FA41EC180BE0
:10BBD000A80705D551EC180B81F0004141EC180B7A
:10BBE00051EC180BBDEC068BF4BD000083C8C96D89
:10BBF000305FE43F0000A0FFFFFFDF410000303E68
:10BC0000FB21B941B410114026A6513E5C14D33C2F
:10BC10009A833B3B09260A1039BA213E3BA861C6EC
:10BC2000F97D92BE63AC30909F01FA3EF6FB51164F
:10BC30006CC156BFB10255555555A53FFFFFDFBF3B
:10BC40000000F03FB08F2FC310D8E53D8F0C73A1DB
:10BC5000E1E55ABE4DADE44FE31DC73E3EE3B519E5
:10BC6000A0012ABFFAF010111111813F425555551C
:10BC70005555C5BF000000000000F03F0122DBE584
:10BC80000022D9E50020704770B504000D001600B1
:10BC900006FB05F12000FFF723FDA560E66001200B
:10BCA0002061200070BD38B505000C00280000F0B0
:10BCB000F7FB00680090200000F0F2FB00682860AD
:10BCC000684600F0EDFB0068206031BD10B504004F
:10BCD000200000F0E6FB200010BD10B5040020009D
:10BCE00000F0E7FB200010BD7047704780B500F002
:10BCF000E4FB02BD0830704780B500F0E5FB02BDF3
:10BD0000001D704770B50C00150000F02EF80121E1
:10BD100000F0E3FB0600002C01D1340035003000B8
:10BD2000FFF7E5FA00F03EF80100042000F0A4F867
:10BD3000002801D0046000E000203000FFF703FB82
:10BD400000F030F80100042000F096F8002801D03F
:10BD5000056000E00020300070BD80B5FFF7CAFF2D
:10BD600002BD80B500F0BDFB02BD80B500F0BAFB9E
:10BD700002BD38B504000D001000FFF7E3FA020021
:10BD80002900200000F0AFFB31BD10B500F0B7FB7B
:10BD9000210000F0B8FB10BD80B5FFF7A0FA001D30
:10BDA00002BD704780B500F0B2FB02BD80B500F067
:10BDB000AFFB01BD80B500F0AFFB01BD38B504009D
:10BDC0000A001900200000F0ADFB200000F0B8FBD5
:10BDD0000500200000F0B8FB2860200032BD38B517
:10BDE00004000A001900200000F0B4FB2000FFF757
:10BDF0007AFA0500200000F0BBFB2860200032BD6D
:10BE00004068704770B504000D0016002000FFF771
:10BE1000F7FFA84210D100252000FFF7F1FF85426F
:10BE200014D2206800EBC50006EBC50191ED000BB4
:10BE300080ED000B6D1CEFE701212000FEF740FEB6
:10BE40000123320029002000FFF708FC70BD38B53F
:10BE50000D000100082000F00FF80400002C07D0AE
:10BE6000280000F08BFB90ED000B84ED000B00E050
:10BE7000002031BDF5F777B90800704700000000D9
:10BE8000D0B52DED048B41EC180B144653EC182B58
:10BE900000206C4900F074FB08BF9FED558B00F04B
:10BEA000838051EC180B544A544BFFF737F91DD8D7
:10BEB0009FED539B53EC182B51EC190BFBF7A6FF8E
:10BEC0000022514BFCF748F906460F4653EC182B5D
:10BED00051EC190BFCF740F902460B463046394647
:10BEE000FCF72CFA41EC180B44F0010451EC180B50
:10BEF00021F0004101224FF07953FFF70FF953D899
:10BF000053EC182B51EC180BFBF780FF41EC190B8D
:10BF100053EC182BFBF77AFF06460F4653EC192B10
:10BF20003A483B49FBF772FF3A4A3B4BFCF714F99E
:10BF300053EC192BFBF76AFF384A394BFCF70CF925
:10BF400032463B46FBF762FF53EC182BFCF704F933
:10BF500006460F4653EC192B32483349FBF756FF80
:10BF6000324A334BFCF7F8F853EC192BFBF74EFF32
:10BF7000304A314BFCF7F0F853EC192BFBF746FF36
:10BF80002E4A2F4BFCF7E8F853EC192BFBF73EFF3A
:10BF900000222C4BFCF7E0F802460B4630463946AF
:10BFA000FCF7CCF941EC180BA00705D551EC180BA8
:10BFB00081F0004141EC180B14F007020BD000BFD8
:10BFC00021A303EBC20251EC180B53681268FCF773
:10BFD000C3F841EC180B200705D551EC180B81F084
:10BFE000004141EC180B51EC180BBDEC048BD0BD9B
:10BFF000182D4454FB21E93F57CD9E5E1426D13FB6
:10C00000AA4C58E87AB6FB3F0000F0BF845D571396
:10C010004B57B03FB2934C19ED5EE43FBEDE02B920
:10C020000240F83FDE39028FC7C0743F8AAB1283EB
:10C03000000CC83F24D7E508B6D8F03F0F34580E9F
:10C040005895FD3F0000F03F000000000000000098
:10C0500066732D3852C1E03F182D4454FB21F93F3F
:10C0600066732D3852C1F03F182D4454FB21F93F1F
:10C0700066732D3852C10040182D4454FB210940ED
:10C080003FD038C6A6F10440F8B52DED0A8B41EC3F
:10C090001A0B48004015109D401C43EC182B24D06F
:10C0A00051EC1A0B21F000410022914208BF90424E
:10C0B0001BD051EC180B48004015401C15D051EC1A
:10C0C000180B31F0004108BF90420ED051EC1A0B12
:10C0D000DFF87433FEF7B0FC80F0B18051EC180B40
:10C0E0009FED870B01F00042BAE051EC1A0B4800BB
:10C0F0004015401C02D1090340F0A08151EC180BFF
:10C1000048004015401C01D109035DD151EC180BCA
:10C1100020F0000221F000430020834208BF824249
:10C1200008D151EC1A0B48004015401C4CD10903B2
:10C130004AD10DE048004015401C12D1090310D12E
:10C1400051EC1A0B48004015401C3DD109033BD16E
:10C15000FEF70CFEBDEC0A8B4FF0FF306FF0004194
:10C16000F4BD51EC1A0B21F000410022002399424A
:10C1700008BF90422BD151EC180B4800400D05EB45
:10C18000000237D151EC180B21F00041994208BF51
:10C19000984206D02A4651EC180BFEF7D7FF41EC27
:10C1A000180B51EC180B20F0000221F00043002086
:10C1B000834208BF824205D048004015401C03D18D
:10C1C000090301D1FEF7D9FD51EC180B38E151EC10
:10C1D0001A0B48004015401C2AD1090328D153EC02
:10C1E0001A2B51EC180BBDEC0A8B01B0BDE8F040E6
:10C1F000FBF70CBE002AC5DD40F2FF7082420FDB68
:10C200009FEDA50B51EC100B084653EC182B03F0D7
:10C210000041084353EC102B034643EC182BC0E7B6
:10C220006FF31E5141EA025153EC182B0B46F4E711
:10C2300051EC180B9FED320B01F0004210E001228F
:10C24000824BFEF76BFF11D89FED930B51EC100B57
:10C250000A4651EC180BFEF790FD01F00040024336
:10C2600051EC100BBDEC0A8B1146F4BD53EC1A2BAC
:10C2700077487849FBF7CAFD41EC100B53EC102BC3
:10C280009FED759B03F0004251EC190B0C461443D3
:10C2900053EC192B51EC100B2346FBF75DFFFCF719
:10C2A00071F90446FEF7E0FB41EC1B0B53EC1B2B32
:10C2B0004FF078406A49FBF7A9FD02460B4651EC66
:10C2C0001A0BFBF775FE06460F4653EC1B2B654811
:10C2D0006549FBF79BFD02460B4630463946FBF7A6
:10C2E00067FE41EC1A0B21F0004100225F4BFEF784
:10C2F000A3FB09D2B0EE48AAF0EE68AA56E000BF50
:10C30000000000000000000053EC1A2B51EC1A0B47
:10C31000FBF77CFD41EC1B0B53EC1B2B54485549A0
:10C32000FBF774FD544A554BFBF716FF53EC1B2BE0
:10C33000FBF76CFD41EC1C0B53EC1B2B5048514997
:10C34000FBF764FD504A514BFBF706FF53EC1B2BE8
:10C35000FBF75CFD53EC192BFBF7FEFE53EC1A2B9D
:10C36000FBF754FD41EC190B53EC1C2BFBF7F4FECF
:10C370009FED47AB53EC1A2BFBF7EEFE06460F463C
:10C3800051EC1C0B53EC192BFBF712FE53EC1A2B40
:10C39000FBF7E2FE02460B4630463946FBF7CEFF7E
:10C3A00053EC182BFBF732FD41EC1A0B51EC1A0B36
:10C3B0002A194800400D02EB00031DD0002B1BDDA5
:10C3C00040F2FF7083420DDB9FED330B51EC100BFD
:10C3D000084653EC1A2B03F00041084353EC102B92
:10C3E000034606E06FF31E5141EA035153EC1A2B4A
:10C3F0000B4643EC1A2B0EE051EC1A0B21F00041D6
:10C400000024A14208BFA04205D051EC1A0BFEF750
:10C410009DFE41EC1A0B51EC1A0B20F0000221F0AA
:10C4200000430020834208BF824205D048004015E7
:10C43000401C03D1090301D1FEF79FFC51EC1A0BFC
:10C44000BDEC0A8BF4BD000000C89CC000C89C4035
:10C45000FE822B654715F73F000000000000E03F1B
:10C46000422EE63FF2E4D5BCE7E84B3E0000903CAC
:10C47000112E5781A03F503F5843128C8F71BC3F03
:10C480004BE8A541B752013F0BBDF3DAE8708C3F92
:10C49000000000000000F03F000000000000F07FFE
:10C4A000704710B5040001212000FEF709FB2000B1
:10C4B00010BD80B500F074F802BD10B50400200076
:10C4C000FFF71AFC200010BD10B504002160110018
:10C4D000200000F068F8200010BD80B500F064F87E
:10C4E00002BD7047704738B504000D001000FEF71C
:10C4F00029FF02002900200000F05DF831BD80B561
:10C5000000F069F802BD80B500F066F802BD704722
:10C5100080B500F065F801BD80B50800110000F09D
:10C5200060F801BD10B50400100000F05EF80100D5
:10C53000200000F05BF8200000F05CF8200010BD47
:10C5400080B500F05CF802BD80B50022002100F04B
:10C550005AF802BD10B50400100000F07FF8010089
:10C56000200000F07CF8200000F07DF8200010BDD5
:10C5700080B500220021FFF7C5FB02BD7047000017
:10C5800090420CD141EA030C50EA4C0C07D099427E
:10C5900005D14FF4001C1CEB410F38BF8942704796
:10C5A000002101607047704780B50800012200211A
:10C5B00000F05EF802BD38B515000420FFF75CFC02
:10C5C0000400002C05D02800FEF7BCFE00682060A7
:10C5D00000E0002031BD704780B500F05BF802BD7F
:10C5E000704780B5FFF75BF801BD704780B500F07C
:10C5F00055F802BD0021016000214160704780B5FF
:10C6000000F04DF802BD70B50C00150000F048F8C0
:10C61000012100F049F80600002C01D1340035005A
:10C62000300000F045F800F047F801000420FFF763
:10C6300023FC002801D0046000E00020300000F05E
:10C640003FF800F039F801000420FFF715FC00283E
:10C6500001D0056000E00020300070BD704780B55B
:10C6600000F032F802BD00210160002141607047F6
:10C6700010B504000020002C09D00548844201D3E5
:10C68000F4F7EEFF0C2044432000FDF7FFFD10BD42
:10C690005655551500487047555555157047704704
:10C6A00080B500F012F802BD80B500F00FF802BDB1
:10C6B00080B500F012F802BD80B500F00FF802BDA1
:10C6C00080B500F00CF802BD7047704780B50800D7
:10C6D0000122002100F006F802BD70477047001DDE
:10C6E0007047000010B504000020002C09D0054858
:10C6F000844201D3F4F7B4FF0C2044432000FDF73B
:10C70000C5FD10BD565555150F003C008C0090011D
:10C71000A0006801280032002600BAFFA6FF23000F
:10C72000040025004006050003001405050007006D
:10C73000FDFF01000A000900190005001400900126
:10C740000100FEFF05005802000023000F00060054
:10C750000F003C008C009001A0006801280032000E
:10C760002600BAFFA6FF23000400250040060500AE
:10C770000300140505000700FDFF01000A00090081
:10C7800019000500140090010100FEFF0500580289
:10C79000040023000F00080011003C008C009001F1
:10C7A000A0006801280032002600BAFFA6FF23007F
:10C7B00004002500400605000300140505000700DD
:10C7C000FDFF01000A000900190005001400900196
:10C7D0000100FEFF05005802040023000F000D00B9
:10C7E0002DE9FC4D016800F10805490805EBC1027F
:10C7F000019200F10802406800F0010A02EBC10852
:10C80000400808EBC00B00200021019A95422FD070
:10C810002A68AE186A68324400920835009A964237
:10C82000F3D016F9014B009A964205D12A68AE184A
:10C830006A6832440092083516F8017B884210D1AC
:10C84000D84508BFF4F70CFFD8F80000D8F804105A
:10C85000BAF1000F18BF48440144884208F10808A3
:10C86000EED0002C00F8017B05D5641CE6D1D5E79D
:10C870005846BDE8F68D641ED5D5CFE77047FEE774
:10C88000FEE7FEE7FEE770477047704780B500F0AF
:10C890003BF801BD704780B51348FDF767F801BD4F
:10C8A00080B51248FDF762F801BD80B51048FDF76C
:10C8B0005DF801BD80B50F48FDF758F801BD80B5A2
:10C8C0000D48F7F704FE01BD80B50C48FAF738FBB8
:10C8D00001BD80B50A48F8F7E3FA01BD80B5094803
:10C8E000F8F7DEFA01BD00007023002028230020A5
:10C8F000E02200209822002050210020B4210020B6
:10C90000002200204C22002004480068044991F9CC
:10C910000010401801490860704700BF242500201E
:10C920001B01002070B504002000FFF709FE00681D
:10C93000FFF7BEFE05682000FFF702FE0068FFF764
:10C94000B7FE06002000FFF7FBFD00683060200006
:10C95000FFF7F6FD0068FFF7B3FE06002000FFF7C3
:10C96000EFFD00683060200000F013F80021016046
:10C9700008E02800FFF79CFE06682900200000F070
:10C980000DF835002000FFF7DBFD00688542F0D18F
:10C9900070BD80B5FFF733FE001D02BD70B5050008
:10C9A0000C002000FFF784FEFFF786FE2000FFF753
:10C9B00087FEFFF781FE200000F011F800F013F869
:10C9C00006002800FFF76CFE310000F010F8280088
:10C9D000FFF766FE0122210000F00DF870BD80B562
:10C9E00000F00DF802BD80B500F00BF802BD80B577
:10C9F00000F008F801BD80B500F008F801BD08306E
:10CA00007047704780B500F007F801BD80B5080099
:10CA1000110000F002F801BD704780B5FEF73FFE3F
:10CA200001BD70B504002000FEF75DFC0068FEF754
:10CA30005EFC05682000FEF756FC0068FEF757FC18
:10CA400006002000FEF74FFC006830602000FEF773
:10CA50004AFC0068FEF777FC06002000FEF743FC66
:10CA6000006830602000FFF797F90021016008E0BE
:10CA70002800FEF73CFC066829002000FEF7C9FCF0
:10CA800035002000FEF72FFC00688542F0D170BD14
:10CA90001348006850F4700011490860114800689C
:10CAA00050F001000F49086000200F4908600D4850
:10CAB00001680E4801400B4801604FF480500C495A
:10CAC00008600848006830F48020064908600020AB
:10CAD000084908605FF0006007490860704700007F
:10CAE00088ED00E00010024008100240FFFFF6EA67
:10CAF0000C1002401810024008ED00E019E050F858
:10CB0000042BD30744BFA9F101039A18091F00237E
:10CB1000042942F8043BF9D25FEA817C134604D52C
:10CB20004FF0000CA2F800C09B1CC90744BF0021B5
:10CB3000197050F8041B0029E1D17047A08601004C
:10CB4000400D0300801A060000350C0040420F0023
:10CB500080841E0000093D0000127A000024F400C9
:10CB600000366E010048E801006CDC0238B50400B4
:10CB70000D002800FFF79CFDFFF79EFD2800FFF742
:10CB80009FFDFFF799FD2000FFF78AFD0122290094
:10CB9000FFF731FF31BD38B504000D002800FEF766
:10CBA000A6FBFFF7FFF82800FEF7CDFBFFF7FAF82A
:10CBB0002000FFF7DAF801222900FFF7FBF831BD6A
:10CBC000253032642C253032642C253032642C25FB
:10CBD0003032642C253032642C253032642C2530E0
:10CBE0003264200D0A00000010B50749794418315D
:10CBF000064C7C44163404E00A68081D114488473A
:10CC00000146A142F8D110BD98000000C400000008
:10CC1000675F62547269676765724F4E203D20748A
:10CC2000727565202D2D2D2D2D2D2D2D2D2D2D0D9C
:10CC30000A0000004779726F2073656E736F72206F
:10CC4000646574656374206661696C21212121200B
:10CC5000633D2564200D0A004163747561746F7231
:10CC600020646574656374206661696C21212121EB
:10CC700020633D2564200D0A000000004EF6885117
:10CC8000CEF20001086840F470000860BFF34F8FD7
:10CC9000BFF36F8F4FF00070E1EE100A7047000095
:10CCA0005DFEFFFF2C2400001C010020000000009E
:10CCB00031FBFFFF020000000200000050030000F3
:10CCC00064000000000000201C01000005000000BE
:10CCD00010B50446044979440E31044878440C30B8
:10CCE000FAF760FB204610BD440200003802000045
:10CCF00000F00DF8002801D0FFF776FFAFF30080B9
:10CD00000020AFF30080F5F7B1F900F002F8012040
:10CD1000704700F001B800000746FAF76AFB384692
:10CD2000F4F7C4FCFBE700004C6F6164466C617370
:10CD300068446174612E2E2E2E2E2E2E2E2E2E2E17
:10CD40002E0D0A00456E746572205374616E646224
:10CD500079206D6F64652121212121200D0A0000B9
:10CD600053746172742120434C4B3D25644D487AC5
:10CD70002C205665723D2573200D0A007374616E78
:10CD80006462792068697420636F756E743D2564F0
:10CD9000200D0A00513D323B313B25642C253032B9
:10CDA000642C253033642C0A0000000010B5040008
:10CDB0002000FFF7C5FB01682000FFF7D7FE200029
:10CDC00010BD10B504002000FEF78DFA01682000A8
:10CDD000FFF7E1FE200010BD566572303331375F3A
:10CDE0003230323630333133000000003C72730091
:10CDF00074002D00630031002E00353C0D0A000048
:10CE00000D0A5B416E64726F6964204150505D2170
:10CE10000D0A00003C74720000005F006A002D00E3
:10CE200073002D3C0D0A000010B50400200000F036
:10CE300005F8200000F006F8200010BD80B5FFF7CF
:10CE400071FD01BD80B500F001F802BD10B5040010
:10CE5000200000F002F8200010BD80B5FFF7A6FF0B
:10CE600002BD10B50400200000F005F8200000F01D
:10CE700006F8200010BD80B5FFF7D3FD01BD80B5D9
:10CE800000F001F802BD10B50400200000F002F827
:10CE9000200010BD80B5FFF794FF02BD457261739D
:10CEA0006572204572726F720D0A000054726967D4
:10CEB0006765723D2564200D0A0000006779726F76
:10CEC0002049443D30782578200D0A0000000000FC
:10CED000000000000102030406070809014880471A
:10CEE0000148004791CA000811CF000862617474BC
:10CEF0003D2564200D0A000041542B53484F570D27
:10CF00000000000041542B444154413D310D0000CC
:10CF1000AFF30080FFF7B2FEFFF7EAFE000000006B
:10CF2000010203049181FFFF9947FFFF00002E00DB
:10CF3000FFF7FEBFFFF7FEBFFFF7FEBFFFF7FEBF25
:10CF4000FFF7FEBFFFF7FEBFFFF7FEBFFFF7FEBF15
:10CF5000FFF7FEBFFFF7FEBFFFF7FEBFFFF7FEBF05
:10CF6000FFF7FEBFFFF7FEBFFFF7FEBFFFF7FEBFF5
:10CF7000FFF7FEBFFFF7FEBFFFF7FEBFFFF7FEBFE5
:10CF8000FFF7FEBFFFF7FEBFFFF7FEBFFFF7FEBFD5
:10CF9000FFF7FEBFFFF7FEBFFFF7FEBFFFF7FEBFC5
:10CFA000FFF7FEBFFFF7FEBFFFF7FEBFFFF7FEBFB5
:10CFB000FFF7FEBFFFF7FEBFFFF7FEBFFFF7FEBFA5
:10CFC000FFF7FEBFFFF7FEBFFFF7FEBFFFF7FEBF95
:10CFD000FFF7FEBFFFF7FEBFFFF7FEBFFFF7FEBF85
:10CFE000FFF7FEBFFFF7FEBFFFF7FEBFFFF7FEBF75
:10CFF000FFF7FEBFFFF7FEBFFFF7FEBFFFF7FEBF65
:10D00000FFF7FEBFFFF7FEBFFFF7FEBF0331320D94
:10D010000A84001B2CCF00082CCF00082CCF00085E
:10D020002CCF00082CCF00082CCF00082CCF0008F4
:10D03000F8FF0B2ECF00082CCF00082CCF0008FAE9
:10D04000FFEE000001EF000520410000FA43F00070
:10D05000003CF2000D3E0D0A0000D8CD000880BB58
:10D06000000014FD000010FC0003093D00D0FD018C
:040000050800CF110F
:00000001FF
